:100000001CC200004BC2000049C2000047C20000F1
:1000100045C2000043C2000041C200003FC20000D0
:100020003DC200000C941F460C941F460C941F46C2
:1000300035C200000C94294631C200002FC20000D6
:100040002DC200002BC2000029C2000027C2000000
:1000500025C2000023C2000021C200000C94A13A76
:100060001DC200000C944F390C94263917C20000B1
:1000700015C2000013C2000011C200000FC2000030
:100080000DC200000BC2000009C2000007C2000040
:1000900005C2000003C2000001C200000C943D47ED
:1000A000FDC10000FBC10000F9C10000F7C1000064
:1000B000F5C10000F3C10000F1C10000EFC1000074
:1000C000EDC10000EBC10000E9C100000C94FD3857
:1000D0000C94D438E3C100000C94AB380C948238F3
:1000E000DDC10000A51E5E1F7520CE23232B5C22E0
:1000F00071227522232B7A22CE23E723FC2393251A
:10010000A9263027E8277C28AF29E82A70357335DF
:10011000623566356C35AA3577357B358135853561
:1001200089358F3593359735AA359D35A135A53558
:10013000084AD73B3BCE016E84BCBFFDC12F3D6C4E
:1001400074319ABD56833DDA3D00C77F11BED9E4B4
:10015000BB4C3E916BAAAABE000000803F076342E1
:1001600036B79BD8A71A39685618AEBAAB558C1D4E
:100170003CB7CC5763BD6DEDFD753EF6177231BFD0
:10018000000000803F08000000BE922449123EABF0
:10019000AAAA2ABECDCCCC4C3E00000080BEABAAA1
:1001A000AAAA3E00000000BF000000803F0000003F
:1001B0000000084178D3BB4387D1133D190E3CC3DF
:1001C000BD4282AD2B3E68EC8276BED98FE1A93E5E
:1001D0004C80EFFFBE01C4FF7F3F00000000000025
:1001E0004E414E494E495459494E46CDCCCC3D0A1C
:1001F000D7233C17B7D13877CC2B329595E6241FFF
:10020000B14F0A000020410000C84200401C4620B7
:10021000BCBE4CCA1B0E5AAEC59D7400407A10F38A
:100220005A00A0724E18090010A5D4E80000E87624
:1002300048170000E40B54020000CA9A3B0000007B
:10024000E1F505000080969800000040420F000094
:1002500000A08601000000102700000000E8030055
:100260000000006400000000000A0000000000011F
:1002700000000000002C76D888DC674F0823DFC11F
:10028000DFAE59E1B1B796E5E3E453C63AE65199DA
:100290007696E8E6C28426EB898C9B62ED407C6F03
:1002A000FCEFBC9C9F40F2BAA56FA5F490055A2ABA
:1002B000F75C936B6CF9676DC11BFCE0E40D47FEC6
:1002C000F520E6B500D0ED902E03009435770500BB
:1002D00080841E080000204E0A000000C80C333342
:1002E00033330F986E12831141EF8D2114893BE651
:1002F0005516CFFEE6DB18D1844B381BF77C1D90DA
:100300001DA4BBE424203284725E228100C9F12442
:10031000ECA1E53D2700002100240027002A002D44
:10032000003000330001010000040107010A010050
:10033000002200250028002B002E0031003400028E
:10034000010000050108010B010000200023002628
:100350000029002C002F00320000010000030106DC
:10036000010901050505050705080808080202023C
:10037000020A0A0808040404040101010101010140
:10038000010303030303030303040707070C0C0C17
:100390000C0C0C0C0C0202020206060606060606EF
:1003A000060B0B0B0B0B0B0B0B010210202008088C
:1003B00010204010204080020102010804020101C7
:1003C00002040810204080804020100804020180B0
:1003D0000402018040201008040201080402010107
:1003E0000204081020408001020408102040800010
:1003F000000A0B02090C0D0E08070304010000009F
:1004000000000000000000000000000000000000EC
:1004100000000000000000000000001211100000A9
:1004200000000000000000000000000000000000CC
:10043000000000000000EA59CE5911241FBECFEF82
:10044000D1E2DEBFCDBF00E00CBF1FE0A0E0B2E014
:10045000E6EFF0ED00E00BBF02C007900D92A43B69
:10046000B107D9F725E1A4EBBFE001C01D92A0368A
:10047000B207E1F712E0CCE1D2E000E006C021973C
:100480000109802FFE010E94BB65CB31D10780E0BE
:100490000807A9F70E943E500C946A68B1CD3F92BC
:1004A0004F925F926F927F928F929F92AF92BF9284
:1004B000CF92DF92EF92FF920F931F93CF93DF9330
:1004C000CDB7DEB7EF970FB6F894DEBF0FBECDBF46
:1004D0008EEC9FE00E949317892B09F46EC280EE88
:1004E00094E10E9418460E946E4860E080E00E94FD
:1004F000522D0E94953A28EE33E040E050E00E94F1
:100500004962BA01A9012AE0CE0101960E94103782
:10051000BE016F5F7F4FCE0182960E94933762E4E7
:1005200074E0CE0182960E943D36BC0180EE94E1DB
:100530000E94B637CE0182960E94DC36CE0101962B
:100540000E94DC364091D20F5091D30F6091D40FAE
:100550007091D50F20E188E892E10E94D93788E8B0
:1005600092E10E946E388091D20F9091D30FA091AA
:10057000D40FB091D50F883025E09207A105B105C1
:1005800009F4F8C108F08DC08934E1E09E07A105A7
:10059000B10509F4F2C1E0F5843421E09207A10528
:1005A000B10509F4DBC1E8F48134E1E09E07A1055F
:1005B000B10509F4C4C138F480349140A105B105F6
:1005C00009F4AEC1DDC1823441E09407A105B10553
:1005D00009F4BEC183349140A105B10509F4BBC142
:1005E000CFC18634F1E09F07A105B10509F4BCC174
:1005F00008F4B7C1873441E09407A105B10509F4B7
:10060000B6C188349140A105B10509F4B3C1B8C1A0
:100610008230F5E09F07A105B10509F499C1E8F41E
:10062000843741E09407A105B10509F444C138F4C9
:1006300082379140A105B10509F448C1A1C18115D6
:1006400025E09207A105B10509F46AC18130954002
:10065000A105B10509F473C193C18530E5E09E079A
:10066000A105B10509F47DC170F4833025E092073E
:10067000A105B10509F46FC184309540A105B1050C
:1006800009F46CC17DC18630E5E09E07A105B10586
:1006900009F46AC187309540A105B10509F467C125
:1006A0006FC18D3B22E492072FEFA207B10509F439
:1006B00028C108F04BC08F3EE0E19E07EFEFAE0788
:1006C000B10509F454C118F5823325E09207A1055C
:1006D000B10509F4FBC038F489309540A105B10596
:1006E00009F44BC14DC18433F5E09F07A105B10565
:1006F00009F4E1C08D3F9240AF4FB10509F040C110
:1007000060E174E081E294E10E947936DCC08D3DC5
:1007100042E294074FEFA407B10509F4CCC038F4C6
:10072000873E9841AF4FB10509F41BC129C18F3CE9
:1007300020E392072FEFA207B10509F40FC1873C10
:100740009843AF4FB10509F415C11AC18739E8E6DE
:100750009E07EFEFAE07B10509F4F1C048F58D3AF9
:1007600022E592072FEFA207B10509F4BBC038F4C8
:10077000853B9A44AF4FB10509F4D2C001C1853A17
:10078000FAE59F07FFEFAF07B10509F4F6C08D3911
:100790009246AF4FB10509F0F3C06DE074E081E21D
:1007A00094E10E947936109232108CEF9FEF80C056
:1007B000873548EA94074FEFA407B105F9F078F4BC
:1007C0008538FAE79F07FFEFAF07B10509F4CCC002
:1007D00087369849AF4FB10509F4BAC0D1C08F34FC
:1007E00040EB94074FEFA407B10509F4B4C08D3373
:1007F000924CAF4FB10509F469C0C2C082E080934A
:1008000031131092341300E010E084EB9FE00E945B
:100810009317892B69F40F5F1F4F093EF3E01F0701
:1008200039F06EE170E080E090E00E945D3AEDCF3B
:1008300061ED77E088E892E10E9481384091B80F3D
:100840005091B90F6091BA0F7091BB0F2AE088E800
:1008500092E10E94D93788E892E10E946E38809137
:10086000B80F9091B90FA091BA0FB091BB0F823021
:10087000E5E09E07A105B10509F4B1C108F0B2C1D8
:10088000833421E09207A105B10509F4B9C108F04C
:10089000BAC18134E1E09E07A105B10509F099C113
:1008A0006AE074E08BE194E10E94793689EF9FEF72
:1008B0000E944B1E7CC060E174E081E294E10E94E2
:1008C0007936109232108BEF9FEFF2CF63E174E034
:1008D00081E294E10E94793681E0809332108DEFBD
:1008E0009FEFE6CF66E174E08BE194E10E947936F8
:1008F00066E174E081E294E10E9479368EEF9FEF29
:10090000D7CF69E174E08BE194E10E94793669E127
:1009100074E081E294E10E9479368FEF9FEFC8CFB7
:1009200069E278E08BE194E10E94793669E278E04F
:1009300081E294E10E94793680E090E0B9CF6AE1EB
:1009400074E08BE194E10E94793681E090E0B0CFD1
:1009500082E090E0ADCF83E090E0AACF84E090E029
:10096000A7CF85E090E0A4CF86E090E0A1CF87E01C
:1009700090E09ECF88E090E09BCF89E090E098CF18
:1009800060E070E0CE0101960E94F643BE016F5F09
:100990007F4F8BE194E10E94A336CE0101960E9425
:1009A000DC3664E670E080E090E00E945D3A82E030
:1009B0008093311310923413CFC065E97EE081E259
:1009C00094E10E9479361092C50F65E97EE081E2DC
:1009D00094E10E94793611E088E892E10E9478342F
:1009E0002091C50F181619060CF038C1211136C117
:1009F000B1C14091000250910102609102027091D8
:100A0000030222E0CE0182960E94E13664E175E0A5
:100A1000CE0101960E949B37BE016E5D7F4FCE01D5
:100A200001960E94543662E474E00E943D36BC0197
:100A3000CE0188960E949337CE0188960E94F63D9B
:100A4000CE0188960E94DC36CE0101960E94DC36EB
:100A5000CE0182960E94DC3640910C0250910D022C
:100A600060910E0270910F0222E0CE0182960E94E8
:100A7000E13664E275E0CE0101960E949B37BE012B
:100A80006E5D7F4FCE0101960E94543662E474E0A1
:100A90000E943D36BC01CE0188960E949337CE015C
:100AA00088960E94F63DCE0188960E94DC36CE01E3
:100AB00001960E94DC36CE0182960E94DC3680EEE2
:100AC00094E10E9418460E946E4860E080E00E9417
:100AD000522D0E94953A28EE33E040E050E00E940B
:100AE0004962BA01A9012AE0CE0101960E9410379D
:100AF000BE016F5F7F4FCE0182960E94933762E402
:100B000074E0CE0182960E943D36BC0180EE94E1F5
:100B10000E94B637CE0182960E94DC36CE01019645
:100B20000E94DC3680912514909126148330910523
:100B300008F04DC58130910509F0DCC4E091211425
:100B4000F0912214309711F40C946E17F0808F2DD1
:100B50000E94F14E0E94953A0E94953A6093CA0F06
:100B60007093CB0F8093CC0F9093CD0F24C08091C6
:100B7000321081110C9418170E94953A0091CA0FF7
:100B80001091CB0F2091CC0F3091CD0FDC01CB0118
:100B9000801B910BA20BB30B88349E4EA105B105AF
:100BA00050F06091F0146B7F6093F014686080EEF9
:100BB00094E10E94164680913210882311F40C941F
:100BC0007B1764E670E080E090E00E945D3A0C9450
:100BD0007B1782349140A105B10509F0E8CE88EF7A
:100BE0009FEF66CE8F3CE0E39E07EFEFAE07B105C7
:100BF00081F0F8F4833025E09207A105B10599F45E
:100C000087EF9FEF55CE843421E09207A105B1050F
:100C100019F486EF9FEF4CCE81309540A105B105C8
:100C200009F43ECEC4CE84309540A105B10589F3C8
:100C3000BECE8736E8E99E07EFEFAE07B10579F241
:100C40008F34F0EB9F07FFEFAF07B105C9F287398B
:100C50009846AF4FB10509F0AACE22CE222361F00B
:100C60002091C50F80912514909126142111A6C0C2
:100C7000009709F0A3C0E2C000E010E0EE24E39486
:100C80008EE491E10E94783418161906D4F58EE4AA
:100C900091E10E9456348093C40F8A30A1F08D30C8
:100CA00091F09091C50F91110EC089831A8241E095
:100CB00050E0BE016F5F7F4F81E294E10E941036E9
:100CC0000F5F1F4F17C08091251490912614892B18
:100CD00089F0E092C50F8EE491E10E9478341816F5
:100CE000190644F465E97EE081E294E10E947936D8
:100CF0001092C50F6FE070E080E090E00E945D3AD6
:100D0000BFCF62E370E080E090E00E945D3A012B8B
:100D100009F4A6CF65E274E0CE0101960E949B37EC
:100D200061E274E1CE0101960E945436BC0188E86C
:100D300092E10E947138CE0101960E94DC368EE469
:100D400091E10E94063564E670E080E090E00E9448
:100D50005D3A86CF88E892E10E9456348093C40FB2
:100D60008A3071F08D3061F089831A8241E050E061
:100D7000BE016F5F7F4F81E294E10E94103617C081
:100D80001093C50F6CE174E0CE0101960E949B3771
:100D900061E274E1CE0101960E945436BC0188E8FC
:100DA00092E10E947138CE0101960E94DC366AE021
:100DB00070E080E090E00E945D3A0ECE019709F06D
:100DC00058C062E474E0CE0101960E949B37CE01C8
:100DD00001960E94C233811112C06AE274E0CE0112
:100DE00082960E949B37CE0182960E94C23311E008
:100DF000811110E0CE0182960E94DC3601C010E025
:100E0000CE0101960E94DC36112389F060E070E08B
:100E1000CE0101960E94F643BE016F5F7F4F8BE1CA
:100E200094E10E94A336CE0101960E94DC3664E173
:100E300070E080E090E00E945D3A1BC064E670E0E4
:100E400080E090E00E945D3A0E94953ACB0168EE06
:100E500073E00E94A865CB0164E670E00E94A8657B
:100E60008236910534F080913210882311F40C946D
:100E70005F176AE070E080E090E00E945D3A809148
:100E8000251490912614009711F40C94F3160197F1
:100E9000E1F56CE274E0CE0188960E949B37CE01AA
:100EA00088960E94C23381110C9475176EE274E02B
:100EB000CE0182960E949B37CE0182960E94C23359
:100EC000811112C06EE979E0CE0101960E949B3734
:100ED000CE0101960E94C23311E0811110E0CE01D3
:100EE00001960E94DC3601C010E0CE0182960E947D
:100EF000DC36CE0188960E94DC36112331F061E2A7
:100F000074E18BE194E10E948E36809125149091DA
:100F100026140497D8F563E279E0CE0101960E9489
:100F20009B37CE0101960E94C233182FCE01019645
:100F30000E94DC36112351F161E070E0CE01019690
:100F40000E94F643CE0101960E9405360AEF1FEF7C
:100F50002FEF3FEF58016901A61AB70AC80AD90A4C
:100F6000B601A5012AE0CE0182960E943C37BE015F
:100F70006E5D7F4F8BE194E10E94A336CE01829695
:100F80000E94DC36CE0101960E94DC3660E374E0FC
:100F9000CE0182960E949B37CE0182960E94C23378
:100FA000811113C064E374E0CE0101960E949B3767
:100FB000CE0101960E94C23311E0811101C010E000
:100FC000CE0101960E94DC3601C011E0CE0182966E
:100FD0000E94DC36112309F472CD68E374E0CE017F
:100FE00001960E949B37CE0101960E94F63DCE01EC
:100FF00001960E94DC36609147037091480380910E
:10100000490390914A030E94F16020E030E048ECEF
:1010100052E40E944163AB01BC0122E0CE01829602
:101020000E94E13664E474E0CE0101960E949B3791
:10103000BE016E5D7F4FCE0101960E94543665E67B
:1010400075E00E943D36BC01CE0188960E94933720
:10105000CE0188960E94F63DCE0188960E94DC362D
:10106000CE0101960E94DC36CE0182960E94DC36CB
:1010700040914303509144036091450370914603AE
:1010800022E0CE0182960E94E13669E574E0CE014D
:1010900001960E949B37BE016E5D7F4FCE01019687
:1010A0000E945436BC01CE0188960E949337CE012F
:1010B00088960E94F63DCE0188960E94DC36CE01CD
:1010C00001960E94DC36CE0182960E94DC36409169
:1010D0003F0350914003609141037091420322E02D
:1010E000CE0182960E94E13666E774E0CE01019659
:1010F0000E949B37BE016E5D7F4FCE0101960E941C
:101100005436BC01CE0188960E949337CE01889652
:101110000E94F63DCE0188960E94DC36CE010196F3
:101120000E94DC36CE0182960E94DC3640914B0351
:1011300050914C0360914D0370914E0322E0CE011B
:10114000C4960E94E1364091570350915803609134
:10115000590370915A0323E0CE018E960E94E13626
:1011600040914F035091500360915103709152038D
:1011700022E0CE0188960E94E136409153035091BF
:101180005403609155037091560323E0CE0182967B
:101190000E94E13666E874E0CE0101960E949B371A
:1011A000BE016E5D7F4FCE0101960E9454366BE901
:1011B00074E00E943D36BE01685D7F4F0E94543648
:1011C0006EE974E00E943D36BE01625D7F4F0E9471
:1011D00054366BE974E00E943D36BE016C5C7F4F73
:1011E0000E94543664EA74E00E943D36BC01CE0190
:1011F000CA960E949337CE01CA960E94F63DCE0150
:10120000CA960E94DC36CE0101960E94DC36CE01E1
:1012100082960E94DC36CE0188960E94DC36CE0192
:101220008E960E94DC36CE01C4960E94DC3669EAB6
:1012300074E0CE0101960E949B376AED74E1CE0105
:1012400001960E945436BC01CE0182960E949337CB
:10125000CE0182960E94F63DCE0182960E94DC3637
:10126000CE0101960E94DC3640919803509199037B
:1012700060919A0370919B0323E0CE0188960E94AF
:10128000E136209190033091910340919203509167
:10129000930360E070E080E291E40E94EF641BA29F
:1012A0001AA21DA21CA21FA21EA28E010F5F1F4F19
:1012B00021E043E00E94235CBC01CE0182960E94A3
:1012C00079366AEB74E0C8010E949B37BE016E5DFF
:1012D0007F4FC8010E9454366DEC74E00E943D3689
:1012E000BE01685D7F4F0E94543663ED74E00E943A
:1012F0003D36BC01CE018E960E949337CE018E966C
:101300000E94F63DCE018E960E94DC36C8010E94F6
:10131000DC36CE0182960E94DC36CE0188960E9491
:10132000DC3640919403509195036091960370913F
:10133000970323E0CE0188960E94E13620918C032A
:1013400030918D0340918E0350918F0360E070E0E7
:1013500080E291E40E94EF641BA21AA21DA21CA2CB
:101360001FA21EA221E043E00E94235CBC01CE012B
:1013700082960E94793666ED74E0C8010E949B3720
:10138000BE016E5D7F4FC8010E9454366DEC74E063
:101390000E943D36BE01685D7F4F0E94543663ED6A
:1013A00074E00E943D36BC01CE018E960E949337B8
:1013B000CE018E960E94F63DCE018E960E94DC36BE
:1013C000C8010E94DC36CE0182960E94DC36CE0136
:1013D00088960E94DC3640913B0350913C0360911B
:1013E0003D0370913E0322E0CE0182960E94E136D9
:1013F00069EE74E0C8010E949B37BE016E5D7F4FAD
:10140000C8010E9454366FEF74E00E943D36BC0163
:10141000CE0188960E949337CE0188960E94F63DB1
:10142000CE0188960E94DC36C8010E94DC36CE01CF
:1014300082960E94DC36BBE2CB2EB3E0DB2E01E0CD
:1014400010E08FE0E82E8091290390912A03801705
:1014500091070CF4CECAD601AD90BD906D014AE063
:10146000B501CE0188960E9468374AE0B801CE01E6
:1014700082960E94683766E075E0CE0101960E9470
:101480009B37BE016E5D7F4FCE0101960E945436A0
:1014900069E97FE00E943D36BE01685D7F4F0E9492
:1014A00054366EE075E00E943D36EA9CB001EB9C3C
:1014B000700D1124605F7D4F0E943D36BC01CE014E
:1014C0008E960E949337CE018E960E94F63DCE01F5
:1014D0008E960E94DC36CE0101960E94DC36CE014B
:1014E00082960E94DC36CE0188960E94DC360F5F21
:1014F0001F4FA9CF029709F02ACB63E279E0CE0112
:1015000001960E949B37CE0101960E94C233182F8C
:10151000CE0101960E94DC36112309F418CB80918C
:10152000251490912614029740F0E0912114F09137
:101530002214309711F0818101C080E01A82198253
:101540001C821B821E821D828AA31BA2BE016E5DAD
:101550007F4FCE0101960E947936BE016F5F7F4FAB
:101560008BE194E10E94A336CE0101960E94DC3605
:101570008091251490912614892B41F0E09121143B
:10158000F0912214309711F0F08001C0F12C6FE13E
:1015900075E0CE0101960E949B3761E274E1CE01B5
:1015A00001960E94543662E77FE00E943D36BC01FE
:1015B00088E892E10E94B637CE0101960E94DC369F
:1015C0006BE174E188E892E10E947138C0CA41E0A1
:1015D00050E060E070E0CE0101960E94B443BE018D
:1015E0006F5F7F4F89E094E10E94A336CE010196A0
:1015F0000E94DC3661E675E0CE0182960E949B3740
:10160000CE0182960E94C233811113C06AE979E04B
:10161000CE0101960E949B37CE0101960E94C233F3
:1016200011E0811101C010E0CE0101960E94DC366C
:1016300001C011E0CE0182960E94DC36112309F42C
:10164000CEC062E070E0CE0101960E94F643BE017A
:101650006F5F7F4F89E094E10E94A336CE0101962F
:101660000E94DC3669E074E188E892E10E947138FA
:101670000E94325020E030E048EC52E40E94506179
:101680000E94DA63AB01BC014093470350934803C7
:101690006093490370934A032AE030E088E892E1BE
:1016A0000E94213888E892E10E946E3860914703D9
:1016B000709148038091490390914A038B019C01EA
:1016C00000591F452140310901341C4921053105CC
:1016D000D0F064E375E0CE0101960E949B3769E08B
:1016E00074E1CE0101960E94543667E475E00E94D1
:1016F0003D36BC018FE094E10E948E36CE0101960A
:101700000E94DC364DC019821A821B821C821D8207
:101710001E821F8218860E94F16020E030E048ECB3
:1017200052E40E9441638E010F5F1F4F22E047E0A9
:101730000E94235CBC018FE094E10E94793667E54A
:1017400075E0CE0182960E949B376FE074E1CE0176
:1017500082960E94543664E675E00E943D36BC01D4
:101760008FE094E10E948E36CE0182960E94DC3694
:1017700010923110109230108091470390914803DD
:10178000A0914903B0914A038093B4109093B5108F
:10179000A093B610B093B71080E090E00E94674429
:1017A0006CE075E0CE0101960E949B376FE074E11A
:1017B000CE0101960E945436BC01CE0182960E9451
:1017C0009337CE0182960E94F63DCE0182960E940A
:1017D000DC36CE0101960E94DC3610E001C011E03B
:1017E00069E675E0CE0182960E949B37CE01829613
:1017F0000E94C233811113C06FE675E0CE010196DD
:101800000E949B37CE0101960E94C23301E08111F4
:1018100001C000E0CE0101960E94DC3601C001E06B
:10182000CE0182960E94DC36002309F4FDC046E01A
:1018300050E065E070E0CE0101960E94B443BE0125
:101840006F5F7F4F89E094E10E94A336CE0101963D
:101850000E94DC3689E094E10E9405362B013C01B0
:101860006DEF74E0CE0101960E949B3780912514A4
:10187000909126142D813E817C01E21AF30A2115F4
:10188000310559F1009749F18217930730F1E816B5
:10189000F90620F07C01E1E0EE1AF108C090211475
:1018A000D090221489809A80C60133243A940FEF95
:1018B0005601AE0CBF1CA816B90690F0B4010E94E8
:1018C0005068009769F09C012C193D09E216F30657
:1018D00010F0322E032F0196EECF6FEF7FEF02C094
:1018E000632D702F6F5F7F4FCE0182960E94F6436B
:1018F000BE016E5D7F4F89E094E10E94A336CE0168
:1019000082960E94DC36CE0101960E94DC3689E088
:1019100094E10E940536F201EE0FFF1FE75DFC4FD8
:1019200071836083FCE14F0E511C9201220F331F23
:10193000F901EC54FF4E718360836090290370902D
:101940002A03C0902303D090240340912503509193
:101950002603809027039090280360919C03709148
:101960009D034090210350902203E0901F03F090CC
:101970002003ECEBF3E0ABE2AA2EA3E0BA2E21E0C9
:1019800030E06216730654F1D5018D919D915D0191
:101990008430910519F48280938018C08A309105B3
:1019A00019F44281538112C08530910519F4C28027
:1019B000D38010C08630910519F4628173810AC00A
:1019C0008730910519F44280538004C00B9714F0BE
:1019D000E280F3802F5F3F4F3296D3CFD092240323
:1019E000C0922303F0922003E0921F03509222033F
:1019F0004092210370939D0360939C0350932603B0
:101A000040932503909228038092270361E274E1BA
:101A100088E892E10E9471381092311010923010D3
:101A200080E090E00E94674465E775E0CE01829611
:101A30000E949B37CE0182960E94C233811113C04F
:101A400069E775E0CE0101960E949B37CE010196B1
:101A50000E94C23301E0811101C000E0CE01019675
:101A60000E94DC3601C001E0CE0182960E94DC3685
:101A7000002309F472C063E070E0CE0101960E9479
:101A8000F643BE016F5F7F4F89E094E10E94A33669
:101A9000CE0101960E94DC3669E074E188E892E1AB
:101AA0000E947138109231101092301069E074E188
:101AB0008AED94E10E948E3680ED90E1892BE1F071
:101AC0000091DE141091DF140115110519F4109224
:101AD000D01012C00730110510F007E010E060913F
:101AE000DA147091DB14A80180ED90E10E94416846
:101AF000F801E053FF4E1082809130109091311028
:101B00000E9467446DE775E0CE0182960E949B3784
:101B10006AED74E1CE0182960E945436BC01CE017A
:101B200001960E949337CE0182960E94DC36BE0158
:101B30006F5F7F4F8EE491E10E94B63768EB7BE0E8
:101B400080E090E00E945D3A80ED90E10E940C43BD
:101B5000CE0101960E94DC3610E065E875E0CE010A
:101B600082960E949B37CE0182960E94C2338111D9
:101B700013C069E875E0CE0101960E949B37CE0143
:101B800001960E94C23301E0811101C000E0CE0144
:101B900001960E94DC3601C001E0CE0182960E94CF
:101BA000DC36002309F4D5C063E070E0CE01019675
:101BB0000E94F643BE016F5F7F4F89E094E10E946F
:101BC000A336CE0101960E94DC360E9432506B0192
:101BD0007C0110923110109230100E947B2B909358
:101BE0002D1080932C10892BC9F16DE875E0CE0182
:101BF00001960E949B37CE0101960E94E24ECE01D3
:101C000001960E94DC3669E074E1CE0101960E94E3
:101C10009337CE0101960E94F63DCE0101960E94B7
:101C2000DC366EEA75E0CE0101960E949B37CE014C
:101C300001960E94F63DCE0101960E94DC3660912D
:101C40003F037091400380914103909142030E94B1
:101C50007B2B90932D1080932C107AC060E070E065
:101C600082E090E00E94662B80E090E090932D103F
:101C700080932C10892B59F16BE076E0CE01019610
:101C80000E949B37CE0101960E94E24ECE01019642
:101C90000E94DC3669E074E1CE0101960E94933720
:101CA000CE0101960E94F63DCE0101960E94DC36DF
:101CB0006EEA75E0CE0101960E949B37CE01019637
:101CC0000E94F63DCE0101960E94DC3641C0C092D2
:101CD0003F03D0924003E0924103F09242036CE351
:101CE00076E0CE0101960E949B37CE0101960E94BC
:101CF000E24ECE0101960E94DC3640913F035091A6
:101D00004003609141037091420322E0CE010196AD
:101D10000E94E136CE0101960E94F63DCE01019669
:101D20000E94DC3680913F0390914003A0914103D3
:101D3000B09142038093BC109093BD10A093BE104D
:101D4000B093BF1080913010909131100E94674481
:101D500010E060E576E0CE0182960E949B37CE01CE
:101D600082960E94C233811113C065E576E0CE01F0
:101D700001960E949B37CE0101960E94C23301E07A
:101D8000811101C000E0CE0101960E94DC3601C045
:101D900001E0CE0182960E94DC36002309F43FC0A8
:101DA00064E070E0CE0101960E94F643BE016F5FD1
:101DB0007F4F89E094E10E94A336CE0101960E94F4
:101DC000DC366AE576E0CE0182960E949B3769E0B8
:101DD00074E1CE0182960E945436BC01CE01019678
:101DE0000E949337CE0182960E94DC36BE016F5F5F
:101DF0007F4F8EE491E10E94B63768EB7BE080E094
:101E000090E00E945D3ABE016F5F7F4F88E892E1EB
:101E10000E947138CE0101960E94DC3610E061E626
:101E200076E0CE0188960E949B37CE0188960E946C
:101E3000C23381112BC064E676E0CE0182960E9407
:101E40009B37CE0182960E94C233811113C067E690
:101E500076E0CE0101960E949B37CE0101960E944A
:101E6000C23301E0811101C000E0CE0101960E9461
:101E7000DC3601C001E0CE0182960E94DC36CE0144
:101E800088960E94DC36011105C020C1CE018896DB
:101E90000E94DC368AE0A82EB12CC12CD12C760110
:101EA00088248A9493E0992E6EE170E080E090E0BF
:101EB0000E945D3A809123030E94133AB4010E946C
:101EC000A865072E000C880B990B0E94F16020E09A
:101ED00030E040EA50E40E9450619B01AC01C70130
:101EE000B6010E947B626B017C01B1E0AB1AB108C4
:101EF000D9F620E030E040E251E40E9441636B01FA
:101F00007C016AE676E0CE0182960E949B37CE0184
:101F100082960E94C2338111E4C76EE676E0CE015C
:101F200001960E949B37CE0101960E94C23301E0C8
:101F3000811101C000E0CE0101960E94DC36CE0185
:101F400082960E94DC36002309F43FC020E030E096
:101F500040E650E4C701B6010E9450619B01AC010C
:101F600060E070E080E890E40E947A62AB01BC011E
:101F70004093040250930502609306027093070297
:101F800022E0CE0101960E94E136BE016F5F7F4FD5
:101F90008FE094E10E94A336CE0101960E94DC36C8
:101FA00062E776E0CE0101960E949B376FE074E114
:101FB000CE0101960E945436BC018FE094E10E944C
:101FC0008E36CE0101960E94DC3661E876E0CE01C5
:101FD00082960E949B37CE0182960E94C233811165
:101FE00082C766E876E0CE0101960E949B37CE015B
:101FF00001960E94C23301E0811101C000E0CE01D0
:1020000001960E94DC36CE0182960E94DC360023C7
:1020100009F43FC020E030E040E650E4C701B601DB
:102020000E9450619B01AC0160E070E080E291E4AD
:102030000E947A62AB01BC014093080250930902EE
:1020400060930A0270930B0222E0CE0101960E9477
:10205000E136BE016F5F7F4F8FE094E10E94A336AF
:10206000CE0101960E94DC366BE876E0CE01019647
:102070000E949B376FE074E1CE0101960E945436B6
:10208000BC018FE094E10E948E36CE0101960E9441
:10209000DC366CE075E0CE0101960E949B376FE064
:1020A00074E1CE0101960E945436BC01CE018296A5
:1020B0000E949337CE0182960E94F63DCE01829611
:1020C0000E94DC36CE0101960E94DC366BE976E098
:1020D000CE0101960E949B37CE0101960E94C23329
:1020E000082FCE0101960E94DC36002309F469C056
:1020F0008091251490912614079708F462C066E039
:1021000070E0CE0101960E94F643BE016F5F7F4FE3
:1021100089E094E10E94A336CE0101960E94DC364C
:102120000E943250AB01BC01409300025093010267
:10213000609302027093030221E0CE0182960E9416
:10214000E13664E175E0CE0101960E949B37BE0145
:102150006E5D7F4FCE0101960E94543662E474E0BA
:102160000E943D36BC018FE094E10E948E36CE0184
:1021700001960E94DC36CE0182960E94DC366FE02A
:1021800074E1CE0101960E949337CE0101960E9420
:10219000F63DCE0101960E94DC360E94953A28EE6B
:1021A00033E040E050E00E944962CA01B9010E9458
:1021B000EF606093C60F7093C70F8093C80F909322
:1021C000C90F62EA76E0CE0101960E949B37CE01EC
:1021D00001960E94C233082FCE0101960E94DC3680
:1021E000002309F456C08091251490912614079776
:1021F00008F44FC066E070E0CE0101960E94F643FD
:10220000BE016F5F7F4F89E094E10E94A336CE014B
:1022100001960E94DC360E943250AB01BC01409313
:102220000C0250930D0260930E0270930F0221E096
:10223000CE0182960E94E13664E275E0CE010196FD
:102240000E949B37BE016E5D7F4FCE0101960E94BA
:10225000543662E474E00E943D36BC018FE094E1A4
:102260000E948E36CE0101960E94DC36CE01829607
:102270000E94DC366FE074E1CE0101960E94933734
:10228000CE0101960E94F63DCE0101960E94DC36F9
:1022900010E069EA76E0CE0182960E949B37CE017B
:1022A00082960E94C233811113C06DEA76E0CE019E
:1022B00001960E949B37CE0101960E94C23301E035
:1022C000811101C000E0CE0101960E94DC3601C000
:1022D00001E0CE0182960E94DC36002309F478C02A
:1022E00080912703909128030E94693B60935303D8
:1022F0007093540380935503909356036093C810D2
:102300007093C9108093CA109093CB1080E090E036
:10231000A0E8BFE380934F0390935003A093510331
:10232000B09352038093C0109093C110A093C21039
:10233000B093C31061EB76E088E892E10E948138A7
:10234000609153037091540380915503909156030B
:102350000E945D31109231101092301080E090E0B8
:102360000E94674440915303509154036091550378
:102370007091560322E0CE0182960E94E1366CEC09
:1023800076E0CE0101960E949B37BE016E5D7F4FC5
:10239000CE0101960E945436BC018FE094E10E9468
:1023A0008E36CE0101960E94DC36CE0182960E94C6
:1023B000DC366FE074E1CE0101960E949337CE01C6
:1023C00001960E94F63DCE0101960E94DC3610E097
:1023D00065ED76E0CE0182960E949B37CE01829613
:1023E0000E94C233811113C06BED76E0CE010196DD
:1023F0000E949B37CE0101960E94C23301E08111F9
:1024000001C000E0CE0101960E94DC3601C001E06F
:10241000CE0182960E94DC36002309F4D6C080915A
:102420002514909126140797D8F066E070E0CE014D
:1024300001960E94F643BE016F5F7F4F89E094E1F1
:102440000E94A336CE0101960E94DC360E943250D3
:1024500060933B0370933C0380933D0390933E0352
:10246000809121030E94133ABC01990F880B990BAC
:102470000E94F1602DE038E643E55BE30E94506185
:102480006B017C01209174033091750340917603B8
:10249000509177030E94EB6018164CF060915C033A
:1024A00070915D0380915E0390915F031BC020914A
:1024B00088033091890340918A0350918B03C701AF
:1024C000B6010E94306487FF05C0C701B6010E94B3
:1024D0001D4308C060917003709171038091720375
:1024E0009091730320E030E048EC52E40E94506188
:1024F0006B017C0120E030E0A9010E94EB6018161E
:1025000034F0C12CD12C38EAE32E31E4F32EC09202
:102510003B03D0923C03E0923D03F0923E03C09215
:10252000E810D092E910E092EA10F092EB1061EE20
:1025300076E088E892E10E94813860913B037091D7
:102540003C0380913D0390913E030E945D311092C7
:1025500031101092301080E090E00E94674440916A
:102560003B0350913C0360913D0370913E0322E098
:10257000CE0182960E94E13662EF76E0CE010196AE
:102580000E949B37BE016E5D7F4FCE0101960E9477
:102590005436BC018FE094E10E948E36CE01019644
:1025A0000E94DC36CE0182960E94DC366FE074E138
:1025B000CE0101960E949337CE0101960E94F63D0E
:1025C000CE0101960E94DC3610E06CEF76E0CE0181
:1025D00082960E949B37CE0182960E94C23381115F
:1025E00013C061E077E0CE0101960E949B37CE01D7
:1025F00001960E94C23301E0811101C000E0CE01CA
:1026000001960E94DC3601C001E0CE0182960E9454
:10261000DC36002309F4B8C080912514909126146B
:102620000697E8F065E070E0CE0101960E94F6435F
:10263000BE016F5F7F4F89E094E10E94A336CE0117
:1026400001960E94DC360E9432500E9471646093B1
:1026500090037093910380939203909393038091DE
:102660009C0390919D030E94293B20E030E048E0CC
:1026700051E40E944163609398037093990380939F
:102680009A0390939B036093D8107093D910809312
:10269000DA109093DB108091900390919103A091B8
:1026A0009203B09193038093E0109093E110A09374
:1026B000E210B093E31066E077E088E892E10E94D0
:1026C0008138209190033091910340919203509171
:1026D000930360E070E080E291E40E94EF6441E0E7
:1026E0000E944E2C66E177E088E892E10E948138F2
:1026F000609198037091990380919A0390919B0344
:102700000E945D31109231101092301080E090E004
:102710000E946744409198035091990360919A03F5
:1027200070919B0323E0CE0182960E94E1366DE119
:1027300077E0CE0101960E949B37BE016E5D7F4F10
:10274000CE0101960E94543666E277E00E943D3643
:10275000BC018FE094E10E948E36CE0101960E946A
:10276000DC36CE0182960E94DC366FE074E1CE0149
:1027700001960E949337CE0101960E94F63DCE014C
:1027800001960E94DC3610E068E277E0CE01829686
:102790000E949B37CE0182960E94C233811113C0E2
:1027A0006DE277E0CE0101960E949B37CE01019643
:1027B0000E94C23301E0811101C000E0CE01019608
:1027C0000E94DC3601C001E0CE0182960E94DC3618
:1027D000002309F4B8C0809125149091261406971F
:1027E000E8F065E070E0CE0101960E94F643BE017C
:1027F0006F5F7F4F89E094E10E94A336CE0101967E
:102800000E94DC360E9432500E94716460938C03F7
:1028100070938D0380938E0390938F0380919C031C
:1028200090919D030E94293B20E030E048E051E474
:102830000E94416360939403709395038093960381
:10284000909397036093DC107093DD108093DE10FB
:102850009093DF1080918C0390918D03A0918E0353
:10286000B0918F038093E4109093E510A093E6104D
:10287000B093E71062E377E088E892E10E94813844
:1028800020918C0330918D0340918E0350918F03E2
:1028900060E070E080E291E40E94EF6441E00E9419
:1028A0004E2C66E177E088E892E10E9481386091E1
:1028B00094037091950380919603909197030E94E1
:1028C0005D31109231101092301080E090E00E9443
:1028D00067444091940350919503609196037091E1
:1028E000970323E0CE0182960E94E13661E477E00F
:1028F000CE0101960E949B37BE016E5D7F4FCE01D7
:1029000001960E94543666E277E00E943D36BC0193
:102910008FE094E10E948E36CE0101960E94DC3653
:10292000CE0182960E94DC366FE074E1CE01019602
:102930000E949337CE0101960E94F63DCE0101968A
:102940000E94DC3610E06AE477E0CE0182960E94B5
:102950009B37CE0182960E94C233811113C06EE470
:1029600077E0CE0101960E949B37CE0101960E942E
:10297000C23301E0811101C000E0CE0101960E9446
:10298000DC3601C001E0CE0182960E94DC360023D5
:1029900009F478C080912703909128030E94693B35
:1029A00060935703709358038093590390935A038D
:1029B0006093CC107093CD108093CE109093CF1075
:1029C00080E090E5A3ECB7E480934B0390934C0335
:1029D000A0934D03B0934E038093C4109093C51001
:1029E000A093C610B093C71062E577E088E892E143
:1029F0000E94813860915703709158038091590368
:102A000090915A030E945D31109231101092301053
:102A100080E090E00E946744409157035091580332
:102A20006091590370915A0322E0CE0182960E9470
:102A3000E1366FE677E0CE0101960E949B37BE013A
:102A40006E5D7F4FCE0101960E945436BC018FE02F
:102A500094E10E948E36CE0101960E94DC36CE01B2
:102A600082960E94DC366FE074E1CE0101960E94EE
:102A70009337CE0101960E94F63DCE0101960E9449
:102A8000DC3610E06AE777E0CE0182960E949B3741
:102A9000CE0182960E94C233811113C06EE777E0A7
:102AA000CE0101960E949B37CE0101960E94C2334F
:102AB00001E0811101C000E0CE0101960E94DC36E8
:102AC00001C001E0CE0182960E94DC36002309F4A9
:102AD000A6C080912514909126140497D8F064E044
:102AE00070E0CE0101960E94F643BE016F5F7F4FFA
:102AF00089E094E10E94A336CE0101960E94DC3663
:102B00000E94325060934F0370935003809351039F
:102B10009093520380914F0390915003A0915103E1
:102B2000B09152038093C0109093C110A093C21033
:102B3000B093C31062E877E088E892E10E948138A0
:102B400060914F0370915003809151039091520313
:102B500042E00E944E2C80912703909128030E940E
:102B6000693B609353037093540380935503909390
:102B700056036093C8107093C9108093CA10909345
:102B8000CB106AE977E088E892E10E948138609191
:102B900053037091540380915503909156030E9402
:102BA0005D31109231101092301080E090E00E9460
:102BB00067444091530350915403609155037091C1
:102BC000560322E0CE0182960E94E13664EA77E065
:102BD000CE0101960E949B37BE016E5D7F4FCE01F4
:102BE00001960E945436BC018FE094E10E948E361B
:102BF000CE0101960E94DC36CE0182960E94DC3620
:102C00006FE074E1CE0101960E949337CE010196E8
:102C10000E94F63DCE0101960E94DC3610E06CEA7F
:102C200077E0CE0182960E949B37CE0182960E9469
:102C3000C233811113C060EB77E0CE0101960E9490
:102C40009B37CE0101960E94C23301E0811101C081
:102C500000E0CE0101960E94DC3601C001E0CE0109
:102C600082960E94DC36002309F4A2C080912514CC
:102C7000909126140497D8F064E070E0CE0101969C
:102C80000E94F643BE016F5F7F4F89E094E10E948E
:102C9000A336CE0101960E94DC360E94325060932A
:102CA0004B0370934C0380934D0390934E0380919C
:102CB0004B0390914C03A0914D03B0914E03809330
:102CC000C4109093C510A093C610B093C71064EBC6
:102CD00077E088E892E10E94813860914B0370911F
:102CE0004C0380914D0390914E0342E00E944E2C84
:102CF00080912703909128030E94693B60935703BA
:102D0000709358038093590390935A036093CC10A7
:102D10007093CD108093CE109093CF106AE977E036
:102D200088E892E10E9481386091570370915803BE
:102D30008091590390915A030E945D311092311095
:102D40001092301080E090E00E9467444091570359
:102D5000509158036091590370915A0322E0CE01BB
:102D600082960E94E13664EA77E0CE0101960E94E5
:102D70009B37BE016E5D7F4FCE0101960E94543697
:102D8000BC018FE094E10E948E36CE0101960E9434
:102D9000DC36CE0182960E94DC366FE074E1CE0113
:102DA00001960E949337CE0101960E94F63D15C010
:102DB000112311F40C94AC056CE075E0CE01019682
:102DC0000E949B3761E274E1CE0101960E94543665
:102DD000BC0188E892E10E947138CE0101960E9400
:102DE000DC360C94AC050E94284D182F882311F472
:102DF0000C94B70580EE94E10E94184665E97EE0E8
:102E00008BE194E10E9479366CEC77E088E892E1FE
:102E10000E948138612F88E892E10E94AF3788E8EC
:102E200092E10E946E38812F0E94F14E0C94AC0505
:102E30000E94953A28EEC22E23E0D22EE12CF12CEE
:102E4000A70196010E944962CA01B9010E94EF6080
:102E50002091C60F3091C70F4091C80F5091C90FF4
:102E60000E947A6220910002309101024091020298
:102E7000509103020E943064181614F00C94BC05A3
:102E80000E94953AA70196010E944962CA01B901C0
:102E90000E94EF606093C60F7093C70F8093C80FB6
:102EA0009093C90F80912E1090912F10F4D664E169
:102EB00070E080E090E00E945D3A0C94DB058BE1CD
:102EC00094E10E940536613071058105910511F08C
:102ED0000C9439070E948D3B0C943907F12C0C940B
:102EE000A70501E02CC801E08EC8CE0188960E949B
:102EF000DC360C948507EF960FB6F894DEBF0FBE54
:102F0000CDBFDF91CF911F910F91FF90EF90DF9098
:102F1000CF90BF90AF909F908F907F906F905F9079
:102F20004F903F9008952F923F924F925F926F92F1
:102F30007F928F929F92AF92BF92CF92DF92EF9249
:102F4000FF920F931F93CF93DF93CDB7DEB72897F0
:102F50000FB6F894DEBF0FBECDBFFC0187E393E14F
:102F6000938782878091341390E09587848780913E
:102F7000011490E09787868780913113853009F09E
:102F8000B7C38091391390913A13885891098D35C0
:102F9000910588F480913413843041F480913B137F
:102FA00090913C138097479708F407C2809134139F
:102FB000843408F0E8C1809134138A3108F448C0A1
:102FC0008091371390913813843F914050F41186CB
:102FD00010868FEF9FEFDC0184839583A683B783F0
:102FE00051C08091391390913A1385974B9780F592
:102FF0001DE3E12E13E1F12E82E090E040E050E08D
:10300000BA018C010F5F1F4F2091341330E002177B
:1030100013076CF4970122503109D9012D913C918D
:10302000275031092730310508F40AC2C801019739
:1030300095958795918780870C971CF4118610864B
:1030400007C0448355836683778384E090E01CC186
:10305000809134138A3108F448C0809137139091DD
:1030600038138032934008F4B2CF80913913909195
:103070003A13C697869708F403C237C04483558332
:10308000668377838BE090E0FFC0D7012D913C9160
:10309000255231092B31310508F004C2440F551F68
:1030A000661F771F41600296B4E0EB0EF11C8C01A5
:1030B0000F5F1F4F2091341330E00217130764F4A1
:1030C000970122503109D9012D913C912C503109A1
:1030D0002B303105D0F2C8010197959587959187DE
:1030E00080870C975CF611861086809134138232AB
:1030F00008F44CC08091391390913A1306970797C2
:1031000008F044C04DE3C42E43E1D42E82E090E0A9
:1031100040E050E0BA018C010F5F1F4F2091341343
:1031200030E0021713070CF5D6011297ED90FC90D2
:1031300011979D01BEE1EB1AF108A7E1EA16F1042F
:1031400008F0BEC1440F551F661F771F4160D601AE
:103150002D913C91B4E0CB0ED11C23503109253088
:10316000310510F40296D7CFC80101979595879540
:103170009187808740971CF41186108607C044838E
:103180005583668377838CE090E07EC07F011C824C
:103190001B8281E090E09A838983809134138D3083
:1031A00008F475C029E733E0AE014D5F5F4FBE0103
:1031B0006F5F7F4FCF010E94714E892B09F067C06E
:1031C00029E733E0AE014D5F5F4FBE016F5F7F4F78
:1031D000C7010E94714E019709F059C029E733E0F9
:1031E000AE014D5F5F4FBE016F5F7F4FC7010E9411
:1031F000714E892B09F04BC0812C912C540100E0B9
:1032000010E08091341390E029813A812817390722
:103210007CF529E733E0AE014D5F5F4FBE016F5F84
:103220007F4FC7010E94714E6C0129E733E0AE0168
:103230004D5F5F4FBE016F5F7F4FC7010E94714EB0
:10324000E1E0CE16D10449F4892B09F5880C991CCC
:10325000AA1CBB1C689480F808C0CD28C1F4019753
:10326000B1F4880C991CAA1CBB1C0F5F1F4FC9CF5F
:10327000D70119961C930E931897F70184829582B3
:10328000A682B78281E090E09183808329C21C826C
:103290001B8281E090E09A838983D7011C968D91EF
:1032A0009C911D97181619060CF061C01A96ED91A5
:1032B000FC911B9782E090E09A83898382819381BD
:1032C00089974E9708F053C083E090E09A838983F2
:1032D000848195810B970A9708F049C02CEB31E067
:1032E000AE014D5F5F4FBE016F5F7F4FC7010E9410
:1032F000714E892BE1F52CEB31E0AE014D5F5F4F54
:10330000BE016F5F7F4FC7010E94714E019779F533
:10331000412C512C320100E010E029813A81D70183
:103320001C968D919C911D97281739070CF010C1A0
:103330002CEB31E0AE014D5F5F4FBE016F5F7F4F01
:10334000C7010E94714E5C010330110509F0C6C02F
:103350002CEB31E0AE014D5F5F4FBE016F5F7F4FE1
:10336000C7010E94714EA816B90609F4B7C0D7016B
:103370001A96ED91FC911B9782819381C69786974F
:1033800008F4F2C03EC180913B1390913C138254EB
:1033900091098E9708F00FCE20E030E0C12CD12C9F
:1033A0007601A901435C5C4EDA014D915C91495074
:1033B00051094930510598F0FECD80913D1390910F
:1033C0003E130997099708F0F1CD118610868FEF0B
:1033D0009FEFDC0184839583A683B7838CC1B901F9
:1033E000615C7C4EDB014D915C914751510942314A
:1033F0005105C0F4D701C601880F991FAA1FBB1F32
:103400006C017D016894C0F82C5F3F4F2038310576
:1034100041F620E230E031872087C482D582E682FF
:10342000F78269C1DB014D915C91465051094730EB
:10343000510508F0C0CDCC0CDD1CEE1CFF1CE4CF08
:10344000D7012D913C91235131092F30310550F492
:10345000440F551F661F771F41600296B4E0EB0EC4
:10346000F11CCFCDD7012D913C912A503109293043
:10347000310508F0EDCD440F551F661F771FEDCFC6
:1034800080913B1390913C13C697869708F02DCE00
:103490008FE3E82E83E1F82E83E090E040E050E0F7
:1034A000BA0105CED7012D913C912C5031092A301B
:1034B000310508F01ACE440F551F661F771FF3CD54
:1034C000D9012D913C912C5031092B30310508F058
:1034D0005DCE440F551F661F771F39CE2CEB31E0B0
:1034E000AE014D5F5F4FBE016F5F7F4FC7010E940E
:1034F000714E6C010330110579F42CEB31E0AE0113
:103500004D5F5F4FBE016F5F7F4FC7010E94714EDD
:10351000C816D90609F02BCFA114B10459F4CA94E6
:10352000CD2809F024CF440C551C661C771C6894E8
:1035300040F80BC0AA94AB2809F019CFCD2809F0A8
:1035400016CF440C551C661C771C0F5F1F4FE5CE31
:1035500019961C930E931897F70144825582668240
:10356000778282E090E090CE848195814B97459759
:1035700008F047C0DF0116966F0126ECC20ED11C81
:1035800020E030E040E050E060E070E080E090E07B
:103590000D911C911197095011090830110588F5FA
:1035A00012960D911C911397015111090D301105BF
:1035B000D8F401E00E94C36521601496AC15BD05E6
:1035C00039F7F701248335834683578300E20E944D
:1035D000DE652283338385E090E09183808380E3FE
:1035E00090E0918780877CC012960D911C91139773
:1035F000045011090530110520F401E00E94C36553
:10360000DCCF80913413893340F0828193818957D4
:1036100091098335910508F47CC18091341382327D
:1036200009F46CC082819381895791098335910592
:1036300008F4E6C1828193818C549109C59708F002
:1036400064C080913413843031F4848195818097F3
:10365000479708F434C280913413843408F455C079
:103660008481958189549109C39708F04EC09F01C8
:103670002A5F3F4FAF014A575F4F812C912C540175
:10368000D9016D917C916950710969307105E8F536
:10369000D90112966D917C91139766517109613130
:1036A000710508F022C2D501C401880F991FAA1F15
:1036B000BB1F4C015D01689480F82C5F3F4F2417BD
:1036C0003507F1F620E230E0F70131872087D70196
:1036D00084829582A682B78287E090E08D939C9346
:1036E00081E090E0BFC282E08093311310923413E6
:1036F00080E090E0B7C283E090E0C6CD8281938104
:103700000A97099708F460C18DCF809134138634ED
:1037100060F1828193810C970B9708F4F6C125C064
:10372000D90112966D917C9113976E517109673191
:10373000710508F01EC2D501C401880F991FAA1F88
:10374000BB1F4C015D01689480F84E5F5F4F2C5F9A
:103750003F4F4534510509F4F3C1D9016D917C9176
:103760006C5071096B307105D8F280913413883533
:1037700078F182819381855891098B35910508F400
:1037800008C226C0BC016F5F7F4FD8012D913C91CC
:10379000275031092730310508F00AC2440F551F60
:1037A000416002960C5F1F4F2091341330E024508B
:1037B0003109821793070CF004C298012250310995
:1037C000D9012D913C912950310928303105D0F291
:1037D000809134138032E1F48281938106970697B9
:1037E000B8F4848195810997099790F49F012A5F25
:1037F0003F4FAF01425C5F4F812C912C5401D901A6
:103800006D917C91665071096630710508F4F3C1C1
:10381000D7011C962D903C901D97B6E02B163104D5
:103820000CF461CF8F010A5F1F4F73E0C72ED12CBC
:10383000E5EC8E2EEDE99E2EECE1AE2EE1E8BE2EFB
:10384000F8016081718134976080718080E090E040
:103850000E94EF606D837E838F839887B30180E041
:1038600090E00E94EF602B013C012DEC3CEC4CE41D
:103870005FE30E9450619B01AC016D817E818F816D
:1038800098850E94EB6087FD19C02DEC3CEC4CE460
:103890005FE36D817E818F8198850E9450619B01DD
:1038A000AC01C301B2010E94EB60E82F880FFF0B4F
:1038B000EE27FF0FEE1FFF27319602C0E0E0F0E099
:1038C000A501940163E971E080E091E00E949965AF
:1038D0004F01FF0FAA08BB0886269726A826B926FF
:1038E000FFEFCF1ADF0A0E5F1F4FC214D30409F097
:1038F000A7CFD70114968D929D92AD92BC92179747
:1039000080E290E019969C938E9318978FEF9FEF2B
:10391000E5CE84819581CA97899708F07ECE9F0174
:103920002A5F3F4F812C912C540143E050E0D90194
:103930006D917C916A5071096930710508F06DCE06
:10394000D90112966D917C9113976651710961317D
:10395000710550F5D501C401880F991FAA1FBB1F1F
:103960004C015D01689480F84E5F5F4F2C5F3F4FC4
:103970004B335105E1F69F012A583F4FD9012D9154
:103980003C912A5031092930310508F046CE2CE10E
:1039900030E0F70131872087D70184829582A682A3
:1039A000B7828AE090E09ACED90112966D917C910F
:1039B0001397665071096730710508F02ECE880C98
:1039C000991CAA1CBB1CD0CF20913413CF01820FAD
:1039D000911D820F911DDC0112978D919C910A9788
:1039E000099708F01FCEF701118610868FEF9FEF21
:1039F000DC0184839583A683B78386E090E044CC82
:103A000080913413813208F415CE84819581CA9750
:103A1000899708F00FCE9F012A5F3F4F812C912C90
:103A2000540143E050E0D9016D917C916A507109D5
:103A30006930710508F0FECDD90112966D917C9127
:103A40001397665171096131710570F112966D918C
:103A50007C911397665071096730710508F0EACDC3
:103A6000880C991CAA1CBB1C4E5F5F4F2C5F3F4FFC
:103A700043325105C1F69F012A5B3F4FD9012D9179
:103A80003C912A5031092930310508F0D3CD20E18D
:103A900030E0F70131872087D70184829582A682A2
:103AA000B78286E090E01ACED501C401880F991F35
:103AB000AA1FBB1F4C015D01689480F8D5CF868199
:103AC00097810997099708F0C6CDD70119961C92DE
:103AD0001E9218978FEF9FEFDC01F7018483958387
:103AE000A683B78387E090E0CFCBD90112966D9182
:103AF0007C911397665071096730710508F005CE07
:103B0000880C991CAA1CBB1CD8CD8481958109976F
:103B1000099708F02ACE868197818C974F9708F0F5
:103B200024CE8085918589974D9708F01ECE9F0100
:103B3000265F3F4F812C912C540145E050E00DCE83
:103B40009F0126573F4FD9012D913C912C503109AF
:103B50002B30310508F009CE20E230E0F701318743
:103B60002087D70184829582A682B78288E090E080
:103B7000B5CDD90112966D917C9113976950710959
:103B80006930710508F0F1CD880C991CAA1CBB1C8A
:103B9000DCCD84819581825491098E9708F018CEEE
:103BA0008F01045C1F4F8DE190E040E050E0FCCDC0
:103BB000D8012D913C912851310922313105C0F0B5
:103BC000CB01019795958795D70119969C938E9374
:103BD00018978A970CF4FCCD052E000C660B770B1A
:103BE000F701448355836683778389E090E04CCB6B
:103BF000440F551FD6CDD90112966D917C91139724
:103C00006951710963317105E8F4D501C401880F68
:103C1000991FAA1FBB1F4C015D01689480F82C5F9F
:103C20003F4F2417350709F0EACD2EE030E0F701C9
:103C300031872087D70184829582A682B7828FE060
:103C400090E04CCDD90112966D917C9113976950FB
:103C500071096930710508F0DBCD880C991CAA1C2C
:103C6000BB1CDDCF28960FB6F894DEBF0FBECDBFCC
:103C7000DF91CF911F910F91FF90EF90DF90CF9048
:103C8000BF90AF909F908F907F906F905F904F907C
:103C90003F902F9008952F923F924F925F926F9294
:103CA0007F928F929F92AF92BF92CF92DF92EF92CC
:103CB000FF920F931F93CF93DF93CDB7DEB7A497F7
:103CC0000FB6F894DEBF0FBECDBF8C0163EE77E078
:103CD00088E892E10E948138C8010E94EA30C80158
:103CE00006960697F8F080912E1090912F1080176D
:103CF0009107F1F00E946E4810932F1000932E1040
:103D00004AE0B801CE0101960E946837BE016F5F9C
:103D10007F4F8BE194E10E94A336CE0101960E9471
:103D2000DC3606C00E3F2FEF120711F40C944D2B1A
:103D3000F8013A96E431F10510F00C94232B882712
:103D4000EE58FF4F8F4F0C94BB6565E97EE0CE01C6
:103D500001960E949B374AE050E061E070E0CE019E
:103D600001960E947748CE0101960E94DC36809130
:103D700021030E94133ABC01990F880B990B0E94F2
:103D8000F1602DE038E643E55BE30E9450616B0192
:103D90007C0120917403309175034091760350911A
:103DA00077030E94EB6018164CF060915C037091F1
:103DB0005D0380915E0390915F031BC02091880397
:103DC0003091890340918A0350918B03C701B6015A
:103DD0000E94306487FF05C0C701B6010E941D43E1
:103DE00008C060917003709171038091720390918B
:103DF000730320E030E048EC52E40E94506120E080
:103E000030E048EA51E40E94506120913B03309138
:103E10003C0340913D0350913E030E9441636B017E
:103E20007C010E946E4860E080E00E94522D0E945A
:103E3000953A28EE33E040E050E00E944962BA0132
:103E4000A9012AE0CE0101960E941037BE016F5FE2
:103E50007F4F89E094E10E94A336CE0101960E9433
:103E6000DC366CEE77E089E094E10E94653669E02B
:103E700074E180EE94E10E94B63762E370E080E086
:103E800090E00E945D3A61E080E00E94522D22E0C5
:103E9000B701A601CE0101960E94E13667E078E005
:103EA000CE0107960E949B37BE016F5F7F4FCE0108
:103EB00007960E94543666EF77E0F1C065E97EE030
:103EC000CE0101960E949B374AE050E061E070E02D
:103ED000CE0101960E947748CE0101960E94DC3601
:103EE00080919C0390919D030E94293B4B015C01B2
:103EF000C0909803D0909903E0909A03F0909B03B0
:103F00008091940390919503A0919603B0919703AB
:103F1000898F9A8FAB8FBC8F209190033091910342
:103F200040919203509193032D8F3E8F4F8F58A352
:103F30009C01AD01C701B6010E947A622B013C01D0
:103F400020918C0330918D0340918E0350918F030B
:103F50006D8D7E8D8F8D98A10E947A629B01AC0140
:103F6000C301B2010E9441632B013C0120E030E01B
:103F700048E051E4C501B4010E9441634B015C017A
:103F800020E030E040EC5FE3C701B6010E945061E1
:103F90009B01AC01C501B4010E94306418167CF18C
:103FA00020E030E040E05FE3698D7A8D8B8D9C8D61
:103FB0000E9450619B01AC01C501B4010E94EB60FD
:103FC00087FD1DC0A7019601C501B4010E947A6258
:103FD000A30192010E9441632D8D3E8D4F8D58A10A
:103FE0000E947B629B01AC0160E070E080E291E4A2
:103FF0000E94EF640E94DA636B017C0104C0CC2450
:10400000CA94DC2C76010E946E4860E080E00E9439
:10401000522D0E94953A28EE33E040E050E00E9495
:104020004962BA01A9012AE0CE0101960E94103727
:10403000BE016F5F7F4F89E094E10E94A336CE01FD
:1040400001960E94DC366BEF77E089E094E10E94F4
:10405000653669E074E180EE94E10E94B63762E370
:1040600070E080E090E00E945D3A61E080E00E94B4
:10407000522D2AE0B701A601CE0101960E943C37DD
:1040800066E078E0CE0107960E949B37BE016F5F25
:104090007F4FCE0107960E9454366BE078E00E9475
:1040A0003D36BC018FE094E10E948E36CE0107962A
:1040B0000E94DC36CE0101960E94DC366FE074E18E
:1040C00080EE94E10E94B63762E370E080E090E019
:1040D0000E945D3A80913210882311F40C94232BB6
:1040E00060E273E080E090E0E3C165E97EE0CE014C
:1040F00001960E949B374AE050E061E070E0CE01FB
:1041000001960E947748CE0101960E94DC360E94FB
:10411000953A6B017C0180913703909138030A979F
:1041200031F48091390390913A030A97B1F08BEE04
:1041300091E10E943C448CED95E0A0E0B0E08093DA
:10414000EF119093F011A093F111B093F21164E686
:1041500070E080E090E00E945D3A0E946E4860E06E
:1041600080E00E94522D6FE078E080EE94E10E94A2
:10417000813862E370E080E090E00E945D3A0E9446
:10418000953ADC01CB018C199D09AE09BF09883B2A
:104190009B40A105B10508F069C00E94024497FD4B
:1041A00006C082349105C9F780E090E002C08FEF2D
:1041B0009FEF892B21F7A8EEAA2EAFE0BA2E45017A
:1041C0000E94024497FF07C08091E80F8D34B9F632
:1041D00080E090E009C0D4018D934D01B7E08B16CB
:1041E000B0E19B0669F7F0CFF50121915F01820FE5
:1041F000911DF5E0AF16F0E1BF06B1F79C012E5B13
:104200003F4F8091051090E0982F8827409106102D
:10421000840F911D2817390709F0B1CF8091EB0F5A
:1042200090E0982F88272091EC0F820F911D90939A
:10423000E70F8093E60F8091ED0F90E0982F88278D
:104240002091EE0F820F911D9093E50F8093E40F64
:104250008091EF0F90E0982F88272091F00F820F28
:10426000911D9093E30F8093E20F89CF0E94953ABE
:10427000DC01CB018C199D09AE09BF09883B9B402D
:10428000A105B10508F400C10E946E4860E080E01D
:104290000E94522D0E94953A28EE33E040E050E013
:1042A0000E944962BA01A9012AE0CE0101960E944A
:1042B0001037BE016F5F7F4F89E094E10E94A33603
:1042C000CE0101960E94DC3662E474E089E094E15C
:1042D0000E94653669E074E180EE94E10E94B63791
:1042E0006CE271E080E090E00E945D3A6FE178E07E
:1042F00089E094E10E94653660E086E00E94522DDC
:1043000060E278E080EE94E10E94813862E370E040
:1043100080E090E00E945D3A61E080E00E94522DD2
:104320006091E20F7091E30F4AE0CE0101960E9486
:1043300068376091E40F7091E50F4AE0CE0107966F
:104340000E9468376091E60F7091E70F4AE0CE0156
:1043500043960E946837BE016D5E7F4FCE010D9679
:104360000E94933769E976E0CE010D960E943D36B2
:10437000BE01695F7F4F0E94543669E976E00E9472
:104380003D36BE016F5F7F4F0E945436BC018FE007
:1043900094E10E948E36CE010D960E94DC36CE014D
:1043A00043960E94DC36CE0107960E94DC36CE0191
:1043B00001960E94DC366FE074E180EE94E10E9489
:1043C000B63761E08CE00E94522D6CE378E080EE1D
:1043D00094E10E9481386091E20F7091E30F4AE00E
:1043E000CE0101960E9468376091E40F7091E50F4D
:1043F0004AE0CE0107960E9468376091E60F7091FF
:10440000E70F4AE0CE010D960E9468376BE278E034
:10441000CE0143960E949B37BE01635F7F4FCE0162
:1044200043960E94543662E77FE00E943D36BE010B
:10443000695F7F4F0E94543662E77FE00E943D36FD
:10444000BE016F5F7F4F0E9454366BE378E00E949D
:104450003D36BC018FE094E10E948E36CE0143963A
:104460000E94DC36CE010D960E94DC36CE01079606
:104470000E94DC36CE0101960E94DC3662E370E0D9
:1044800080E090E00E945D3A80913703909138037C
:104490000A9741F48091390390913A030A9711F4F5
:1044A0000C94232B0E949B3262E370E080E090E04A
:1044B0000E945D3A0C94232B90912B1081E0892768
:1044C00080932B1080913210882331F06FE074E1DB
:1044D0008EE491E10E94713868EC70E080E090E039
:1044E000E7CF109232100C94232B81E0809332108E
:1044F0000C94232B61E478E0CE0107960E949B3751
:104500006AED74E1CE0107960E945436BC01CE01DB
:1045100001960E94933748EE53E060E070E0CE01D0
:1045200001960E947748CE0101960E94DC36CE01AA
:1045300007960E94DC3665E478E0CE0101960E9481
:104540009B3740ED57E061E070E0CE0101960E949C
:104550007748CE0101960E94DC3665E578E0CE0111
:1045600001960E949B3748EC50E060E070E0CE017D
:1045700001960E947748CE0101960E94DC3665E6DE
:1045800078E0CE0101960E949B3740ED57E061E054
:1045900070E0CE0101960E947748CE0101960E94FC
:1045A000DC3662E778E0CE0101960E949B3748EC4A
:1045B00050E060E070E0CE0101960E947748CE01A5
:1045C00001960E94DC366FE778E0CE0101960E94EA
:1045D0009B3740ED57E061E070E0CE0101960E940C
:1045E0007748CE0101960E94DC366AE878E0CE0179
:1045F00001960E949B3748EC50E060E070E0CE01ED
:1046000001960E947748CE0101960E94DC3666E949
:1046100078E0CE0101960E949B3740ED57E061E0C3
:1046200070E0CE0101960E947748CE0101960E946B
:10463000DC3667EA78E0CE0101960E949B3748ECB1
:1046400050E060E070E0CE0101960E947748CE0114
:1046500001960E94DC3661EB78E0CE0101960E9463
:104660009B3740ED57E061E070E0CE0101960E947B
:104670007748CE0101960E94DC366CEB78E0CE01E3
:1046800001960E949B3748EC50E060E070E0CE015C
:1046900001960E947748CE0101960E94DC3669ECB3
:1046A00078E0CE0101960E949B3740ED57E061E033
:1046B00070E0CE0101960E947748CE0101960E94DB
:1046C000DC3668ED78E0CE0101960E949B3748EC1D
:1046D00050E060E070E0CE0101960E947748CE0184
:1046E00001960E94DC3665EE78E0CE0101960E94CC
:1046F0009B3740ED57E061E070E0CE0101960E94EB
:104700007748CE0101960E94DC3665EF78E0CE0155
:1047100001960E949B3748EC50E060E070E0CE01CB
:1047200001960E947748CE0101960E94DC3662E035
:1047300079E0CE0101960E949B3740ED57E061E0A1
:1047400070E0CE0101960E947748CE0101960E944A
:10475000DC366EE079E0CE0101960E949B3748EC92
:1047600050E060E070E0CE0101960E947748CE01F3
:1047700001960E94DC366AE179E0CE0101960E9442
:104780009B3740ED57E061E070E0CE0101960E945A
:104790007748CE0101960E94DC3655C765E97EE078
:1047A000CE0101960E949B374AE050E061E070E044
:1047B000CE0101960E947748CE0101960E94DC3618
:1047C00080912703909128030E94B7323CC765E986
:1047D0007EE0CE0101960E949B374AE050E061E006
:1047E00070E0CE0101960E947748CE0101960E94AA
:1047F000DC360E948D3B27C780911E03882309F475
:1048000022C765E97EE0CE0101960E949B374AE00F
:1048100050E061E070E0CE0101960E947748CE0141
:1048200001960E94DC360E946E486EE170E080E0E6
:1048300090E00E945D3A0E94802E2B013C0164E6CC
:1048400070E080E090E00E945D3A0E94FA2D4B01FA
:104850005C0164E670E080E090E00E945D3A609167
:104860004703709148038091490390914A030E9445
:10487000F1609B01AC0169A33AA34BA35CA30E9426
:10488000802E0E94F16029A13AA14BA15CA10E9457
:10489000416321E03EED42E45EE30E94EF649B0150
:1048A000AC0160E070E080E89FE30E947A6220E063
:1048B0003AE24DE257E40E9450616B017C0164E6EC
:1048C00070E080E090E00E945D3A60E080E00E944D
:1048D000522D0E94953A28EE33E040E050E00E94CD
:1048E0004962BA01A9012AE0CE0107960E94103759
:1048F000BE01695F7F4FCE0101960E94933761E14F
:1049000075E0CE0101960E943D36BC0189E094E13C
:104910000E948E36CE0101960E94DC36CE010796AB
:104920000E94DC36C301B2010E94F16020E030E059
:1049300048EC52E40E944163AB01BC0122E030E04C
:10494000CE0101960E949C48BE016F5F7F4F83E0BD
:1049500094E10E94A336CE0101960E94DC3665E602
:1049600075E083E094E10E94653663E074E189E0DC
:1049700094E10E94733661E675E0CE0101960E94D3
:104980009B3763E074E1CE0101960E945436BC016E
:1049900083E094E10E948E36CE0101960E94DC36BF
:1049A00064E670E080E090E00E945D3A66E775E0C2
:1049B0008FE094E10E94793621E030E0B501A40156
:1049C000CE0101960E949C48BE016F5F7F4F8FE031
:1049D00094E10E947336CE0101960E94DC3665E2B6
:1049E00079E08FE094E10E94653621E030E0B70184
:1049F000A601CE0107960E949C48BE01695F7F4FC9
:104A0000CE0101960E94933760E377E0CE010196D4
:104A10000E943D36BC018FE094E10E947336CE01C6
:104A200001960E94DC36CE0107960E94DC3663E0D8
:104A300074E1CE0101960E94933762E77FE0CE01D8
:104A400001960E943D366FE074E10E945436BC012D
:104A50008FE094E10E948E36CE0101960E94DC36F2
:104A600069E074E180EE94E10E94B63721E030E025
:104A7000B501A401CE0107960E949C48BE01695F62
:104A80007F4FCE0101960E9493376BE279E0CE0111
:104A900001960E943D36BC0185E194E10E948E366C
:104AA000CE0101960E94DC36CE0107960E94DC36CC
:104AB00021E030E0B701A601CE0107960E949C4894
:104AC000BE01695F7F4FCE0101960E94933760E37C
:104AD00077E0CE0101960E943D36BC0185E194E16C
:104AE0000E947336CE0101960E94DC36CE010796F5
:104AF0000E94DC3661E080E0D5D765E174E180EEAC
:104B000094E10E94B63764E670E080E090E00E9495
:104B10005D3A80913210882309F495C568E572E00A
:104B200080E090E0C5CC65E97EE0CE0101960E9470
:104B30009B374AE050E061E070E0CE0101960E94B0
:104B40007748CE0101960E94DC368091321088238E
:104B500049F082E090E0A0E0B0E0898F9A8FAB8FBF
:104B6000BC8F08C02EE130E040E050E0298F3A8F42
:104B70004B8F5C8F60E379E08FE094E10E9479369F
:104B800061E080E08FD76FE074E180EE94E10E94F5
:104B9000B637812C912C5401C12CD12C760183E2A3
:104BA0000E94F54487E090E00E9463440E9498448C
:104BB00066E970E080E090E00E945D3A83E20E9446
:104BC000F54480E290E00E9463440E94984466E9C4
:104BD00070E080E090E00E945D3A62E070E083E285
:104BE00090E075D7412C512C32018091531090E008
:104BF00020915410821B9109181619066CF485E255
:104C000093E10E944145762C652C542C4424480E97
:104C1000511C611C711CE9CFC301B2010E94F160FB
:104C20002AE939E949E95FE30E9441630E94DA63B6
:104C30002B013C01C616D706E806F9060CF04AC05F
:104C40000E94953A28EE33E040E050E00E9449622D
:104C5000BA01A9012AE0CE0101960E941037BE01D7
:104C60006F5F7F4F89E094E10E94A336CE010196E9
:104C70000E94DC362AE0B301A201CE0101960E9417
:104C80003C3760E479E0CE0107960E949B37BE0175
:104C90006F5F7F4FCE0107960E94543665E479E03E
:104CA0000E943D36BC0189E094E10E947336CE013A
:104CB00007960E94DC36CE0101960E94DC3660E049
:104CC00080E0F0D669E074E180EE94E10E94B637AE
:104CD0007301620162E370E080E090E00E945D3A5F
:104CE0003FEF831A930AA30AB30A898D9A8DAB8D7D
:104CF000BC8D88159905AA05BB050CF050CF2AE09C
:104D0000B701A601CE0101960E943C3769E479E023
:104D1000CE0107960E949B37BE016F5F7F4FCE0189
:104D200007960E9454366CE479E00E943D366FE0AD
:104D300074E10E945436BC018FE094E10E948E36EB
:104D4000CE0107960E94DC36CE0101960E94DC3629
:104D5000ABCB65E97EE0CE0101960E949B374AE02D
:104D600050E061E070E0CE0101960E947748CE01EC
:104D700001960E94DC3681E080935B0364E670E07C
:104D800080E090E00E945D3A0E946E4860E080E022
:104D900089D60E94953A28EE33E040E050E00E9428
:104DA0004962BA01A9012AE080EE94E10E94D93754
:104DB00062E474E080EE94E10E94813888E30E940E
:104DC000133A60E074E0681B790B4AE0CE0101966B
:104DD0000E94683761E579E0CE0107960E949B3713
:104DE000BE016F5F7F4FCE0107960E945436BC0113
:104DF0008FE094E10E948E36CE0107960E94DC3649
:104E0000CE0101960E94DC3660E086E04BD661E878
:104E100078E080EE94E10E94813861E080E042D643
:104E20006FE074E180EE94E10E94B63768E579E0C6
:104E3000CE0101960E949B376FE074E1CE0101968E
:104E40000E945436BC018FE094E10E948E36CE0160
:104E500001960E94DC3664E670E080E090E038C99C
:104E600065E97EE0CE0101960E949B374AE050E062
:104E700061E070E0CE0101960E947748CE01019674
:104E80000E94DC36F0901F030E946E4860E080E0D4
:104E900009D60E94953A28EE33E040E050E00E94A7
:104EA0004962BA01A9012AE0CE0101960E94103799
:104EB000BE016F5F7F4F89E094E10E94A336CE016F
:104EC00001960E94DC3661E175E089E094E10E9480
:104ED000653669E074E180EE94E10E94B6378F2D6B
:104EE0000E94133A7C01909308108093071062E3AC
:104EF00070E080E090E00E945D3A60E088E0D2D50A
:104F00004AE0B701CE0101960E946837BE016F5F8B
:104F10007F4F8FE094E10E94A336CE0101960E945C
:104F2000DC3662E370E080E090E00E945D3A8091C0
:104F30003210882331F060E273E080E090E00E945C
:104F40005D3A80912F03909130038B3091053CF1B5
:104F50002FE0289FB001299F700D1124605F7D4FC5
:104F6000CE0101960E949B37BE016F5F7F4FCE013D
:104F700007960E9493376DEF74E0CE0107960E946A
:104F80003D366FE074E10E945436BC018FE094E13D
:104F90000E948E36CE0107960E94DC3611C062E672
:104FA00079E0CE0101960E949B376FE074E1CE015B
:104FB00001960E945436BC018FE094E10E948E3627
:104FC000CE0101960E94DC3661E080E06BD5F9C22B
:104FD00080911E03882309F436C380913210882300
:104FE00029F082E090E00E9409492DC3C0900C0294
:104FF000D0900D02E0900E02F0900F0220E030E021
:1050000040E450E4C701B6010E94306418166CF405
:1050100020E030E04AE754E4C701B6010E94506145
:105020000E94DA636B017C0106C070E3C72E75E74E
:10503000D72EE12CF12C0E946E4860E080E032D542
:105040006DE679E080EE94E10E94813861E080E0D5
:1050500029D56EE779E080EE94E10E94813868EC12
:1050600070E080E090E00E945D3A0E94953A609383
:10507000DE0F7093DF0F8093E00F9093E10F0E949B
:10508000953A2B013C0162E3862E912CA12CB12C88
:105090008091DE0F9091DF0FA091E00FB091E10FB2
:1050A000A3019201281B390B4A0B5B0B2C153D0504
:1050B0004E055F050CF0C7C283E090E00E940949ED
:1050C0000E94953ADC01CB0184199509A609B7091C
:1050D00088329105A105B10554F4A5019401281B5E
:1050E000390B4A0B5B0BCA01B9010E945D3A0E9461
:1050F000953A2B013C01CCCF65E97EE0CE010196CB
:105100000E949B374AE050E061E070E0CE010196DA
:105110000E947748CE0101960E94DC360E94953AA3
:1051200028EE33E040E050E00E944962BA01A90154
:105130002AE0CE0101960E941037BE016F5F7F4FBB
:1051400089E094E10E94A336CE0101960E94DC36EC
:1051500069E074E1CE0101960E94933766E879E038
:10516000CE0101960E943D36BC0189E094E10E9487
:105170008E36CE0101960E94DC368091321081116C
:1051800002C00E946E4880913703909138030A97BD
:1051900071F48091390390913A030A9741F40E9487
:1051A0009B3264E670E080E090E00E945D3A8CE41F
:1051B0000E94E1316B017C019B01AC010E94806582
:1051C000882339F06AE879E08FE094E10E9479362B
:1051D00095C021E030E0B701A601CE0101960E9402
:1051E0009C4864E979E0CE0107960E949B37BE0196
:1051F0006F5F7F4FCE0107960E9454366DE979E0CC
:105200000E943D36BC018FE094E10E948E36CE01B3
:1052100007960E94DC36CE0101960E94DC3661E0E2
:1052200080E040D46FE074E180EE94E10E94B637F4
:1052300062E370E080E090E00E945D3A86E60E94C2
:10524000E131AB01BC0121E030E0CE0101960E94CA
:105250009C4866E775E0CE0107960E949B37BE0129
:105260006F5F7F4FCE0107960E9454366DE979E05B
:105270000E943D36BC0185E194E10E948E36CE014C
:1052800007960E94DC36CE0101960E94DC3662E76A
:105290007FE0CE0101960E949B3765E174E1CE016B
:1052A00001960E945436BC0189E094E10E94733655
:1052B000CE0101960E94DC3660E080E0F3D369E025
:1052C00074E180EE94E10E94B63765E174E1CE01AD
:1052D00001960E94933762E77FE0CE0101960E941B
:1052E0003D366FE074E10E945436BC018FE094E1DA
:1052F0000E948E36CE0101960E94DC3680913703E3
:10530000909138030A97B1F48091390390913A0350
:105310000A9781F48BEE91E10E943C448CED95E07C
:10532000A0E0B0E08093EF119093F011A093F11101
:10533000B093F21164E670E080E090E00E945D3A84
:1053400080913210882331F060E273E080E090E0D9
:105350000E945D3A8EE491E10E94063574C165E9D0
:105360007EE0CE0101960E949B374AE050E061E06A
:1053700070E0CE0101960E947748CE0101960E940E
:10538000DC360E946E4860E080E08CD360E080E014
:1053900089D30E94953A28EE33E040E050E00E9425
:1053A0004962BA01A9012AE0CE0101960E94103794
:1053B000BE016F5F7F4F89E094E10E94A336CE016A
:1053C00001960E94DC3661E175E089E094E10E947B
:1053D000653669E074E180EE94E10E94B63761E0E1
:1053E00080E060D330912303398F809123108111A5
:1053F0000DC00E94953A60931F1070932010809307
:1054000021109093221081E0809323108091171037
:1054100081110DC00E94953A60931310709314107F
:10542000809315109093161081E0809317101092BE
:10543000121010921110209011103090121058E29A
:10544000251631040CF084C0898D0E94133AF101B5
:10545000EE0FFF1FE250FF4E918380830E94FE41BA
:1054600020E030E040EA50E40E94506120E030E06B
:1054700040E85AE30E9450616B017C0160930D107B
:1054800070930E1080930F109093101040900402B0
:10549000509005026090060270900702A3019201ED
:1054A000609108027091090280910A0290910B02AA
:1054B0000E947A629B01AC0160E070E080EC90E4B5
:1054C0000E947A624B015C0120E030E0A9010E9459
:1054D000EB6020E030E040E650E4811105C0C701F8
:1054E000B6010E9450611EC0C701B6010E94506102
:1054F000A30192010E947B6220E030E040E850E48A
:105500000E947A62A50194010E94416320E030E08C
:1055100040EC50E40E94506120E030E040E850E46C
:105520000E947B626093091070930A1080930B10A5
:1055300090930C1064E170E080E090E00E945D3A8E
:105540004FEF241A340A309212102092111073CFA8
:10555000C0900910D0900A10E0900B10F0900C1041
:1055600020E030E0A901C701B6010E94306487FD48
:1055700022C022E0B701A601CE0101960E94E136C9
:1055800060EA79E0CE0107960E949B37BE016F5F0B
:105590007F4FCE0107960E945436BC018FE094E104
:1055A0000E948E36CE0107960E94DC36CE0101960F
:1055B0000E94DC3606C064EA79E08FE094E10E9444
:1055C00079366FE074E180EE94E10E94B6373BC01B
:1055D00080911E038823B9F165E97EE0CE01019632
:1055E0000E949B374AE050E061E070E0CE010196F6
:1055F0000E947748CE0101960E94DC3680913210DD
:10560000811117C020E030E040EA51E460910C02C3
:1056100070910D0280910E0290910F020E945061D4
:105620000E94DA639B01AC016AE070E080E090E0E8
:1056300008C021E030E040E050E064EF71E080E03D
:1056400090E00E94033E61E080E02CD28091131430
:1056500090911414009799F0419718F402301105B5
:10566000ACF46FE074E1CE0101960E949337CE0155
:1056700001960E94F63DCE0101960E94DC3664E65A
:1056800070E080E090E00E945D3A07C06FE074E156
:1056900080EE94E10E94B637E4CFA4960FB6F8945A
:1056A000DEBF0FBECDBFDF91CF911F910F91FF9055
:1056B000EF90DF90CF90BF90AF909F908F907F90B2
:1056C0006F905F904F903F902F9008950F931F938E
:1056D000CF93DF938C01EB018EE10E94F544C8016A
:1056E0000E946344CE010E946344DF91CF911F91D9
:1056F0000F910C949844CF92DF92EF92FF926B013E
:105700007C012EEA37E441E65FE30E94EB60811101
:105710000EC088E491EEAAE3BFE380933E14909319
:105720003F14A0934014B093411460E0ABC026E650
:1057300036E646EA5FE3C701B6010E94EB608111DD
:105740000EC08FE195E8ABE6BFE380933E149093E3
:105750003F14A0934014B093411461E093C023E33D
:1057600033E343EF5FE3C701B6010E94EB608111B1
:105770000EC086EF98E2ACE9BFE380933E149093AD
:105780003F14A0934014B093411462E07BC020E02A
:1057900030E040E250E4C701B6010E94EB608111A5
:1057A0000EC08CE59FE8A2ECBFE380933E1490937B
:1057B0003F14A0934014B093411463E063C020E011
:1057C00030E040E850E4C701B6010E94EB6081116F
:1057D0000EC08EEA97E4A1E1B0E480933E1490936A
:1057E0003F14A0934014B093411464E04BC026E6EC
:1057F00036E646E950E4C701B6010E94EB6081112C
:105800000EC08AE097EDA3E2B0E480933E1490933B
:105810003F14A0934014B093411465E033C023E3D8
:1058200033E343EB50E4C701B6010E94EB60811102
:105830000EC085E89BEEA1E4B0E480933E14909303
:105840003F14A0934014B093411466E01BC02AE9B2
:1058500039E941E051E4C701B6010E94EB608111D2
:105860000EC083E393E3ABE8B0E480933E149093DF
:105870003F14A0934014B093411467E003C081E04B
:1058800090E007C06295660F607E70E081E090E076
:105890001DDFFF90EF90DF90CF9008954F925F92C1
:1058A0006F927F928F929F92AF92BF92CF92DF9230
:1058B000EF92FF926B017C01B42E9B01AC010E9420
:1058C0008065882319F063E77EE027C02601370151
:1058D000E89477F82FEF3FEF4FE75FE7C301B2019E
:1058E0000E94806581110DC02FEF3FEF4FE75FE70A
:1058F000C301B2010E94EB6018161CF467E77EE05A
:105900000CC02FEF3FEF4FE75FE4C701B6010E94E5
:105910003064181694F46BE77EE088E892E1FF901B
:10592000EF90DF90CF90BF90AF909F908F907F903F
:105930006F905F904F900C94C4372FEF3FEF4FE77D
:105940005FECC701B6010E94EB6087FDE4CF20E069
:1059500030E0A901C701B6010E94EB6087FF0BC0D0
:105960006DE288E892E10E94AF374C01F7FAF094BB
:10597000F7F8F09402C0812C912CA12C60E070E02B
:1059800080E09FE3AB1441F020E030E040E251E4DE
:105990000E944163A394F6CF9B01AC01C701B601FD
:1059A0000E947B622B013C010E94DF636B017C0142
:1059B0000E94EF609B01AC01C301B2010E947A62B8
:1059C0002B013C012AE0B701A60188E892E10E9480
:1059D000D9377C01E80CF91CBB2039F06EE288E86D
:1059E00092E10E94AF37E80EF91EDB2CDD2031F189
:1059F00020E030E040E251E4C301B2010E94506176
:105A00002B013C010E94DF634B01A12CB12C2AE049
:105A1000B501A40188E892E10E94D937E80EF91E89
:105A2000C501B4010E94EF609B01AC01C301B2014A
:105A30000E947A622B013C01DA94D8CFC701FF9013
:105A4000EF90DF90CF90BF90AF909F908F907F901E
:105A50006F905F904F9008951092541010925310D1
:105A6000109292101092B3101092901081E08093D7
:105A70008F1010926A1061E084E10E94A23961E007
:105A800085E10E94A239E9EBF0E080818E7F80837E
:105A900080818D7F808388E48093B80085E4809343
:105AA000BC000895643008F063E09091F314691726
:105AB00010F06FEF690FE62FF0E0E052FB4E948993
:105AC000682F690F606880EE94E10C9416469091FF
:105AD00090109111FCCF613208F060E291E0909358
:105AE000901090938F102FEF20938E1010928D10A6
:105AF000260F20938C1090936B1090916B10880F51
:105B0000892B80936B1080916A10813061F4109220
:105B10006A1080916B108093BB008091BC0083FD64
:105B2000F8CF85EC01C085EE8093BC008091901089
:105B30008130E1F380918D10861710F460918D1003
:105B4000ACE6B0E123E330E1F9018E2F821B86172A
:105B500018F48D918193F9CF1092541060935310E3
:105B6000862F08950F931F93CF93DF931F92CDB786
:105B7000DEB7682F87E769830E94F544698185E273
:105B800093E10E948C450E94984487E70E94F54467
:105B900062E070E087E790E09ADF85E293E10E949F
:105BA000414500E010E0182F85E293E10E94414555
:105BB000082B192B0E949844C8010F90DF91CF91B8
:105BC0001F910F91089587E70E94F54464EF85E2E5
:105BD00093E10E948C456EE285E293E10E948C4540
:105BE0000E94984465E070E080E090E00E945D3A99
:105BF00086EFB8CFCF92DF92EF92FF920F931F9371
:105C0000E2DFAC0160E070E0E7E2F4E185899689CB
:105C10009A01AB01281B390B41095109A389B489A9
:105C20000E9439626B017C018FE0F594E794D79470
:105C3000C7948A95D1F765857685CB01770FAA0B36
:105C4000BB0BBC01CD012BE0660F771F881F991F8E
:105C50002A95D1F7278530898901330F220B330B21
:105C6000A90198012C0D3D1D4E1D5F1D0E941D6256
:105C7000D701C601820F931FA41FB51F0896A11D4F
:105C8000B11DBC01CD0134E0959587957795679559
:105C90003A95D1F70E94F16020E030E040E251E413
:105CA0000E9441631F910F91FF90EF90DF90CF9082
:105CB00008951F93CF93DF931F92CDB7DEB7682F60
:105CC00087E769830E94F544698185E293E10E9438
:105CD0008C450E94984487E70E94F54461E070E09B
:105CE00087E790E0F4DE85E293E10E944145182FBA
:105CF0000E949844812F0F90DF91CF911F910895BA
:105D00003F924F925F926F927F928F929F92AF924B
:105D1000BF92CF92DF92EF92FF920F931F93CF9398
:105D2000DF93CDB7DEB728970FB6F894DEBF0FBE6E
:105D3000CDBF49DF6C01E12CF12C10912714129595
:105D4000110F110F107C1C5C87E70E94F54464EF73
:105D500085E293E10E948C45612F85E293E10E94E8
:105D60008C450E94984480912714811105C065E0FC
:105D700070E080E090E012C0813029F468E070E0CB
:105D800080E090E00BC0823029F46EE070E080E0AB
:105D900090E004C06AE170E080E090E00E945D3A2B
:105DA00086EFE0DE4C01A12CB12CBA2CA92C982C4A
:105DB000882488EF7EDF882A3090271480913C1455
:105DC00090913D14A7019601281B390B41095109F7
:105DD000A0913A14B0913B140E9439626B017C018E
:105DE000AFE0F594E794D794C794AA95D1F7609162
:105DF000341470913514CB01770FAA0BBB0BBC0187
:105E0000CD01BBE0660F771F881F991FBA95D1F7A8
:105E100020913614309137148901330F220B330B44
:105E2000A90198012C0D3D1D4E1D5F1D0E941D6294
:105E3000C20ED31EE41EF51E20EAC21A2FE0D20ABB
:105E4000E108F108A7019601C701B6010E94996512
:105E50009B01AC011CE055954795379527951A9500
:105E6000D1F729833A834B835C83009128141091E6
:105E70002914A0912C14B0912D14A70196010E9411
:105E800043622B013C018DE07594679457944794CD
:105E90008A95D1F7A0912E14B0912F1429813A81BF
:105EA0004B815C810E944362BB2797FDB095AB2F6D
:105EB000840D951DA61DB71D0296A11DB11D32E0D2
:105EC000B595A795979587953A95D1F79C01AD0122
:105ED00030584F4F5F4FA0913814B09139140E9441
:105EE00039622B013C014FE07694679457944794B4
:105EF0004A95D1F788E090E083199109A5019401B2
:105F000004C056954795379527958A95D2F72D83E6
:105F10003E834F8358874801110FAA08BB0852E0FF
:105F2000880C991CAA1CBB1C5A95D1F7A09130145F
:105F3000B091311429813A814B815C810E94436286
:105F40009B01AC016BE055954795379527956A9570
:105F5000D1F729833A834B835C83A0912A14B091B3
:105F60002B14A70196010E944362DC01CB017BE068
:105F7000B595A795979587957A95D1F729813A8117
:105F80004B815C81820F931FA41FB51F880D991D43
:105F9000AA1DBB1D032C04C0880F991FAA1FBB1F7D
:105FA0000A94D2F7BC01CD016E5F7F4F8F4F9F4F98
:105FB00024E030E040E050E00E941D628D819E812F
:105FC000AF81B885821B930BA40BB50B9C01AD016F
:105FD00080E593ECA0E0B0E0BC01CD0104C0969553
:105FE0008795779567953A94D2F70E94996597FDC2
:105FF0000BC0660F771F881F991FA30192010E9493
:10600000496269017A010AC0A30192010E944962B2
:1060100069017A01CC0CDD1CEE1CFF1C9927F7FCF2
:106020009A958F2D7E2D6D2D9B01AC010E94996557
:106030009B01AC01AEEDBBE00E9439624C01BB2478
:1060400097FCB094AB2CA3E4B3EEA70196010E9499
:106050004562BB2797FDB095AB2F880D991DAA1DF2
:10606000BB1D8153914FAF4FBF4F44E0B595A795EE
:10607000979587954A95D1F7BC01CD016C0D7D1D93
:106080008E1D9F1D28960FB6F894DEBF0FBECDBFA4
:10609000DF91CF911F910F91FF90EF90DF90CF9004
:1060A000BF90AF909F908F907F906F905F904F9038
:1060B0003F9008951F93CF93DF93CDB7DEB72C9712
:1060C0000FB6F894DEBF0FBECDBF8EE10E94F5443F
:1060D00083E090E00E9463440E9498448EE10E9415
:1060E000F54466E070E08EE190E0F1DC80915310C1
:1060F00090E020915410821B9109069741F410E022
:1061000085E293E10E9441451F5F1630C9F70E9466
:1061100098446B8170E0762F66278C81682B4D81C7
:1061200050E0542F44278E81482B298130E0322FB4
:1061300022278A81282B38872F835A8749877C8793
:106140006B8738855A857C8580E090E02C960FB669
:10615000F894DEBF0FBECDBFDF91CF911F910895A0
:10616000EF92FF920F931F93CF93DF93C82F8B0172
:106170007A0183E50E94F5446C2F85E293E10E9449
:106180008C450E94984483E50E94F544B80183E55C
:1061900090E09DDCE701CE018E199F0930915310EC
:1061A00020915410321731F085E293E10E9441456D
:1061B0008993F1CF8017910729F01092541481E050
:1061C00080935514DF91CF911F910F91FF90EF9025
:1061D0000C949844CF93DF93AC01990F660B770B27
:1061E0002AE030E088E892E12CD7EC0188E892E1DF
:1061F00075D78C0F9D1FDF91CF9108951F93CF937B
:10620000DF931F92CDB7DEB7162FAE014F5F5F4F02
:1062100061E070E0A5DF898190E002C095958795E7
:106220001A95E2F781700F90DF91CF911F91089539
:10623000CF93DF93D82FC62F83E50E94F5446D2FAF
:1062400085E293E10E948C456C2F85E293E10E94E8
:106250008C45DF91CF910C949844FF920F931F933C
:10626000CF93DF931F92CDB7DEB7182F062FF42EF2
:10627000AE014F5F5F4F61E070E072DF8981FF2008
:1062800049F041E050E001C0440F0A95EAF7482B7D
:10629000498309C021E030E001C0220F0A95EAF7E6
:1062A0002095282329836981812FC2DF0F90DF91F8
:1062B000CF911F910F91FF900895CF93DF9342E00C
:1062C000EDDAEC0188E892E109D78C0F9D1FDF9190
:1062D000CF910895AF92BF92CF92DF92EF92FF924B
:1062E0001F93CF93DF93CDB7DEB72A970FB6F894FD
:1062F000DEBF0FBECDBF182F42E654E166E070E06E
:1063000082E39F832DDF2091631430E0322F222718
:1063100080916214282B3A8329832091651430E000
:10632000322F222780916414282B3C832B832091C9
:10633000671430E0322F222780916614282B3E8389
:106340002D839E012F5F3F4F590156E5C52E54E125
:10635000D52EE12E9F81F92EF501619171915F019A
:10636000F60121913191419151916F01072E000C5D
:10637000880B990B2F83388749875A870E94F160D1
:106380002F81388549855A850E945061F7016193B4
:106390007193819391937F01F2E6CF16F4E1DF06CA
:1063A000D9F62A960FB6F894DEBF0FBECDBFDF91A7
:1063B000CF911F91FF90EF90DF90CF90BF90AF9063
:1063C00008953F924F925F926F927F928F929F9229
:1063D000AF92BF92CF92DF92EF92FF920F931F93F3
:1063E000CF93DF9300D01F921F92CDB7DEB7982EC8
:1063F0000E94953A2B013C0120ED420E27E0521EEF
:10640000611C711C60E08091D7149CD735E0832E0D
:10641000CE0101966C01AA24A394B12C55E0352E2F
:10642000380EF601282D11922A95E9F7860127E00A
:10643000E22EF12C8091D8145BD7019739F40E9499
:10644000953A6415750586059705A0F38091D814D3
:106450004FD7892B39F40E94953A64157505860546
:106460009705A0F38091D91443D7892B51F0F801F7
:106470002081C5010E2C01C0880F0A94EAF7822BF7
:106480008083F1E0EF1AF108A8F60F5F1F4F30127A
:10649000CECF0E94953A641575058605970548F09C
:1064A00061E08091D7144ED760E070E080EC9FE708
:1064B0002BC089818911B5CF9B818A81980F990D55
:1064C0008C818913AECF8D818D3009F0AACF61E028
:1064D0008091D71437D76A818B8170E0762F662739
:1064E000680F711D072E000C880B990B0E94F1603C
:1064F00020E030E040E85DE30E94506123E333E9AF
:1065000048E853E40E947A620F900F900F900F902A
:106510000F90DF91CF911F910F91FF90EF90DF903F
:10652000CF90BF90AF909F908F907F906F905F9033
:106530004F903F9008958BEE91E168D2EBEEF1E140
:10654000A289B3898C918F7E8C93A289B3898C9117
:10655000877F8C93A289B3898C918F778C93A28942
:10656000B3898C918F7D8C93828D818F08954F920A
:106570005F926F927F928F929F92AF92BF92CF92D3
:10658000DF92EF92FF92CF93DF93CDB7DEB76497A0
:106590000FB6F894DEBF0FBECDBF0E94693B698B7A
:1065A0007A8B8B8B9C8B8090530390905403A0909C
:1065B0005503B0905603A501940160915703709163
:1065C00058038091590390915A030E947A622B01DB
:1065D0003C0120E030E0A9010E94EB60882309F42F
:1065E00051C0C0904F03D0905003E0905103F09001
:1065F000520320E030E0A901C701B6010E94EB6020
:1066000018160CF03FC080914B0390914C03A09161
:106610004D03B0914E038D879E87AF87B88B9C0149
:10662000AD01C701B6010E94EB60882359F1A701B3
:1066300096016D857E858F8598890E9441630E94B1
:106640007C646D877E878F87988BA501940169890B
:106650007A898B899C890E947A62A30192010E94A7
:1066600041632D853E854F8558890E9450610E9467
:10667000AE639B01AC01C701B6010E9450616B0182
:106680007C0103C0C12CD12C760160E080E00ADAE5
:106690004CD728EE33E040E050E00E944962BA0156
:1066A000A9012AE0CE010196BBD3BE016F5F7F4FE7
:1066B00089E094E148D3CE0101967ED369E074E18C
:1066C000CE01019630D46FE77EE0CE010196D5D29F
:1066D000BC0189E094E122D3CE0101966DD30E94E2
:1066E0006E4860E080E0DED969E074E180EE94E11C
:1066F0003DD421E0B701A601CE01019662D36BE83B
:106700007EE0CE01079617D4BE016F5F7F4FCE01AA
:106710000796CAD26FE87EE0B0D2BC018FE094E168
:10672000FDD2CE01079648D3CE01019645D361E054
:1067300080E0B8D96FE074E180EE94E117D464E6AC
:1067400070E080E090E0B9D680913210882329F083
:1067500060E273E080E090E0B0D664960FB6F89403
:10676000DEBF0FBECDBFDF91CF91FF90EF90DF90E6
:10677000CF90BF90AF909F908F907F906F905F90E1
:106780004F900895FC01448155818091251490918A
:1067900026148417950780F080912114909122147B
:1067A000009751F0608171816115710529F00E9497
:1067B000336821E0892B09F020E0822F089596E0CC
:1067C000899FD0011124A859BB4E90967C936E935B
:1067D0005F9791E091969C9391979091D414E0915A
:1067E000D514F091D614992339F0309751F08111D6
:1067F00008C08091841404C0309719F05C968C9185
:10680000199408950895CF92DF92EF92FF920F931B
:106810001F93CF93DF936C017A018B01C0E0D0E02E
:10682000CE15DF0589F0D8016D918D01D601ED916E
:10683000FC910190F081E02DC6011995892B11F48E
:106840007E0102C02196ECCFC701DF91CF911F914D
:106850000F91FF90EF90DF90CF900895FC01A089F9
:10686000B1898C91A689B78982FD0FC09C91818DD9
:106870008F5F8F73228D821749F0218DDF01A20F68
:10688000B11D5D969C93818F08958C910895FC01B4
:10689000538D448D252F30E0842F90E0821B930B85
:1068A000541710F0CF96089501970895FC01918D2B
:1068B000828D981761F0828DDF01A80FB11D5D9662
:1068C0008C91928D9F5F9F73928F90E008958FEFD0
:1068D0009FEF0895FC01918D828D981731F0828D84
:1068E000E80FF11D858D90E008958FEF9FEF0895DB
:1068F000FC01918D228D892F90E0805C9F4F821B3F
:1069000091098F73992708958EE491E1F1DF21E0D9
:10691000892B09F420E0822F08958BEE91E1E8DFC6
:1069200021E0892B09F420E0822F089588E892E184
:10693000DFDF21E0892B09F420E0822F0895FC019C
:10694000848DDF01A80FB11DA35ABF4F2C91848DF8
:1069500090E001968F739927848FA689B7892C932D
:10696000A089B1898C9180648C93938D848D9813C8
:1069700006C00288F389E02D80818F7D8083089591
:10698000EF92FF920F931F93CF93DF93EC0181E07F
:10699000888F9B8D8C8D981305C0E889F98980813B
:1069A00085FD23C0F62E0B8D10E00F5F1F4F0F7378
:1069B0001127E02E8C8DE8120BC00FB607FCFACF22
:1069C000E889F989808185FFF5CFCE01B8DFF2CF64
:1069D0008B8DFE01E80FF11DE35AFF4FF0820B8F04
:1069E000EA89FB898081806207C0EE89FF89608324
:1069F000E889F98980818064808381E090E0DF917B
:106A0000CF911F910F91FF90EF900895CF93DF9357
:106A1000EC01888D8823C1F0EA89FB89808185FD9E
:106A200005C0A889B9898C9186FD0EC00FB607FCF8
:106A3000F5CF808185FFF2CFA889B9898C9185FF38
:106A4000EDCFCE017CDFE8CFDF91CF91089580E0DC
:106A500090E0892B19F06ADF81111BC080E090E083
:106A6000892B41F080E090E0892B21F00E9400000A
:106A7000811112C080E090E0892B19F04EDF811166
:106A80000EC080E090E0892B79F03EDF81110AC0D2
:106A900008950E940000E2CF0E940000EBCF0E9408
:106AA0000000EFCF0C940000089590E0FC013197B6
:106AB000E231F10508F04EC08827EA57FF4F8F4FAB
:106AC0000C94BB65809180008F7703C0809180001B
:106AD0008F7D80938000089580918000877FF9CF1B
:106AE00084B58F7702C084B58F7D84BD0895809171
:106AF000B0008F7703C08091B0008F7D8093B0008D
:106B00000895809190008F7707C0809190008F7DCD
:106B100003C080919000877F8093900008958091BA
:106B2000A0008F7707C08091A0008F7D03C0809167
:106B3000A000877F8093A0000895809120018F7727
:106B400007C0809120018F7D03C080912001877F45
:106B50008093200108950E941F68CF93DF93EC017A
:106B600088819981009711F00E94A366198218828A
:106B70001D821C821B821A82DF91CF9108950F9390
:106B80001F93CF93DF93EC0188819981009729F0BF
:106B90002A813B812617370788F48B016F5F7F4F6F
:106BA0000E943B67009761F0998388831B830A8367
:106BB0002C813D81232B11F4FC01108281E001C066
:106BC00080E0DF91CF911F910F910895EF92FF9296
:106BD0000F931F93CF93DF93EC017B018A01BA01DE
:106BE000CEDF811103C0CE01B8DF07C01D830C8347
:106BF000B701888199810E942C68CE01DF91CF91E5
:106C00001F910F91FF90EF900895FC018081918179
:106C1000009711F00C94455C60E070E0CB010895A2
:106C2000EF92FF920F931F93CF93DF93FC01248188
:106C300035816115710511F480E018C041155105C9
:106C4000A1F07B01EC018A01020F131FB80197DF4D
:106C5000882391F3288139818C819D81B701820F2E
:106C6000931F0E942C681D830C8381E0DF91CF91DC
:106C70001F910F91FF90EF900895CF93DF93EC0158
:106C80006115710559F0FB0101900020E9F731977A
:106C9000AF01461B570BC4DF811102C0CE015DDF7F
:106CA000CE01DF91CF910895CF93DF93EC01FB01EB
:106CB0004481558160817181B3DF811102C0CE01B1
:106CC0004CDFCE01DF91CF9108956115710549F038
:106CD000FB0101900020E9F73197AF01461B570BEC
:106CE0009FCF80E00895FB014481558160817181CF
:106CF00097CFCF93DF93EC016115710551F0FB0144
:106D000001900020E9F73197AF01461B570B5EDF7A
:106D100001C023DFCE01DF91CF910895CF93DF93A0
:106D2000EC01FB018617970751F0608171816115B5
:106D3000710521F04481558149DF01C00EDFCE018C
:106D4000DF91CF9108950F931F93CF93DF938C0121
:106D5000EB01FC01808191810097B1F0688179811C
:106D60006115710579F0428153812C813D81421773
:106D7000530740F00E942C688C819D81F801958317
:106D8000848313C00E94A36688819981F80191834E
:106D900080838A819B81938382838C819D8195836B
:106DA0008483198218821B821A821D821C82DF91C1
:106DB000CF911F910F910895FC01808191810C94D6
:106DC000A366EF92FF920F931F93CF93DF93CDB7FC
:106DD000DEB7A1970FB6F894DEBF0FBECDBF7C0122
:106DE000CB01BA01F701118210821382128215823F
:106DF000148242E0420F8E010F5F1F4F0E94235CFE
:106E0000BC01C70176DFA1960FB6F894DEBF0FBEB6
:106E1000CDBFDF91CF911F910F91FF90EF9008951B
:106E20000F931F93CF93DF93CDB7DEB7A1970FB624
:106E3000F894DEBF0FBECDBF8C01CB01BA01F801C3
:106E400011821082138212821582148230E0AE0108
:106E50004F5F5F4F0E94AC5CBE016F5F7F4FC80108
:106E600048DFA1960FB6F894DEBF0FBECDBFDF910D
:106E7000CF911F910F9108950F931F93CF93DF939D
:106E8000CDB7DEB7A2970FB6F894DEBF0FBECDBF69
:106E90008C01CB01BA01F801118210821382128297
:106EA0001582148230E0AE014F5F5F4F0E947F5C1D
:106EB000BE016F5F7F4FC8011CDFA2960FB6F8942A
:106EC000DEBF0FBECDBFDF91CF911F910F9108950F
:106ED0000F931F93CF93DF93CDB7DEB762970FB6B3
:106EE000F894DEBF0FBECDBF8C01CB01F80111823B
:106EF0001082138212821582148250E0BE016F5FED
:106F00007F4F0E946B5CBE016F5F7F4FC801F1DE57
:106F100062960FB6F894DEBF0FBECDBFDF91CF9162
:106F20001F910F910895FC01118210821382128229
:106F300015821482F3CEFC01118210821382128218
:106F4000158214826115710549F0FB010190002042
:106F5000E9F73197AF01461B570B38CE0895DC0196
:106F6000ED91FC910190F081E02D1994DC01ED91FF
:106F7000FC91DB0114964D915C9115976D917C917C
:106F80000280F381E02D19946115710579F0FB0100
:106F900001900020E9F73197AF01461B570BDC0148
:106FA000ED91FC910280F381E02D199480E090E056
:106FB00008954F925F926F927F92EF92FF920F939C
:106FC0001F93CF93DF93CDB7DEB7A1970FB6F89499
:106FD000DEBF0FBECDBF7C01FA01CB0119A222306A
:106FE00008F42AE08E010F5D1F4F422E512C612CB8
:106FF000712CBF01A30192010E944962F901CA01EB
:10700000015011096A3014F4605D01C0695CD80157
:107010006C93232B242B252B61F7B801C701B4DF18
:10702000A1960FB6F894DEBF0FBECDBFDF91CF9112
:107030001F910F91FF90EF907F906F905F904F9016
:107040000895CF92DF92EF92FF920F931F93CF9309
:10705000DF93EC016A017B012115310579F4E881A8
:10706000F9810190F081E02D642FDF91CF911F9184
:107070000F91FF90EF90DF90CF9019942A30310557
:10708000D9F477FF18C06DE26ADF8C0144275527D9
:10709000BA014C195D096E097F092AE0CE0189DF2A
:1070A000800F911FDF91CF911F910F91FF90EF9073
:1070B000DF90CF9008952AE0B701A601CE01DF91BD
:1070C000CF911F910F91FF90EF90DF90CF9071CFF4
:1070D0009A01AB01770F660B770BB3CF63E97EE0C4
:1070E00053CF0F931F93CF93DF93EC013FDF8C01BE
:1070F000CE01F4DF800F911FDF91CF911F910F918F
:10710000089542CF1F920F920FB60F9211240BB623
:107110000F922F933F934F935F936F937F938F9330
:107120009F93AF93BF93EF93FF938EE491E107DCBE
:10713000FF91EF91BF91AF919F918F917F916F914F
:107140005F914F913F912F910F900BBE0F900FBE0B
:107150000F901F9018951F920F920FB60F92112447
:107160000BB60F922F933F934F935F936F937F9341
:107170008F939F93AF93BF93EF93FF938EE491E12F
:107180006DDBFF91EF91BF91AF919F918F917F91B7
:107190006F915F914F913F912F910F900BBE0F9088
:1071A0000FBE0F901F9018951F920F920FB60F925F
:1071B00011240BB60F922F933F934F935F936F93CE
:1071C0007F938F939F93AF93BF93EF93FF938BEE38
:1071D00091E1B5DBFF91EF91BF91AF919F918F91BD
:1071E0007F916F915F914F913F912F910F900BBEC7
:1071F0000F900FBE0F901F9018951F920F920FB611
:107200000F9211240BB60F922F933F934F935F93DE
:107210006F937F938F939F93AF93BF93EF93FF935E
:107220008BEE91E11BDBFF91EF91BF91AF919F91AD
:107230008F917F916F915F914F913F912F910F901F
:107240000BBE0F900FBE0F901F9018951F920F92BC
:107250000FB60F9211240BB60F922F933F934F93BB
:107260005F936F937F938F939F93AF93BF93EF93AE
:10727000FF9388E892E163DBFF91EF91BF91AF91BB
:107280009F918F917F916F915F914F913F912F913E
:107290000F900BBE0F900FBE0F901F9018951F926E
:1072A0000F920FB60F9211240BB60F922F933F93AC
:1072B0004F935F936F937F938F939F93AF93BF93FE
:1072C000EF93FF9388E892E1C9DAFF91EF91BF91C4
:1072D000AF919F918F917F916F915F914F913F916E
:1072E0002F910F900BBE0F900FBE0F901F9018950F
:1072F000CF93DF93282F30E0F901E151FC4F8491C7
:10730000F901E755FC4FD491F901ED59FC4FC491B7
:10731000CC2389F08111C9DBEC2FF0E0EE0FFF1FC9
:10732000E75BFC4FA591B491EC91ED2381E090E0F7
:1073300021F480E002C080E090E0DF91CF910895D9
:10734000862FD6CF1F93CF93DF93282F30E0F901FC
:10735000E151FC4F8491F901E755FC4FD491F901BB
:10736000ED59FC4FC491CC23C1F0162F81119DDB48
:10737000EC2FF0E0EE0FFF1FE15DFC4FA591B49103
:107380008FB7F894111105C09C91ED2FE095E9237A
:1073900002C0EC91ED2BEC938FBFDF91CF911F9149
:1073A0000895862F642FCECFCF93DF9390E0FC011A
:1073B000E755FC4F2491FC01ED59FC4F8491882343
:1073C00061F190E0880F991FFC01EB5EFC4FC591C5
:1073D000D491FC01E15DFC4FA591B491611109C00C
:1073E0009FB7F8948881209582238883EC912E237F
:1073F0000BC0623061F49FB7F8943881822F80957A
:1074000083238883EC912E2B2C939FBF06C08FB7CC
:10741000F894E8812E2B28838FBFDF91CF910895B8
:10742000862F642FC1CF863308F0865390917B005E
:10743000282F2870977F922B90937B008770209144
:107440005B0390E4299F90011124822B80937C00A0
:1074500080917A00806480937A0080917A0086FD22
:10746000FCCF809178002091790090E0922B0895D4
:107470003FB7F89480915A1090915B10A0915C10E6
:10748000B0915D1026B5A89B05C02F3F19F001965D
:10749000A11DB11D3FBFBA2FA92F982F8827820F9A
:1074A000911DA11DB11DBC01CD0142E0660F771FEA
:1074B000881F991F4A95D1F708958F929F92AF9296
:1074C000BF92CF92DF92EF92FF926B017C01D0DFEF
:1074D0004B015C01C114D104E104F104E9F0C8DFFF
:1074E000DC01CB0188199909AA09BB09883E9340A0
:1074F000A105B10578F321E0C21AD108E108F1082D
:1075000088EE880E83E0981EA11CB11CC114D10422
:10751000E104F10421F7DECFFF90EF90DF90CF90F0
:10752000BF90AF909F908F9008952FB7F89460917F
:1075300056107091571080915810909159102FBF8C
:1075400008951F920F920FB60F9211242F933F931D
:107550008F939F93AF93BF93809156109091571044
:10756000A0915810B09159103091551023E0230F7D
:107570002D3720F40196A11DB11D05C026E8230F6B
:107580000296A11DB11D2093551080935610909323
:107590005710A0935810B093591080915A109091A1
:1075A0005B10A0915C10B0915D100196A11DB11D02
:1075B00080935A1090935B10A0935C10B0935D1071
:1075C000BF91AF919F918F913F912F910F900FBEDF
:1075D0000F901F901895CF93DF93EC0160E08E81A0
:1075E000B1DE61E08E81AEDE60E08E81ABDE8BE8E5
:1075F00091E00197F1F7DF91CF910895CF92DF925B
:10760000EF92FF920F931F93CF93DF937C016C0156
:1076100087E0C80ED11CC0E0D0E0062F10E0B80112
:107620000C2E02C0759567950A94E2F76170F60119
:1076300081916F0187DE2196C430D10581F7C701A2
:10764000DF91CF911F910F91FF90EF90DF90CF903E
:10765000C2CFCF92DF92EF92FF921F93CF93DF932F
:10766000182FCAE0D0E0C12CD12C7601812FDBDEAF
:10767000BC01990F880B990B0E94F1609B01AC0132
:10768000C701B6010E947B626B017C0162E370E07E
:1076900080E090E012DF219749F720E030E040E2FF
:1076A00051E4C701B6010E94416320E030E040EAA6
:1076B00050E40E94506120E030E040E85AE30E942C
:1076C0005061DF91CF911F91FF90EF90DF90CF90AD
:1076D00008951F93CF93DF93182FCEEFD0E1812F22
:1076E000A2DE899399936CE370E080E090E0E5DEA0
:1076F00081E1CE34D80799F781D620E030E040EA26
:1077000050E40E94506120E030E040E85AE30E94DB
:107710005061DF91CF911F9108954F925F926F92C8
:107720007F928F929F92AF92BF92CF92DF92EF9211
:10773000FF920F931F93CF93DF93CDB7DEB72C97B4
:107740000FB6F894DEBF0FBECDBF61E080E00E94AF
:10775000522D66E97EE080EE94E1D3DC64EF71E0C7
:1077600080E090E0AADE60E080E00E94522DDDDE45
:1077700028EE33E040E050E00E944962BA01A901DE
:107780002AE080EE94E115DC67EA7EE080EE94E189
:10779000B8DC19821A821B821C821D8261E087E399
:1077A00003DE60E087E3CEDD62E170E080E090E040
:1077B00084DE61E087E3C6DD8BE990E00197F1F7B5
:1077C00060E087E3F1DD01E117E287E391DD892BDA
:1077D00031F401501109C9F78EEF9FEF6DC001E13F
:1077E00017E287E385DD019721F401501109C9F7FC
:1077F000F3CF28E2E22EF12C17E0D12CAA24A39497
:10780000B12C91E1892E97E2992E87E371DD892BC6
:1078100029F481E0881A9108C1F7DECF29DE2B0117
:107820003C0181E1882E87E2982E87E361DD019794
:1078300029F481E0881A9108C1F7CECF19DEDC0166
:10784000CB0184199509A609B7098997A105B10546
:1078500078F0E1E0F0E0EC0FFD1FED0DF11D20816F
:10786000C501012E01C0880F0A94EAF7822B80839C
:10787000111103C0D39417E001C0115081E0E81A40
:10788000F10809F0BECF8981282F30E030936710CE
:10789000209366102B81422F50E050936910409343
:1078A0006810280F81E090E03D81321302C080E033
:1078B00090E0919581959109892B09F00CC1609117
:1078C000681070916910072E000C880B990B0E94AC
:1078D000F1606B017C016093621070936310809380
:1078E0006410909365108091661090916710BC01B0
:1078F000990F880B990B0E94F16060935E10709352
:107900005F10809360109093611021E030E0B70128
:10791000A601CE0107960E949C4866E775E0CE015D
:10792000019609DBBE01695F7F4FCE010196BCD98C
:10793000BC018FE094E1F2D9CE0101963DDACE018F
:1079400007963ADA40915E1050915F106091601096
:107950007091611021E030E0CE0107960E949C48B2
:107960006DEA7EE0CE010196E6DABE01695F7F4FE7
:10797000CE01019699D9BC018FE094E1B4D9CE0132
:1079800001961ADACE01079617DA69EF77E08FE0F1
:1079900094E19BD960E086E00E94522D60916210D4
:1079A0007091631080916410909165100E94DA6369
:1079B0004AE050E080EE94E18BDB6FED80EE94E1E5
:1079C000CEDA63EB7EE080EE94E19BDB60915E10AB
:1079D00070915F1080916010909161100E94DA6345
:1079E0004AE050E080EE94E173DB66EB7EE080EEEF
:1079F00094E187DB64E670E080E090E05EDD8BE19F
:107A000094E103D9613071058105910509F0D7C072
:107A100061E080E00E94522D64E67FE080EE94E118
:107A200070DB61E080E00E94522DC0906210D09027
:107A30006310E0906410F090651020E030E040EFBB
:107A400051E4C701B6010E94306487FD03C06AEBB0
:107A50007EE038C020E030E040ED51E4C701B601DF
:107A60000E94306487FD11C06AEC7EE080EE94E1F4
:107A700048DB6CED75E080E090E01FDD61E080E0C8
:107A80000E94522D6AED7EE01DC020E030E040EB08
:107A900051E4C701B6010E94306487FD03C06AEE5D
:107AA0007EE010C06AEF7EE080EE94E12ADB6CEDB0
:107AB00075E080E090E001DD61E080E00E94522D01
:107AC0006AE07FE080EE94E11CDB6CED75E080E025
:107AD00090E0F3DC74C00E946E486EE170E080E0DC
:107AE00090E0EBDC0E94FA2D6B017C0164E670E013
:107AF00080E090E0E2DC60E080E00E94522D15DD45
:107B000028EE33E040E050E00E944962BA01A9014A
:107B10002AE0CE01079684D9BE01695F7F4FCE016E
:107B2000019601DA61E175E0CE010196A6D8BC01AB
:107B300089E094E1F3D8CE0101963ED9CE010796B3
:107B40003BD966E775E08FE094E1D3D821E030E0DF
:107B5000B701A601CE0101960E949C48BE016F5F4D
:107B60007F4F8FE094E1BFD8CE01019625D96DE912
:107B700079E08FE094E1A9D869E074E1CE01019643
:107B8000D2D96FE074E1CE0101968ED8BC018FE0AE
:107B900094E1C4D8CE0101960FD96FE074E180EE74
:107BA00094E1E4D961E080E00E94522DC09262101D
:107BB000D0926310E0926410F09265103ECF2C9644
:107BC0000FB6F894DEBF0FBECDBFDF91CF911F91EE
:107BD0000F91FF90EF90DF90CF90BF90AF909F906C
:107BE0008F907F906F905F904F900895CF93DF9329
:107BF000EC01BC0188E892E174DABE018EE491E107
:107C0000DF91CF916ECA2F923F924F925F926F9207
:107C10007F928F929F92AF92BF92CF92DF92EF921C
:107C2000FF920F931F93CF93DF93CDB7DEB7C3546B
:107C3000D1090FB6F894DEBF0FBECDBF6EAF7FAFD8
:107C40001C0129AB3AAB4BAB5CAB6FDC24966CAF41
:107C50007DAF8EAF9FAF249729A93AA94BA95CA904
:107C60002A303105410551052CF42DA73EA74FA719
:107C700058AB08C08AE090E0A0E0B0E08DA79EA7D6
:107C8000AFA7B8AB80913210882341F029A93AA957
:107C90004BA95CA92DA73EA74FA758AB31E03DAF3C
:107CA00094EF492E55245394612C712C19A61AA6D1
:107CB0001BA61CA68E01035F1F4F89A59AA5ABA525
:107CC000BCA52DA53EA54FA558A982179307A407CB
:107CD000B5070CF0D1C229DC24962CAD3DAD4EADDC
:107CE0005FAD2497621B730B840B950B0E94EF60B2
:107CF00020E030E04AE754E40E944163AB01BC015C
:107D000022E030E0C8010E949C48B80189E094E17B
:107D10001AD8C80151D8CE0101960E946A316AE191
:107D20007FE08FE094E10E947936AE014F5F5F4FB4
:107D30005EA34DA3C12CD12C7601ADA1BEA18D9027
:107D40009D90AD90BD90BEA3ADA3A5019401C501CA
:107D5000B4010E9450619B01AC01C701B6010E94B1
:107D60007B626B017C0123E030E0B501A401C80116
:107D70000E949C48B801CE014396D5D862E77FE0C7
:107D8000CE0143960E943D36BC018FE094E10E94F3
:107D90007336CE01439610D8C8010ED8EDA1FEA1CE
:107DA000E017F10751F6C701B6010E943F656B016C
:107DB0007C01FDE24F16F1E05F066104710434F0CE
:107DC0000E946E4860E080E00E94522D23E030E087
:107DD000B701A601CE0143960E949C4864E97EE06B
:107DE000C801A9D869E074E1C8010E94543667E26D
:107DF0007FE00E943D36BE016D5E7F4F0E9454368B
:107E00006CE27FE00E943D36BC018FE094E10E946D
:107E10007336C8010E94DC36CE0143960E94DC36E0
:107E200026E636E646E65FE3C701B6010E94306407
:107E300089849A84AB84BC8418160CF080C12DEC24
:107E40003CEC4CE85FE3C701B6010E94EB6087FFA2
:107E500082C12DAD222309F489C120E030E0A901BF
:107E6000C501B4010E94EB60C980DA80EB80FC8020
:107E70002D813E814F8158852DA33EA34FA358A746
:107E8000882309F1A7019601C701B6010E9450613C
:107E90006DAB7EAB8FAB98AF2DA13EA14FA158A586
:107EA000CA01B9010E9450619B01AC016DA97EA974
:107EB0008FA998AD0E947B620E943F65A501940145
:107EC0000E94EE6204C06BED7FE089EC9FE320EE40
:107ED0003EE245E652E40E9450616DAB7EAB8FAB53
:107EE00098AF20E030E0A9016DA17EA18FA198A5F7
:107EF0000E94EB60882309F1A7019601C701B60132
:107F00000E94506169AF7AAF8BAF9CAFA50194011D
:107F1000C501B4010E9450619B01AC0169AD7AAD0D
:107F20008BAD9CAD0E947B620E943F652DA13EA15E
:107F30004FA158A50E94EE6204C06BED7FE089EC72
:107F40009FE320EE3EE245E652E40E94506169AFB5
:107F50007AAF8BAF9CAF20E030E0A901C701B6013A
:107F60000E94EB608823F9F0A5019401C501B401DA
:107F70000E9450614B015C012DA13EA14FA158A56B
:107F8000CA01B9010E9450619B01AC01C501B40155
:107F90000E947B620E943F65A70196010E94EE62EB
:107FA0006B017C0108C08BEDC82E8FE0D82E89ECC8
:107FB000E82E8FE3F82E6FE27FE08FE094E10E94DD
:107FC0007936B3DA28EE33E040E050E00E944962AF
:107FD000BA01A9012AE0C8010E941037B801CE01F8
:107FE00043960E94933767E47FE0CE0143960E9458
:107FF0003D36BC0189E094E10E948E36CE01439665
:108000000E94DC36C8010E94DC3621E04DA95EA941
:108010006FA978ADCE014F960E94E13621E049ADBF
:108020005AAD6BAD7CADCE0149960E94E13620EE93
:108030003EE245E652E4C701B6010E945061AB0141
:10804000BC0121E0C8010E94E136B801CE0143968F
:108050000E94933762E77FE0CE0143960E943D364F
:10806000BE01675E7F4F0E94543662E77FE00E9448
:108070003D36BE01615E7F4F0E945436BC0183E0F5
:1080800094E10E948E36CE0143960E94DC36C801F0
:108090000E94DC36CE0149960E94DC36CE014F9616
:1080A0000E94DC363DE2431631E053066104710460
:1080B00044F489A59AA5ABA5BCA5892B8A2B8B2B4B
:1080C00081F469E074E180EE94E10E94B63761E0EA
:1080D00080E00E94522D63E074E180EE94E10E9402
:1080E000B63763E074E18FE094E10E9473369DE25D
:1080F000491691E059066104710444F429A53AA592
:108100004BA55CA5232B242B252B51F46FE074E1A8
:10811000C8010E949337C80169DDC8010E94DC369E
:10812000C301B201CAD989A59AA5ABA5BCA5019680
:10813000A11DB11D89A79AA7ABA7BCA790C04EAC43
:108140005FAC310129A93AA94BA95CA92DA73EA78B
:108150004FA758AB0BC04EAC5FAC310189A99AA9AF
:10816000ABA9BCA98DA79EA7AFA7B8AB23E030E011
:10817000B501A401CE014396DFD764E57FE0C801D5
:108180000E949B37BE016D5E7F4FC8010E9454362E
:108190006DE27FE00E943D36BC0189E094E10E94DF
:1081A0007336C8010E94DC36CE0143960E94DC364D
:1081B0009DE2491691E059066104710454F069E0AA
:1081C00074E180EE94E10E94B63761E080E00E94A5
:1081D000522D4D815E816F81788523E030E0CE01A4
:1081E0004996AAD749815A816B817C8123E030E08E
:1081F000C801A2D7B801CE0143960E9493376AE521
:108200007FE0CE0143960E943D36BE01675E7F4F00
:108210000E9454366DE27FE00E943D36BC0183E04F
:1082200094E10E948E36CE0143960E94DC36C8014E
:108230000E94DC36CE0149960E94DC36ADE24A1639
:10824000A1E05A066104710434F063E074E180EE49
:1082500094E10E94B637C301B2012FD91DAE29A502
:108260003AA54BA55CA52F5F3F4F4F4F5F4F29A706
:108270003AA74BA75CA721CD31D761E080E00E94EF
:10828000522D63E074E180EE94E10E94B63760E025
:1082900080E00E94522D69E074E180EE94E10E943A
:1082A000B637CD5BDF4F0FB6F894DEBF0FBECDBF44
:1082B000DF91CF911F910F91FF90EF90DF90CF90C2
:1082C000BF90AF909F908F907F906F905F904F90F6
:1082D0003F902F900895EF92FF920F931F93CF93AB
:1082E000DF93EC01623018F08F8588608F876B8B8D
:1082F0001C8A80E48D8B80E18E8B80E58F8B61E022
:108300008C8152D88D818F3F11F061E04DD861E0B2
:108310008E814AD87E0187E0E80EF11C00E010E073
:108320008F8584FD03C084E090E002C088E090E087
:108330000817190744F461E0F70181917F0134D8EF
:108340000F5F1F4FEDCF8BE39DE00197F1F760E0EA
:108350008C810E94A23960E08E810E94A2398D81B9
:108360008F3F19F060E00E94A2396F8564FD19C04B
:1083700063E0CE0143D90BE416E4C8010197F1F79D
:1083800063E0CE013BD9C8010197F1F763E0CE016C
:1083900035D983E592E00197F1F762E0CE012ED95D
:1083A00013C06062CE0142D48BE496E40197F1F7EA
:1083B0006F856062CE013AD483E592E00197F1F7D0
:1083C0006F856062CE0132D46F856062CE012ED49B
:1083D00084E0888BCE012CD461E0CE0127D48BE3DE
:1083E0009FE10197F1F782E0898B66E0CE01DF9192
:1083F000CF911F910F91FF90EF9018C42F923F9251
:108400004F925F926F927F928F929F92AF92BF92A4
:10841000CF92DF92EF92FF920F931F93CF93DF9350
:1084200000D01F92CDB7DEB74091FE105091FF10E3
:10843000C0900011D09001114C155D052CF03C2D21
:108440002D2D6A01432F522FE2E0F1E160E070E050
:10845000CB01019111910417150754F44A01550FEE
:10846000AA08BB08680D791D8A1D9B1DA80115C0AF
:10847000C016D10654F40D2C000CEE08FF086C0D4C
:108480007D1D8E1D9F1D680108C0012E000C220B52
:10849000330B600F711F821F931F21E1EE34F2072F
:1084A000C1F60E94F16020E030E048E152E40E9411
:1084B00041636B017C010EEF10E1812C912C540182
:1084C000D8016D917D918D01072E000C880B990BC1
:1084D0000E94F160A70196010E947A629B01AC01A3
:1084E0000E9450619B01AC01C501B4010E947B62F6
:1084F0004B015C01B1E10E341B0711F720E030E0C5
:108500004CE152E40E9441630E943F654B015C01D3
:1085100020E030E040E85FE30E94306418160CF081
:1085200062C00EEF10E1212C312C412C512C320174
:10853000F801819191918F019C01990F440B550B8A
:1085400029833A834B835C83CA01B9010E94F1609D
:10855000A70196010E947A620E94DA639B0177FF6D
:1085600004C022273327261B370BB901330F880B92
:10857000990B0E94F160A50194010E94EB6087FFB6
:108580000BC089819A81AB81BC81480E591E6A1E3D
:108590007B1E9FEF291A390AA1E10E341A0741F612
:1085A00020E030E040EC5FE3C501B4010E9450617F
:1085B0004B015C01B5E02B1631040CF4B2CFC301C2
:1085C000B2010E94F1606B017C01B101330C880B98
:1085D000990B0E94F1609B01AC01C701B6010E949A
:1085E00041636B017C01C701B6010F900F900F90A2
:1085F0000F90DF91CF911F910F91FF90EF90DF903F
:10860000CF90BF90AF909F908F907F906F905F9032
:108610004F903F902F900895CF93DF93BC0188E84F
:1086200092E10E94C437EC0188E892E10E946E3822
:108630008C0F9D1FDF91CF9108954F925F926F92A3
:108640007F928F929F92AF92BF92CF92DF92EF92E2
:10865000FF920F931F93CF93DF9300D01F92CDB75C
:10866000DEB76B017C0111E0A12EB12C4501880C15
:10867000991C880C991CF401EC58FC4F40805180E7
:1086800062807380A3019201C701B6010E94306429
:10869000181614F41F5FE8CFA3019201C701B601B9
:1086A0000E94EB608401045A1C4F811106C0D8015E
:1086B0006D917D918D919C9142C0C5018150904CEE
:1086C000880F991F880F991FFC01EC58FC4F2081DF
:1086D00031814281538129833A834B835C83FC013E
:1086E000E45AFC4F80809180A280B380C701B6011C
:1086F0000E947A626B017C01A5019401D8016D9101
:108700007D918D919C910E947A629B01AC01C70181
:10871000B6010E9450616B017C0129813A814B8135
:108720005C81C301B2010E947A629B01AC01C70166
:10873000B6010E944163A50194010E947B620F90E3
:108740000F900F900F90DF91CF911F910F91FF909D
:10875000EF90DF90CF90BF90AF909F908F907F90E1
:108760006F905F904F900895DF92EF92FF920F937A
:108770001F93CF93DF937C018B01EA0146175707C4
:1087800020F4812F8A01C62FD82F65E97EE0C7012A
:108790000E949B3780912514909126140817190781
:1087A000E0F48C179D0708F4EC01E0912114F0919E
:1087B0002214EC0FFD1FD080108260912114709163
:1087C0002214600F711FC7010E947936E0912114B5
:1087D000F0912214EC0FFD1FD082C701DF91CF91E1
:1087E0001F910F91FF90EF90DF900895CF93DF934B
:1087F000EC014091251450912614B6DFCE01DF9193
:10880000CF9108950F931F930E94953A6093F311AF
:108810007093F4118093F5119093F611E091EB11A0
:10882000F091EC110284F385E02D8BEE91E1199526
:1088300097FF1FC00E94953A0091F3111091F41117
:108840002091F5113091F611DC01CB01801B910BC9
:10885000A20BB30B0091EF111091F0112091F111C7
:108860003091F21180179107A207B307B8F28FEF8A
:108870009FEF1F910F910895FC01A089B18982E0BB
:108880008C93A485B5851C92A685B7858FEC8C93B7
:10889000108EA489B58986E08C93A289B3898C91C6
:1088A00080618C93A289B3898C9188608C93A28912
:1088B000B3898C9180688C930288F389E02D808144
:1088C0008F7D80830895682F85E293E125C1CF9243
:1088D000DF92EF92FF920F931F93CF93DF931F923C
:1088E000CDB7DEB76C0104EB10E17C018AE4E80E41
:1088F000F11CF80161918F01C60169830E94076232
:108900006981681719F0C6010E940F62FFEFCF1A44
:10891000DF0ACE14DF0469F784EB90E10F90DF915A
:10892000CF911F910F91FF90EF90DF90CF9008951E
:108930002091B3109091F814213208F04AC0809130
:1089400090108111FCCF32E03093901031E03093E1
:108950008F103FEF30938E1010928D1020938C105B
:10896000A3E9B0E14CE650E1FA013E2F341B321787
:1089700018F43D913193F9CF10926B1020916B1048
:10898000990F922B90936B1090916A10913061F433
:1089900010926A1090916B109093BB009091BC0064
:1089A00093FDF8CF95EC01C095EE9093BC009091AB
:1089B00090109230E1F390918E109F3F79F080916A
:1089C0008E10803241F080918E10803331F084E03F
:1089D00005C081E003C082E001C083E010929210E4
:1089E0001092B31010929110089591E0909391100D
:1089F0008093F814109292101092B310089585EDA0
:108A00008093BC008091BC0084FDFCCF109290103C
:108A1000089540911B15262F30E0240F311D21327F
:108A20003105DCF4209190102430C9F4FC0180E081
:108A300090E0861758F430911B152191DC01A75066
:108A4000BB4EA30FB11D2C930196F3CF80911B1544
:108A5000680F60931B1580E0089581E0089582E01F
:108A600008950895E091541080915310E81730F460
:108A7000F0E0ED5CFF4E808190E008958FEF9FEF76
:108A800008959091541080915310981750F4E92F45
:108A9000F0E0ED5CFF4E208130E09F5F909354103A
:108AA00002C02FEF3FEFC90108958091531090E06D
:108AB00020915410821B91090895CF92DF92EF927A
:108AC000FF920F931F93CF93DF937C01262F972F55
:108AD0008A0180919110882391F0C62FD72F6E01C3
:108AE000C40ED51ECC15DD0569F06991D701ED9155
:108AF000FC910190F081E02DC7011995F3CF642F0F
:108B0000822F87DFC801DF91CF911F910F91FF90D6
:108B1000EF90DF90CF900895CF93DF931F92CDB762
:108B2000DEB76983209191102223D1F02091B310F8
:108B3000203240F021E030E0FC013383228380E0EA
:108B400090E014C080919210E82FF0E0ED56FF4EB7
:108B5000998190838F5F809392108093B31004C0AB
:108B600061E0CE01019655DF81E090E00F90DF914A
:108B7000CF910895089580E090E00895CF92DF921C
:108B8000EF92FF920F931F93CF93DF93EC01F62E9A
:108B9000642F8C810E94A2398D818F3F19F060E093
:108BA0000E94A2398F850F2D10E084FF25C06E0131
:108BB00087E0C80ED11CE12CF12CB8010E2C02C0AC
:108BC000759567950A94E2F76170F60181916F01DE
:108BD0000E94A239FFEFEF1AFF0A88E0E816F104BD
:108BE00061F7CE01DF91CF911F910F91FF90EF9030
:108BF000DF90CF900C94EB3AB80184E075956795BF
:108C00008A95E1F7CE010E94FE3A6F2DCE01DF91E9
:108C1000CF911F910F91FF90EF90DF90CF900C9428
:108C2000FE3A41E0ABDF81E090E0089540E0A6CF5E
:108C3000FC016089262F2460208B6C60F7CF1F9287
:108C40000F920FB60F9211240F900FBE0F901F902E
:108C500018951F920F920FB60F9211240BB60F9218
:108C60002F933F934F935F936F937F938F939F9334
:108C7000AF93BF93EF93FF93809132130E947839A3
:108C800020913513309136132F5F3F4F30933613B9
:108C90002093351390913413953618F096E0909305
:108CA0003113909131139430C9F128F4923069F066
:108CB0009330D1F05EC0953009F451C0963009F080
:108CC00058C091E09093011451C0811152C020917D
:108CD0003513309136132436310508F442C0109212
:108CE0000114109234131CC0813009F042C0E0918D
:108CF000341391E09E0F90933413F0E020913513DC
:108D000030913613EE0FFF1FE95CFC4E3183208358
:108D1000109236131092351394E029C0811117C0B8
:108D2000E091341391E09E0F90933413F0E0209182
:108D3000351330913613EE0FFF1FE95CFC4E318383
:108D40002083109236131092351393E010C02091B7
:108D50003513309136132536310558F007C081118F
:108D600008C0109236131092351303C095E090930B
:108D7000311390913313992329F0811102C02F9A56
:108D800001C02F98FF91EF91BF91AF919F918F916B
:108D90007F916F915F914F913F912F910F900BBEFB
:108DA0000F900FBE0F901F901895CF92DF92EF9209
:108DB000FF92CF93DF93EC01072E000C880B990BE9
:108DC0000E94F1606B017C0120E030E040E45FE351
:108DD0000E94506120E030E048E452E40E94416388
:108DE0000E94DA63C617D707D4F020E030E040EAEB
:108DF0005FE3C701B6010E94506120E030E048E423
:108E000052E40E94416320E030E040E85FE30E94CA
:108E10007B620E94DA6321E06C177D070CF420E08E
:108E2000822F90E0DF91CF91FF90EF90DF90CF9075
:108E300008950F931F93CF93DF93082F6EE274E092
:108E400088E892E10E948138C7E0D0E010E0B801E4
:108E50000C2E02C0759567950A94E2F7617077272A
:108E600042E050E088E892E10E946838219778F764
:108E7000DF91CF911F910F9108951F920F920FB61E
:108E80000F9211240BB60F922F933F934F935F9342
:108E90006F937F938F939F93AF93BF93EF93FF93C2
:108EA0008091B900887F803609F49CC068F58832CB
:108EB00009F45BC090F4803109F454C038F488237D
:108EC00009F4F6C0883009F44DC0F5C0883109F4C2
:108ED0004CC0803209F45DC0EEC0803409F468C033
:108EE00048F4803309F455C0883309F0E4C0809316
:108EF0008E10D8C0803509F44FC0883509F45DC0A4
:108F0000883409F0D8C0D6C0883909F4C7C0A8F49D
:108F1000883709F467C038F4883609F463C08037AD
:108F200009F460C0C8C0883809F4B8C0803909F4B1
:108F30005FC0803809F0BFC05BC0803B09F486C0C9
:108F400038F4803A09F466C0883A09F47FC0B3C0A7
:108F5000803C09F4A7C0883C09F4A4C0883B09F40C
:108F60008AC0A9C080916B1010C090918D10809123
:108F70008C10981770F5E0918D1081E08E0F809322
:108F80008D10F0E0E459FF4E80818093BB0085ECAA
:108F900086C080938E108EC0E0918D1081E08E0F80
:108FA00080938D108091BB00F0E0E459FF4E8083E8
:108FB00090918D1080918C106EC0E0918D1081E0A9
:108FC0008E0F80938D108091BB00F0E0E459FF4E2E
:108FD000808380918F1081116DC081E080936A1031
:108FE00084EA61C083E08093901010923F15CFCF48
:108FF00080913F15803208F051C0E0913F1581E02B
:109000008E0F80933F158091BB00F0E0E15EFA4E39
:109010008083BDCF85EC8093BC001092901080912E
:109020003F15803230F4E0913F15F0E0E15EFA4EFA
:10903000108260913F1570E0E0911D15F0911E15B2
:109040008FE195E1199510923F1535C084E080932A
:10905000901010921C1510921B15E0911915F091AB
:109060001A15199580911B15811105C081E0809317
:109070001B151092F914E0911C1581E08E0F80935E
:109080001C15F0E0E750FB4E80818093BB0090916F
:109090001C1580911B15981708F479CF85E88093EB
:1090A000BC0009C085EC8093BC001092901003C0F6
:1090B00010928E10A4DCFF91EF91BF91AF919F9120
:1090C0008F917F916F915F914F913F912F910F9071
:1090D0000BBE0F900FBE0F901F90189561E080EEB1
:1090E00094E1A4DD8BE39FE10197F1F70895EF92FE
:1090F000FF920F931F93CF938C01C62F7A0180E0CC
:109100000E94522D63E67FE080EE94E10E94813858
:109110006C2F80E00E94522DB80180EE94E10E94F5
:10912000B637B701FF0C880B990BCF911F910F91A8
:10913000FF90EF900C945D3A8F929F92AF92BF9206
:10914000CF92DF92EF92FF920F931F93CF93DF9313
:10915000CDB7DEB728970FB6F894DEBF0FBECDBFF0
:109160007C014A015B01690119821A821B821C82FF
:109170001D821E821F821886CB01BA010E94DA630B
:109180009B0177FF04C022273327261B370BB90129
:10919000330F880B990B0E94F1600E947C642EE8CB
:1091A0003DE543E150E40E9441630E94DA638B0194
:1091B0000F5F1F4F1016110614F001E010E00F5F53
:1091C0001F4FA8014C0D5D1D4930510514F048E0BA
:1091D00050E08E010F5F1F4F2C2DC501B4010E947E
:1091E000235CBC01C7010E949B37C70128960FB6BC
:1091F000F894DEBF0FBECDBFDF91CF911F910F91CD
:10920000FF90EF90DF90CF90BF90AF909F908F90A6
:1092100008954F925F926F927F928F929F92AF923A
:10922000BF92CF92DF92EF92FF920F931F93CF9353
:10923000DF93CDB7DEB76E970FB6F894DEBF0FBEE3
:10924000CDBF8C0165E97EE0CE010D960E949B3773
:109250000E945A3062E370E080E090E00E945D3A44
:109260000E945A3029833A834B835C836D837E83CB
:10927000C0903E14D0903F14E0904014F090411400
:1092800069817A81072E000C880B990B0E94F1608E
:10929000A70196010E9450614B015C016D817E81A6
:1092A000072E000C880B990B0E94F160A701960114
:1092B0000E9450612B013C016B817C81072E000CC8
:1092C000880B990B0E94F160A70196010E945061E2
:1092D00080924E1590924F15A0925015B092511554
:1092E00060935215709353158093541590935515B0
:1092F0004092561550925715609258157092591514
:109300009801215031092330310508F07CC1A501B5
:1093100094010E94EE6220914303309144034091F6
:109320004503509146030E947B626B017C0120E063
:1093300030E0A9010E94EB6087FD09C0C0924A1588
:10934000D0924B15E0924C15F0924D1510C02BEDBC
:109350003FE049EC50E4C701B6010E947B62609394
:109360004A1570934B1580934C1590934D15C090F2
:109370004A15D0904B15E0904C15F0904D152BED03
:109380003FE049EC50E4C701B6010E943064181672
:1093900084F42BED3FE049EC50E4C701B6010E9494
:1093A0007A6260934A1570934B1580934C15909395
:1093B0004D1520E030E044E353E460914A1570918C
:1093C0004B1580914C1590914D150E9450612BEDDD
:1093D0003FE049E450E40E94416360934615709376
:1093E000471580934815909349150E94DA634AE027
:1093F000CE0143960E94683764E77FE0CE01019674
:109400000E949B37BE016D5E7F4FCE0101960E9488
:1094100054366EE77FE00E943D36BC0185E194E161
:109420000E948E36CE0101960E94DC36CE01439614
:109430000E94DC36C0904615D0904715E090481544
:10944000F090491520E030E044EB52E4C701B6014A
:109450000E94EB60181664F0C701B6010E94DA633F
:109460004AE0CE0143960E94683765E87FE023C05A
:1094700020E030E044E353E4C701B6010E94EB6012
:1094800018163CF1A701960160E070E084E393E4D4
:109490000E947A6260934615709347158093481531
:1094A000909349150E94DA634AE0CE0143960E94E8
:1094B00068376BE87FE0CE0101960E949B37BE01C2
:1094C0006D5E7F4FCE0101960E94543668E87FE0C2
:1094D0004AC020E030E047E853E4C701B6010E94EB
:1094E000EB601816D4F020E030E044E353E4C70109
:1094F000B6010E947A626093461570934715809377
:109500004815909349150E94DA634AE0CE014396CC
:109510000E9468376BE87FE019C0A701960160E000
:1095200070E084EB93E40E947A6260934615709336
:10953000471580934815909349150E94DA634AE0D5
:10954000CE0143960E94683765E87FE0CE01019620
:109550000E949B37BE016D5E7F4FCE0101960E9437
:1095600054366EE87FE00E943D36BC01CE010D9678
:109570000E948E36CE0101960E94DC36CE014396C3
:109580000E94DC36ABDD60E080E00E94522D0E943C
:10959000953A28EE33E040E050E00E941D62BA01A7
:1095A000A9012AE0CE0101960E943C37BE016F5FFF
:1095B0007F4F89E094E10E94A336CE0101960E947C
:1095C000DC3661E175E089E094E10E94653669E08E
:1095D00074E1CE0101960E949337BE01635F7F4F15
:1095E000CE0101960E945436BC0180EE94E10E94A7
:1095F000B637CE0101960E94DC3664E170E080E06F
:1096000090E00E945D3AC8010297029708F0A1C15C
:109610000E94953AC090DE0FD090DF0FE090E00FEF
:10962000F090E10F6C197D098E099F090E94EF608F
:1096300020E030E04AE754E40E944163AB01BC0102
:1096400022E0CE0101960E94E136BE016F5F7F4F9E
:10965000CE0143960E94933761E175E0CE014396B7
:109660000E943D36BC0183E094E10E948E36CE011B
:1096700043960E94DC36CE0101960E94DC3663E000
:1096800074E1CE0101960E94933765E174E1CE0149
:1096900001960E945436BE01635F7F4F0E9454368C
:1096A000BC01CE010D960E948E36CE0101960E941D
:1096B000DC3661E97FE08FE094E10E9479364091E9
:1096C0004E1550914F15609150157091511521E034
:1096D000CE0101960E94E136BE016F5F7F4F8FE0A1
:1096E00094E10E947336CE0101960E94DC364091CF
:1096F000561550915715609158157091591521E0E4
:10970000CE0149960E94E136409152155091531571
:10971000609154157091551521E0CE0143960E9439
:10972000E13662E77FE0CE0101960E949B37BE01E1
:109730006D5E7F4FCE0101960E94543662E77FE056
:109740000E943D36BE01675E7F4F0E9454366CE931
:109750007FE00E943D36BC018FE094E10E947336A9
:10976000CE0101960E94DC36CE0143960E94DC3683
:10977000CE0149960E94DC3660914E1570914F15CE
:1097800080915015909151158090521590905315DD
:10979000A0905415B0905515C0905615D0905715FF
:1097A000E0905815F09059159B01AC010E94506152
:1097B0002B013C01A5019401C501B4010E94506137
:1097C0009B01AC01C301B2010E947B624B015C01B1
:1097D000A7019601C701B6010E9450619B01AC012F
:1097E000C501B4010E947B620E943F656B017C0150
:1097F00060934215709343158093441590934515DB
:1098000060EA7FE08FE094E10E94653620E030E07E
:109810004AE754E4C701B6010E94EB6087FF08C025
:1098200021E0B701A601CE0101960E94E1360BC0EE
:10983000C701B6010E94DA63AB01BC012AE0CE0188
:1098400001960E943C37BE016F5F7F4FCE01439669
:109850000E9493376DE97FE0CE0143960E943D362A
:10986000BC0185E194E10E948E36CE0143960E94B0
:10987000DC36CE0101960E94DC3620E030E64AE676
:1098800056E4609142157091431580914415909172
:1098900045150E94EB6087FF55C065E174E18FE0DC
:1098A00094E10E947336BE01635F7F4FCE01019643
:1098B0000E94933764E97EE0CE0101960E943D3616
:1098C0006FE074E10E945436BC018FE094E10E9485
:1098D0008E36CE0101960E94DC360330110571F4FC
:1098E0006FE074E1CE0101960E949337CE0101969C
:1098F0000E94F63DCE0101960E94DC3661E080E0D8
:109900000E94522D63E67FE080EE94E10E94813850
:1099100061E080E00E94522D64EA7FE0CE01019672
:109920000E949B3765E174E1CE0101960E94543696
:10993000BC0180EE94E10E94B637CE0101960E94F0
:10994000DC3607C0BE01635F7F4F8FE094E10E9469
:109950008E3668E270E080E090E00E945D3ACE01D1
:109960000D960E94DC366E960FB6F894DEBF0FBEE1
:10997000CDBFDF91CF911F910F91FF90EF90DF90BE
:10998000CF90BF90AF909F908F907F906F905F909F
:109990004F9008950F931F93CF93DF93C82FD62F27
:1099A00086E0C89FF0011124E859FB4E11A2878D73
:1099B00090A181309105F1F01CF4892B49F043C04E
:1099C00082309105A9F10397F1F560E070E034C0B1
:1099D0006623C9F161E070E08C2F0E94DF330E94A2
:1099E000953A6093C0147093C1148093C2149093FD
:1099F000C31429C00E94953A0091C0141091C1145B
:109A00002091C2143091C314AB01BC01401B510B17
:109A1000620B730B8091D2149091D314A0E0B0E04C
:109A200084179507A607B70718F462E070E004C032
:109A3000D11109C063E070E08C2FDF91CF911F91AD
:109A40000F910C94DF33DF91CF911F910F91089507
:109A50006F927F928F929F92AF92BF92CF92DF923E
:109A6000EF92FF920F931F93CF93DF9381E0809348
:109A7000D4140E94953A0091C4141091C5142091F9
:109A8000C6143091C714AB01BC01401B510B620BD3
:109A9000730B8091D0149091D114A0E0B0E08417A2
:109AA0009507A607B70708F00AC1C0E08091CE1459
:109AB000C81760F4E091CA14F091CB14EC0FF11DBB
:109AC00062E080810E94D439CF5FF0CF712C812C6D
:109AD000912C540183948091CF14781608F05FC0C4
:109AE000072D10E0E091CC14F091CD14E00FF11FA0
:109AF00061E080810E94D439E091CC14F091CD14C2
:109B0000E00FF11F60E080810E94A239D501C401FD
:109B1000072C04C0880F991FAA1FBB1F0A94D2F7F5
:109B20006C017C01E094F094612C8091CE14681655
:109B3000F8F4C62DD0E0E091CA14F091CB14EC0FEC
:109B4000FD1F80810E9478392496CC0FDD1FC859F3
:109B5000DB4E892B29F4888199818C299D2904C0A9
:109B6000888199818E219F21998388836394DDCF99
:109B7000E091CC14F091CD14E00FF11F61E08081F1
:109B80000E94A2398091CC149091CD14FC01E00F79
:109B9000F11F60E080810E94D43973949CCFE4E887
:109BA000F4E18FEF9FEF23813481232B21F4108286
:109BB000928381831582369624E1E03CF20799F77F
:109BC00010E096E0F92E8091CE14181708F051C0DD
:109BD00000E0C12FD0E0CC0FDD1FC059DB4E20913B
:109BE000CF14021708F043C068817981002E02C0AB
:109BF000769567950A94E2F761707727129F900136
:109C00001124200F311DE091C814F091C914E20F06
:109C1000F31F4081E8E6F4E180E0A58DB68DA21740
:109C2000B30711F461701AC08F5F36968A30A9F7B6
:109C3000672BD9F0E4E8F4E180E090E05081511125
:109C40000FC0F89EF001F99EF00D1124E859FB4E6B
:109C5000448F368F258F10A2178E61E09BDE05C0E2
:109C6000019636968A30910549F70F5FB8CF1F5F8E
:109C7000AACF80E090E0C0E0FC01E859FB4E21A1B2
:109C80002111C1E006968C339105B1F70E94953AF7
:109C90006093C4147093C5148093C6149093C71432
:109CA000CC2369F080918914882349F0809187142E
:109CB00090918814019719F48091841403C0109234
:109CC000D41480E0DF91CF911F910F91FF90EF901E
:109CD000DF90CF90BF90AF909F908F907F906F90CC
:109CE00008958F929F92AF92BF92CF92DF92EF92A0
:109CF000FF920F931F93CF93DF93DB01CD91DC9104
:109D0000DC011C96ED91FC911D97CE17DF070CF03E
:109D100047C0FE01EE0FFF1F1A968D919C911B9775
:109D2000E80FF91F80809180C170DD27B1E0CB275B
:109D3000209719F404E610E002C00CE91FEF790146
:109D40005A016B01020F131FB801C4012ED8892BD1
:109D500089F40E0D1F1DB801C40127D8892B69F4A1
:109D6000B8016E0D7F1DC40120D8892BE1F023E0DE
:109D700030E005C021E030E002C022E030E0F50133
:109D80008081918101968217930734F011821082AD
:109D9000F60180819181019691838083CE0105C077
:109DA00081E090E002C08FEF9FEFDF91CF911F9194
:109DB0000F91FF90EF90DF90CF90BF90AF909F906A
:109DC0008F900895CF93DF93EC01BC0188E892E176
:109DD0000E94B637BE018EE491E1DF91CF910C94E1
:109DE000B637CF92DF92EF92FF920F931F93CF93EC
:109DF000DF93CDB7DEB728970FB6F894DEBF0FBE5E
:109E0000CDBF823409F4B8C0D4F4803309F4D4C08F
:109E10007CF4833209F4C7C08A3209F0EDC069E1ED
:109E200074E081E294E10E9479368FEF9FEFE1C008
:109E3000813309F4D0C0813409F493C0DDC0813688
:109E400009F48FC034F4833409F4A1C0843449F098
:109E5000D3C0833609F49BC00CF48EC0843609F05D
:109E6000CBC08BE194E10E94053616161706180642
:109E700019067CF56DEA7FE088E892E10E9481385E
:109E80006BE174E188E892E10E9471388BE194E122
:109E90000E9405360AEF1FEF2FEF3FEF68017901AF
:109EA000C61AD70AE80AF90AB701A6012AE0CE01C4
:109EB00001960E943C37BE016F5F7F4F8BE194E1BA
:109EC0000E94A336CE0101960E94DC368BE194E11C
:109ED00044C0BEDD182FE12CF12C111111C08FEF01
:109EE000E81AF80A89EEE81683E0F80649F06EE110
:109EF00070E080E090E00E945D3AAADD182FEDCF7F
:109F00006AE270E0611B710917FD73954AE0CE01AA
:109F100001960E946837BE016F5F7F4F81E294E136
:109F20000E94A336CE0101960E94DC3661E274E104
:109F30008BE194E10E948E366DEA7FE088E892E141
:109F40000E948138612F88E892E10E94AF3788E84B
:109F500092E10E946E3881E294E10E940536CB01C5
:109F600048C060E174E081E294E10E94793680911A
:109F70002E1090912F103DC06DE074E081E294E1CD
:109F80000E947936109232108CEF9FEF32C063E15D
:109F900074E081E294E10E94793681E0809332108E
:109FA0008DEF9FEF26C066E174E081E294E10E94AC
:109FB00079368EEF9FEF1DC069E278E08BE194E186
:109FC0000E94793669E278E081E294E10E94793674
:109FD00080E090E00EC06AE174E08BE194E10E94C1
:109FE00079366AE174E081E294E10E94793681E099
:109FF00090E00E944B1E27C01A8219821C821B828D
:10A000001E821D828F831886BE01695F7F4FCE013D
:10A0100001960E947936BE016F5F7F4F8BE194E11C
:10A020000E94A336CE0101960E94DC368BE194E1BA
:10A030000E940536CB010E944B1E64E670E080E072
:10A0400090E00E945D3A28960FB6F894DEBF0FBEEE
:10A05000CDBFDF91CF911F910F91FF90EF90DF90D7
:10A06000CF9008958091091490910A14009711F0EF
:10A070000C94425C60E070E0CB010895CF93DF93D5
:10A08000CDB7DEB7A5970FB6F894DEBF0FBECDBF34
:10A09000789484B5826084BD84B5816084BD85B5C3
:10A0A000826085BD85B5816085BD80916E008160CF
:10A0B00080936E0010928100809181008260809375
:10A0C0008100809181008160809381008091800077
:10A0D0008160809380008091B10084608093B100A2
:10A0E0008091B00081608093B00080919100826087
:10A0F0008093910080919100816080939100809184
:10A1000090008160809390008091A1008260809394
:10A11000A1008091A10081608093A1008091A000A6
:10A1200081608093A0008091210182608093210151
:10A1300080912101816080932101809120018160C3
:10A140008093200180917A00846080937A008091CE
:10A150007A00826080937A0080917A008160809397
:10A160007A0080917A00806880937A001092C10012
:10A1700062E080EE94E10E946B4180EE94E10E94E7
:10A18000184662EB79E080EE94E10E94813888E81D
:10A1900092E10E943C448EE491E10E943C4460EDD7
:10A1A00077E080E090E00E945D3A88E892E10E94CA
:10A1B0005634782E83E7781609F46BC1109231106B
:10A1C0001092301014EBE12E10E1F12E00E010E0BF
:10A1D000C8010E940762D7018D937D010F5F1F4F59
:10A1E0000A341105A9F78091B4109091B510A0918F
:10A1F000B610B091B71085369105A105B1050CF4E4
:10A200003AC18093470390934803A0934903B093C6
:10A210004A038091B8109091B910A091BA10B091F2
:10A22000BB108093430390934403A0934503B093E2
:10A2300046038091BC109091BD10A091BE10B091CA
:10A24000BF1080933F0390934003A0934103B093CA
:10A25000420360ED70E1CE0101960E949B37BE0182
:10A260006F5F7F4F8AED94E10E94A336CE01019685
:10A270000E94DC368091C0109091C110A091C21054
:10A28000B091C31080934F0390935003A093510358
:10A29000B09352038091C4109091C510A091C61044
:10A2A000B091C71080934B0390934C03A0934D0340
:10A2B000B0934E038091C8109091C910A091CA101C
:10A2C000B091CB108093530390935403A093550304
:10A2D000B09356038091CC109091CD10A091CE10E8
:10A2E000B091CF108093570390935803A0935903D4
:10A2F000B0935A038091D8109091D910A091DA10A0
:10A30000B091DB108093980390939903A0939A03E4
:10A31000B0939B038091DC109091DD10A091DE1032
:10A32000B091DF108093940390939503A0939603CC
:10A33000B09397038091E0109091E110A091E2100A
:10A34000B091E3108093900390939103A0939203B4
:10A35000B09393038091E4109091E510A091E610E2
:10A36000B091E71080938C0390938D03A0938E039C
:10A37000B0938F038091E8109091E910A091EA10BA
:10A38000B091EB1080933B0390933C03A0933D036B
:10A39000B0933E034091230350912403A0902503E2
:10A3A000B0902603809027039090280360919C032F
:10A3B00070919D03009121031091220340901F038F
:10A3C00050902003ECEBF3E0AEEEEA2EA0E1FA2E83
:10A3D000BBE2CB2EB3E0DB2E21E030E080912903FD
:10A3E00090912A038217930774F1D7018D919D9163
:10A3F0007D01D6018D939D936D018430910519F4F3
:10A400008280938018C08A30910519F4A280B380AD
:10A4100012C08530910519F44281538110C08630F5
:10A42000910519F4628173810AC08730910519F48E
:10A430000281138104C00B9714F0428053802F5F78
:10A440003F4F3296CBCF10932203009321035092BB
:10A45000200340921F0370939D0360939C035093CD
:10A46000240340932303B0922603A09225039092E5
:10A470002803809227038091B4109091B510A09189
:10A48000B610B091B71085369105A105B1050CF055
:10A49000FEC08091470390914803A0914903B09179
:10A4A0004A038093B4109093B510A093B610B09364
:10A4B000B7108091430390914403A0914503B0915C
:10A4C00046038093B8109093B910A093BA10B0933C
:10A4D000BB1080913F0390914003A0914103B09144
:10A4E00042038093BC109093BD10A093BE10B09314
:10A4F000BF1080ED90E1892BE1F00091DE14109106
:10A50000DF140115110519F41092D01012C0073094
:10A51000110510F007E010E06091DA147091DB147F
:10A52000A80180ED90E10E944168F801E053FF4EE0
:10A53000108280914F0390915003A0915103B091EC
:10A5400052038093C0109093C110A093C210B09397
:10A55000C31080914B0390914C03A0914D03B09197
:10A560004E038093C4109093C510A093C610B0936F
:10A57000C7108091530390915403A0915503B0915B
:10A5800056038093C8109093C910A093CA10B0933B
:10A59000CB108091570390915803A0915903B0912B
:10A5A0005A038093CC109093CD10A093CE10B0930B
:10A5B000CF108091980390919903A0919A03B09144
:10A5C0009B038093D8109093D910A093DA10B09386
:10A5D000DB108091940390919503A0919603B09124
:10A5E00097038093DC109093DD10A093DE10B0935E
:10A5F000DF108091900390919103A0919203B0910C
:10A6000093038093E0109093E110A093E210B09335
:10A61000E31080918C0390918D03A0918E03B091F3
:10A620008F038093E4109093E510A093E610B0930D
:10A63000E71080913B0390913C03A0913D03B091C2
:10A640003E038093E8109093E910A093EA10B09332
:10A65000EB102091290330912A03A9E2B3E0ECEE3C
:10A66000F0E180E090E02817390734F04D915D91DA
:10A67000419351930196F7CFB3E77B1208C0109234
:10A6800031101092301080E090E00E9467446CE23C
:10A6900071E080E090E00E945D3A68EC70E080E05C
:10A6A00090E00E945D3A68EC70E080E090E00E94EB
:10A6B0005D3AF89482E08093B0008093B10094E614
:10A6C0009093B3001092B2008093700078948093BE
:10A6D0003113109234138091321360E00E94D43908
:10A6E0000E946E4860E080E00E94522D63EC79E0A9
:10A6F00080EE94E10E94813861E080E00E94522D5A
:10A700006AED74E1CE0101960E9493376DEE79E017
:10A71000CE0101960E943D36BC0180EE94E10E947C
:10A72000B637CE0101960E94DC368E01035F1F4FC3
:10A730006CE075E0C8010E949B376AED74E1C801C6
:10A740000E94543663ED79E00E943D36BC01CE0193
:10A7500001960E949337CE0101960E94F63DCE01EC
:10A7600001960E94DC36C8010E94DC3680913703D6
:10A77000909138030A97B1F48091390390913A038C
:10A780000A9781F48BEE91E10E943C448CED95E0B8
:10A79000A0E0B0E08093EF119093F011A093F1113D
:10A7A000B093F21168EE73E080E090E00E945D3AB1
:10A7B00085EF99E00E940C430E942C2D84E09AE0E2
:10A7C0000E940C4380E090E0A0E8BFE380933E1439
:10A7D00090933F14A0934014B093411461E17AE048
:10A7E00088E892E10E94813860913F0370914003B4
:10A7F000809141039091420341E00E944E2C8AE1F6
:10A800009AE00E940C4360913F0370914003809155
:10A810004103909142030E947B2B90932D108093D3
:10A820002C10892B21F08EEA95E00E940C438EE1DA
:10A830009AE00E940C4360E070E082E090E00E94A9
:10A84000662B80E090E090932D1080932C10892B44
:10A8500021F08EEA95E00E940C430E942C2D64E6C4
:10A8600070E080E090E00E945D3A83E20E94F5444F
:10A8700081E090E00E9463440E94984483E08093CA
:10A8800027140E942C2D80ED0E94592E853509F049
:10A8900074C58AEA0E94B22D9093291480932814DB
:10A8A0008CEA0E94B22D90932B1480932A148EEA86
:10A8B0000E94B22D90932D1480932C1480EB0E9453
:10A8C000B22D909339148093381482EB0E94B22DEC
:10A8D00090933B1480933A1484EB0E94B22D909392
:10A8E0003D1480933C1486EB0E94B22D90932F145C
:10A8F00080932E1488EB0E94B22D90933114809394
:10A9000030148AEB0E94B22D90933314809332144A
:10A910008CEB0E94B22D90933514809334148EEBFF
:10A920000E94B22D90933714809336140E94802E8B
:10A930000E94F1600E94DA630E94F16020E030E042
:10A9400048EC52E40E944163AB01BC0122E0CE011D
:10A9500001960E94E13660E37AE0C8010E949B37CD
:10A96000BE016F5F7F4FC8010E94543665E675E0F7
:10A970000E943D36BC018FE094E10E948E36C801F2
:10A980000E94DC36CE0101960E94DC366FE074E155
:10A9900088E892E10E947138609147037091480302
:10A9A0008091490390914A030E94F16020E030E0D9
:10A9B00048EC52E40E944163AB01BC0122E0CE01AD
:10A9C00001960E94E13664E47AE0C8010E949B3758
:10A9D000BE016F5F7F4FC8010E94543665E675E087
:10A9E0000E943D36BC018FE094E10E948E36C80182
:10A9F0000E94DC36CE0101960E94DC366FE074E1E5
:10AA000088E892E10E94713885E99EE00E940C433B
:10AA10000E942C2D60E08DE20E94183160E18DE2F1
:10AA20000E94183168E08DE20E941831409056145F
:10AA300050905714609058147090591449825A825B
:10AA40006B827C8280905A1490905B14A0905C146E
:10AA5000B0905D148D829E82AF82B886C0905E14E5
:10AA6000D0905F14E0906014F0906114C986DA868B
:10AA7000EB86FC868BE59AE00E940C43FE01319642
:10AA80001F01D1016D917D918D919D911D0146E038
:10AA90000E944E2C62E77FE088E892E10E948138B4
:10AAA0002016310671F785E99EE00E940C4323E9E8
:10AAB00038E144E85FE3C301B2010E9450612B0119
:10AAC0003C016D877E878F87988B22E430E645E8CE
:10AAD0005FE3C501B4010E9450614B015C01698BC9
:10AAE0007A8B8B8B9C8B25E83BEE41E95FE3C701BA
:10AAF000B6010E9450616D8B7E8B8F8B988F409238
:10AB000056145092571460925814709259148092AF
:10AB10005A1490925B14A0925C14B0925D146093EE
:10AB20005E1470935F14809360149093611489E6AF
:10AB30009AE00E940C438E01075E1F4FF101619164
:10AB40007191819191911F0142E00E944E2C62E728
:10AB50007FE088E892E10E9481382016310671F783
:10AB600085E99EE00E940C4342E654E166E070E015
:10AB700082E30E94B030C0906314D12CDC2CCC2432
:10AB800080916214C82AE0906514F12CFE2CEE240A
:10AB900080916414E82A0091671410E0102F0027B8
:10ABA00080916614082B66E77AE088E892E10E94BB
:10ABB00081384AE050E0B60188E892E10E946838A6
:10ABC00062E77FE088E892E10E9481384AE050E045
:10ABD000B70188E892E10E94683862E77FE088E880
:10ABE00092E10E9481384AE050E0B80188E892E1A1
:10ABF0000E94683885E99EE00E940C43C1010E94D2
:10AC00006A3163E87AE088E892E10E9481388E0137
:10AC10000B5D1F4FD1016D917D918D919D911D0116
:10AC20004AE00E944E2C62E77FE088E892E10E94B1
:10AC300081382016310671F785E99EE00E940C43A9
:10AC400061E08DE10E9418316CE87AE088E892E1D9
:10AC50000E948138A80161E070E08DE10E94B0306F
:10AC60008DA190E00E94EA3062E08EE10E941831EE
:10AC700063E08FE10E94183164E080E20E941831A5
:10AC800060EA7AE088E892E10E948138A80161E0F8
:10AC900070E08EE10E94B030ADA0B12CA80161E05F
:10ACA00070E08FE10E94B030CDA0D12CA80161E00E
:10ACB00070E080E20E94B030EDA0F12C4AE050E05C
:10ACC000B50188E892E10E94683862E77FE088E891
:10ACD00092E10E9481384AE050E0B60188E892E1B2
:10ACE0000E94683862E77FE088E892E10E9481383C
:10ACF0004AE050E0B70188E892E10E94683885E9AF
:10AD00009EE00E940C4365E081E20E9418316CEBEA
:10AD10007AE088E892E10E948138A80161E070E061
:10AD200081E20E94B0308DA190E00E94EA3066E09E
:10AD300082E20E9418316FEC7AE088E892E10E948A
:10AD40008138A80161E070E082E20E94B0308DA1FC
:10AD500090E00E94EA3067E083E20E94183167EEDB
:10AD60007AE088E892E10E948138A80161E070E011
:10AD700083E20E94B0308DA190E00E94EA3068E04A
:10AD800084E20E9418316DEF7AE088E892E10E9437
:10AD90008138A80161E070E084E20E94B0308DA1AA
:10ADA00090E00E94EA3069E085E20E94183165E196
:10ADB0007BE088E892E10E948138A80161E070E0C0
:10ADC00085E20E94B0308DA190E00E94EA306AE0F6
:10ADD00086E20E9418316FE27BE088E892E10E94EF
:10ADE0008138A80161E070E086E20E94B0308DA158
:10ADF00090E00E94EA306BE088E20E94183165E43E
:10AE00007BE088E892E10E948138A80161E070E06F
:10AE100088E20E94B0308DA190E00E94EA306CE0A0
:10AE200089E20E9418316EE57BE088E892E10E9499
:10AE30008138A80161E070E089E20E94B0308DA104
:10AE400090E00E94EA3066E77BE088E892E10E94A9
:10AE5000813866E070E087E20E94FE3090E00E9458
:10AE6000EA306DE87BE088E892E10E94813865E095
:10AE700070E087E20E94FE3090E00E94EA3064EACF
:10AE80007BE088E892E10E94813864E070E087E22C
:10AE90000E94FE3090E00E94EA306BEB7BE088E895
:10AEA00092E10E94813862E070E087E20E94FE3009
:10AEB00090E00E94EA3064ED7BE088E892E10E9435
:10AEC000813861E070E087E20E94FE3090E00E94ED
:10AED000EA306DEE7BE088E892E10E94813860E024
:10AEE00070E087E20E94FE3090E00E94EA3066E067
:10AEF0007CE088E892E10E94813863E070E087E2BC
:10AF00000E94FE3090E00E94EA3041E067E070E08D
:10AF100087E20E942D3141E063E070E087E20E9409
:10AF20002D3141E063E070E08AE20E942D3167E15B
:10AF30007CE088E892E10E94813863E070E08AE278
:10AF40000E94FE3090E00E94EA3040E063E070E052
:10AF50008AE20E942D3160E37CE088E892E10E9461
:10AF6000813863E070E08AE20E94FE3090E00E9447
:10AF7000EA3041E062E070E08AE20E942D316AE44A
:10AF80007CE088E892E10E94813862E070E08AE229
:10AF90000E94FE3090E00E94EA3040E062E070E003
:10AFA0008AE20E942D3166E67CE088E892E10E9408
:10AFB000813862E070E08AE20E94FE3090E00E94F8
:10AFC000EA3041E061E070E08AE20E942D3163E8FE
:10AFD0007CE088E892E10E94813861E070E08AE2DA
:10AFE0000E94FE3090E00E94EA3040E061E070E0B4
:10AFF0008AE20E942D316FE97CE088E892E10E94AC
:10B00000813861E070E08AE20E94FE3090E00E94A8
:10B01000EA3041E060E070E08AE20E942D316CEBA2
:10B020007CE088E892E10E94813860E070E08AE28A
:10B030000E94FE3090E00E94EA3040E060E070E064
:10B040008AE20E942D3168ED7CE088E892E10E945E
:10B05000813860E070E08AE20E94FE3090E00E9459
:10B06000EA3041E066E070E087E20E942D3141E085
:10B0700065E070E087E20E942D3141E064E070E01D
:10B0800087E20E942D3140E062E070E087E20E949A
:10B090002D3140E061E070E087E20E942D3140E018
:10B0A00060E070E087E20E942D3165EF7CE088E887
:10B0B00092E10E94813866E070E08BE20E94FE30EF
:10B0C00090E00E94EA306DE07DE088E892E10E9425
:10B0D000813865E070E08BE20E94FE3090E00E94D3
:10B0E000EA306BE27DE088E892E10E94813864E01A
:10B0F00070E08BE20E94FE3090E00E94EA3069E44A
:10B100007DE088E892E10E94813862E070E08BE2A5
:10B110000E94FE3090E00E94EA3062E67DE088E81E
:10B1200092E10E94813861E070E08BE20E94FE3083
:10B1300090E00E94EA306BE77DE088E892E10E94AF
:10B14000813860E070E08BE20E94FE3090E00E9467
:10B15000EA3064E97DE088E892E10E94813863E0AA
:10B1600070E08BE20E94FE3090E00E94EA3067EAD5
:10B170007DE088E892E10E94813864E070E08CE232
:10B180000E94FE3090E00E94EA3040E064E070E00F
:10B190008CE20E942D31A80161E070E08CE20E94F7
:10B1A000B0306DA1607F66608CE20E9418316CEB5C
:10B1B0007DE088E892E10E948138A80161E070E0BA
:10B1C0008CE20E94B0306DA16F7070E06650710922
:10B1D000072E000C880B990B0E94F1609B01AC01BB
:10B1E00060E070E080E090E40E94EF6420E030E0F6
:10B1F00048EC50E40E9450610E945D3160ED7DE0BA
:10B2000088E892E10E948138A80161E070E080E363
:10B210000E94B0304DA150E060E070E02AE088E884
:10B2200092E10E94D93788E892E10E946E3867EE79
:10B230007DE088E892E10E94813861E070E080E37F
:10B240000E94FE3090E00E94EA306FEF7DE088E8D7
:10B2500092E10E94813861E070E08FE20E94FE304E
:10B2600090E00E94EA3041E061E070E08FE20E94ED
:10B270002D3168E17EE088E892E10E94813861E04A
:10B2800070E08EE20E94FE3090E00E94EA3041E0E1
:10B2900061E070E08EE20E942D3140E067E070E0F6
:10B2A00081E30E942D3160E37EE088E892E10E9414
:10B2B000813867E070E081E30E94FE3090E00E94F8
:10B2C000EA3063E47EE088E892E10E948138A801D8
:10B2D00061E070E080E00E94B0308DA10E941947CB
:10B2E00085E99EE00E940C438DE1E82EF12C6AE492
:10B2F0007EE088E892E10E94813840E150E0B701A9
:10B3000088E892E10E9468386FE57DE088E892E184
:10B310000E948138A80161E070E08E2D0E94B0305B
:10B320008DA10E94194785E99EE00E940C43BFEF62
:10B33000EB1AFB0AEAE3EE16F104C9F668EE73E0D5
:10B3400080E090E00E945D3A6AE174E08BE194E174
:10B350000E94793681E090E090932F1080932E1018
:10B360000E948D3B60ED77E080E090E00E945D3AC6
:10B370000E944F020E942735FBCF6DE47EE0CE0194
:10B3800001960E949B37CE0101960E94F63DCE01A8
:10B3900001960E94DC3610921E03D0CF83E094E128
:10B3A0000E94DC3689E094E10E94DC368FE094E173
:10B3B0000E94DC3685E194E10E94DC368BE194E169
:10B3C0000E94DC3681E294E10E94DC368AED94E151
:10B3D0000C94DC368F929F92AF92BF92CF92DF9205
:10B3E000EF92FF92109251111092501188EE93E05B
:10B3F000A0E0B0E08093521190935311A0935411A8
:10B40000B093551122ED33E030934F1120934E113C
:10B4100045E351E050935B1140935A1144E351E0EE
:10B4200050935D1140935C1140E351E050935F11E4
:10B4300040935E1141E351E05093611140936011DC
:10B4400042E351E0509363114093621146E351E0AF
:10B450005093651140936411109267111092681116
:10B460001092691110926A111092EE111092ED1162
:10B470008093EF119093F011A093F111B093F2111A
:10B480003093EC112093EB1145ED50E05093F811FF
:10B490004093F71144ED50E05093FA114093F911A5
:10B4A00040ED50E05093FC114093FB1141ED50E012
:10B4B0005093FE114093FD1142ED50E05093001265
:10B4C0004093FF1146ED50E0509302124093011259
:10B4D0001092041210920512109206121092071286
:10B4E00010928B1210928A1280938C1290938D126C
:10B4F000A0938E12B0938F123093891220938812EA
:10B5000025EC30E0309395122093941224EC30E037
:10B51000309397122093961220EC30E030939912DA
:10B520002093981221EC30E030939B1220939A12D2
:10B5300022EC30E030939D1220939C1226EC30E0F8
:10B5400030939F1220939E121092A1121092A21279
:10B550001092A3121092A412109228131092271383
:10B560008093291390932A13A0932B13B0932C1339
:10B5700084EE93E090932613809325131092E314A6
:10B580001092E21480E094E09093E1148093E01430
:10B590008CE08093E4148FEF8093E5148BE080932C
:10B5A000E61485E08093E71484E08093E81483E058
:10B5B0008093E91482E08093EA141092EB141092C5
:10B5C000EC141092ED141092EE141092EF1461E04E
:10B5D00080EE94E10E946B416DE57FE08AED94E19D
:10B5E0000E949B3788E18093D71481E18093D8141F
:10B5F00080E18093D91461E088E10E94D43961E050
:10B600008091D7140E94A23960E08091D8140E94E2
:10B61000D43960E08091D9140E94D43961E08091DE
:10B62000D8140E94A23961E08091D9140E94A239F5
:10B6300061E08091D7140E94A23910926A1410928E
:10B640006E1410926D1410926F1486EF93E0909325
:10B6500069148093681480E090E0FC01E859FB4E87
:10B66000148E10A2178E11A206968C339105A9F79D
:10B6700082EA93E09093CB148093CA148EE993E00E
:10B680009093CD148093CC1484E08093CE14809357
:10B69000CF1486EA93E09093C9148093C8148AE08B
:10B6A00090E09093D1148093D01484EF91E0909324
:10B6B000D3148093D2141092D6141092D5141092F1
:10B6C000C4141092C5141092C6141092C71410928C
:10B6D000D41481E0809354141092551483EC9BEAA7
:10B6E000A6E7BBE38093561490935714A093581485
:10B6F000B093591488ED9BE6A6E7BBE380935A14F8
:10B7000090935B14A0935C14B0935D1482EF94EE5D
:10B71000A4E6BBE380935E1490935F14A09360143F
:10B72000B093611480919C0390919D039093531466
:10B73000809352148090980390909903A0909A035C
:10B74000B0909B0320919403309195034091960310
:10B7500050919703C501B401CDD66B017C01609374
:10B760004E1470934F148093501490935114609121
:10B770009003709191038091920390919303609351
:10B780004214709343148093441490934514809210
:10B79000461490924714A0924814B09249142091F4
:10B7A0008C0330918D0340918E0350918F03A2D66C
:10B7B0009B01AC01C701B60164D760934A14709332
:10B7C0004B1480934C1490934D1480E090E0A0E8CB
:10B7D000BFE380933E1490933F14A0934014B09322
:10B7E000411465E97EE081E294E10E949B3765E9BE
:10B7F0007EE08BE194E10E949B3765E97EE085E184
:10B8000094E10E949B3765E97EE08FE094E10E941D
:10B810009B3765E97EE089E094E10E949B3765E90A
:10B820007EE083E094E10E949B3787E080933213AF
:10B8300010923313FF90EF90DF90CF90BF90AF90B6
:10B840009F908F900895EF920F931F93CF93DF9364
:10B85000E80147FD02C034E001C034E1E42F440FA9
:10B86000FF0BF7FF03C0F195E195F109E32E022FDD
:10B870002E2FAE01B5D0CE01DF91CF911F910F9148
:10B88000EF9008956627772738C21F93FC01992708
:10B890008827BC01E89411911032E9F3193010F0B7
:10B8A0001E30C8F31B3249F01D3241F4689405C0C4
:10B8B0003ED0610F711D811D911D119110531A30E1
:10B8C000B8F33EF490958095709561957F4F8F4FBA
:10B8D0009F4F1F9108954532510518F4423008F0EA
:10B8E00004C0FB011082CB010895BB274A3031F41C
:10B8F000992322F4BDE2909581959F4F59C025323E
:10B90000310518F4223008F004C0FA011082CA018F
:10B910000895BB272A3051F4992342F4BDE2909553
:10B920008095709561957F4F8F4F9F4F20C0592F05
:10B93000482F372F262F660F771F881F991F660FF6
:10B94000771F881F991F620F731F841F951F660F33
:10B95000771F881F991F08952532310518F422306A
:10B9600008F004C0FA011082CA010895BB27FA0149
:10B97000A62F6217710581059105330B30FB66F028
:10B98000AA27660F771F881F991FAA1FA21710F0FA
:10B99000A21B63953850A9F7A05DAA3308F0A95DF2
:10B9A000A19336F7B111B1931082CA0104C4BB2729
:10B9B000FB015527AA27880F991FAA1FA41710F06B
:10B9C000A41B83955051B9F7A05DAA3308F0A95D77
:10B9D000A193009779F7B111B1931192CB01EBC309
:10B9E0004F925F926F927F929F92AF92BF92CF924F
:10B9F000DF92EF92FF920F931F93CF93DF93CDB718
:10BA0000DEB729970FB6F894DEBF0FBECDBF6A012F
:10BA1000122FB02E2BE3201720F0FF24F394F00E0A
:10BA200002C0BCE3FB2E0F2D27E0AE014F5F5F4F3E
:10BA3000CAD2AC018981982F9970913031F0E1FC24
:10BA400006C0E0FE06C090E205C09DE203C09BE296
:10BA500001C090E0EE2DE07183FF3CC0911102C067
:10BA600083E001C084E0811718F4212F281B01C056
:10BA700020E0E1110BC0F601822F30E2882319F09B
:10BA800031938150FBCFC20ED11C20E0992329F0C5
:10BA9000D6019C93F60131966F01C6010396E2FE32
:10BAA0000AC03EE4D6013C9341E411964C931197B1
:10BAB00012963C9306C03EE6F601308341E6418390
:10BAC0003283FC01322F40E2332309F442C0419318
:10BAD0003150FACF82FF44C0911102C083E001C00F
:10BAE00084E0811718F4212F281B01C020E0E11108
:10BAF0000BC0F601822F30E2882319F03193815078
:10BB0000FBCFC20ED11C20E0992329F0D6019C93D3
:10BB1000F60131966F01C6010396E2FE0BC039E4CF
:10BB2000D6013C933EE411963C93119736E412966D
:10BB30003C9307C039E6F60130833EE6318336E6B2
:10BB40003283FC01322F40E2332319F0419331500C
:10BB5000FBCFFC01E20FF11D10828EEF9FEFB7C00B
:10BB6000F1E0911101C0F0E06F2F70E0141615069E
:10BB700024F49A012F5F3F4F02C021E030E0260FEE
:10BB8000371FBB2029F06B2D70E06F5F7F4F02C025
:10BB900060E070E0260F371F612F70E0261737072F
:10BBA0001CF4121B212F01C020E03E2D387159F4E6
:10BBB000D601322F60E2332319F06D933150FBCF61
:10BBC000C20ED11C20E0FF2331F0D6019C93B601B8
:10BBD0006F5F7F4F6B01E1110BC0F601922F30E3D5
:10BBE000992319F031939150FBCFC20ED11C20E064
:10BBF0009F2D940F3A81782F7071A72E84FF03C078
:10BC0000313309F49150191624F4993018F098E062
:10BC100001C091E0E42F852F57FF02C0E0E080E0F3
:10BC20006E2F782FE0E0F0E0AEE29A2E3A01691A2A
:10BC300071082A01461A570A0B2D10E0119501953B
:10BC400011096F3F8FEF780729F4D6019C92C60146
:10BC500001966C014617570784F0661677066CF458
:10BC60007F01E40CF51CA1E0B0E0AC0FBD1FEA0EB3
:10BC7000FB1ED7011196BC9002C090E3B92E615013
:10BC800071093196C60101967C016017710724F095
:10BC9000D601BC926C01D5CF6417750741F43633D9
:10BCA00020F4353321F4A11002C081E3B82EF6014F
:10BCB000B082F701822F90E2882319F0919381508E
:10BCC000FBCFF701E20FF11D108280E090E0299692
:10BCD0000FB6F894DEBF0FBECDBFDF91CF911F919D
:10BCE0000F91FF90EF90DF90CF90BF90AF909F901B
:10BCF0007F906F905F904F9008956F927F928F9298
:10BD00009F92AF92BF92CF92DF92EF92FF920F93EA
:10BD10001F93CF93DF93EC017B016115710519F03F
:10BD2000DB018D939C938E010F5F1F4F7880872DD1
:10BD300090E021D2892B11F0E801F5CFBDE27B1212
:10BD400005C00F5F1F4F7980C1E008C0EBE27E1293
:10BD500004C08E010E5F1F4F7980C0E06801F1E0E2
:10BD6000CF1AD10843E050E068EE71E0C6010BD273
:10BD7000892BE9F4680122E0C20ED11C45E050E0B5
:10BD800063EE71E0C601FFD1892B21F4680187E0E1
:10BD9000C80ED11CE114F10419F0D701CD92DC9248
:10BDA000C111F9C060E070E080E89FE7FDC043E0AA
:10BDB00050E060EE71E0C601E6D1892B51F4E11448
:10BDC000F10409F4EDC00E5F1F4FF70111830083EA
:10BDD000E7C0680160E070E0CB0100E010E0F60130
:10BDE000D0EDD70DDA3050F52C2F2260622E2C2F9B
:10BDF0002870C2FF05C0211127C00F5F1F4F24C04C
:10BE0000222311F001501109A5E0B0E09B01AC0123
:10BE100030D34B015C01880C991CAA1CBB1CC501CA
:10BE2000B4016D0F711D811D911D6839A9E97A0753
:10BE30008A07A9E19A0740F0C66005C0DE3F51F4C9
:10BE4000C3FD44C0C8606C2EBFEFCB1ADB0A708004
:10BE5000C62DC5CF2D2F2F7D2531C1F540814D3207
:10BE600011F4C06106C04B3221F0319621E030E080
:10BE700006C03296D60111964C9122E030E0A0ED3A
:10BE8000A40FAA3018F0E21BF30B20C040E050E0F2
:10BE90004038BCE05B075CF49A01220F331F220F8D
:10BEA000331F420F531F440F551F4A0F511D319628
:10BEB000DF0111972C91A0EDA20FAA3048F3C4FF27
:10BEC00003C0519541955109040F151FC1FF07C0CB
:10BED000E114F10421F03197D701ED93FC937FD168
:10BEE000C370C33019F06B017C0106C06B017C018B
:10BEF000F7FAF094F7F8F09420E030E0A901C701D8
:10BF0000B60169D1882309F443C017FF06C0119513
:10BF100001951109CFEFD1E002C0C7E1D2E05E0187
:10BF2000B8E1AB1AB1084601BE2DAF2D90E2E92E63
:10BF3000F12C0E151F057CF0FE01259135914591E0
:10BF40005491B4018B2F9A2FABD14B01B82FA92F4D
:10BF50000E191F09EECF2497F594E794CA15DB0557
:10BF600041F76401EB2EFA2E8E2D880F8F2D881F3E
:10BF70008F3F41F020E030E0A901C701B6012BD18D
:10BF8000811106C082E290E090935B1580935A1570
:10BF9000C701B60109C060E070E080E89FEF04C00F
:10BFA00060E070E080EC9FE7DF91CF911F910F91EF
:10BFB000FF90EF90DF90CF90BF90AF909F908F90C9
:10BFC0007F906F900895283008F027E03327DA013A
:10BFD000990F311D87FD916000966105710539F457
:10BFE00032602E5F3D9330E32A95E1F708959F3F3D
:10BFF00030F080387105610509F03C5F3C5F3D938E
:10C00000913008F08068911DDF93CF931F930F93B9
:10C01000FF92EF92192F987F9695E92F9695969516
:10C02000E90FFF27EB58FD4F99273327EE24FF2414
:10C03000A701E70105900894079428F4360FE71E3E
:10C04000F81E491F511D660F771F881F991F069400
:10C05000A1F70590079428F4E70EF81E491F561F14
:10C06000C11D770F881F991F661F0694A1F70590C1
:10C07000079428F4F80E491F561FC71FD11D880FBB
:10C08000991F661F771F0694A1F70590079420F467
:10C09000490F561FC71FD81F990F661F771F881F8C
:10C0A0000694A9F784911095177041F0D695C7951D
:10C0B00057954795F794E7941A95C1F7EBE1F2E0AD
:10C0C00068941590159135916591959105907FE251
:10C0D0007395E118F10A430B560BC90BD009C0F751
:10C0E000E10CF11E431F561FC91FD01D7EF4703393
:10C0F00011F48A95E6CFE894015030F0080F0AF465
:10C100000027021708F4202F2395022F7A3328F0F6
:10C1100079E37D932A95E9F710C07D932A9589F6F6
:10C12000069497956795379517951794E118F10A36
:10C13000430B560BC90BD00998F023957E9173954C
:10C140007A3308F070E37C932013B8F77E91706126
:10C150007D9330F0839571E37D9370E32A95E1F749
:10C160001124EF90FF900F911F91CF91DF919927AC
:10C1700087FD909508959111F6C0803219F089508D
:10C180008550D0F70895FB01DC014150504088F004
:10C190008D9181341CF08B350CF4805E6591613497
:10C1A0001CF06B350CF4605E861B611171F3990B0A
:10C1B0000895881BFCCFDC01FC01672F7191772368
:10C1C000E1F7329704C07C916D9370836291AE1752
:10C1D000BF07C8F3089540D008F481E00895E894BB
:10C1E00009C097FB3EF490958095709561957F4FBF
:10C1F0008F4F9F4F9923A9F0F92F96E9BB2793956D
:10C20000F695879577956795B795F111F8CFFAF47C
:10C21000BB0F11F460FF1BC06F5F7F4F8F4F9F4FAD
:10C2200016C0882311F096E911C0772321F09EE80B
:10C23000872F762F05C0662371F096E8862F70E071
:10C2400060E02AF09A95660F771F881FDAF7880F4B
:10C250009695879597F90895990F0008550FAA0BA1
:10C26000E0E8FEEF16161706E807F907C0F0121609
:10C270001306E407F50798F0621B730B840B950B0C
:10C2800039F40A2661F0232B242B252B21F4089561
:10C290000A2609F4A140A6958FEF811D811D0895FE
:10C2A0000BD07BC06CD028F071D018F0952309F02A
:10C2B0005DC062C01124A5C081D0A0F3959FD1F3C9
:10C2C000950F50E0551F629FF001729FBB27F00D44
:10C2D000B11D639FAA27F00DB11DAA1F649F662799
:10C2E000B00DA11D661F829F2227B00DA11D621FE8
:10C2F000739FB00DA11D621F839FA00D611D221FA2
:10C30000749F3327A00D611D231F849F600D211D85
:10C31000822F762F6A2F11249F5750408AF0E1F028
:10C3200088234AF0EE0FFF1FBB1F661F771F881F71
:10C3300091505040A9F79E3F510570F017C061C061
:10C340005F3FECF3983EDCF3869577956795B7955C
:10C35000F795E7959F5FC1F7FE2B880F911D969586
:10C36000879597F9089599278827089597F99F67E2
:10C3700080E870E060E008959FEF80EC089500246D
:10C380000A941616170618060906089500240A943A
:10C3900012161306140605060895092E0394000CC0
:10C3A00011F4882352F0BB0F40F4BF2B11F460FF4F
:10C3B00004C06F5F7F4F8F4F9F4F089557FD905878
:10C3C000440F551F59F05F3F71F04795880F97FB59
:10C3D000991F61F09F3F79F0879508951216130613
:10C3E0001406551FF2CF4695F1DF08C01616170642
:10C3F0001806991FF1CF8695710561050894089577
:10C40000E894BB2766277727CB0197F90895F99918
:10C41000FECF92BD81BDF89A992780B50895262F49
:10C42000F999FECF1FBA92BD81BD20BD0FB6F89419
:10C43000FA9AF99A0FBE01960895052E97FB16F405
:10C4400000940FD057FD05D024D007FC02D046F44D
:10C4500008C050954095309521953F4F4F4F5F4F05
:10C46000089590958095709561957F4F8F4F9F4F60
:10C47000089531D0A59F900DB49F900DA49F800D7D
:10C48000911D11240895B7FFF4CFF3DF821B930BA6
:10C490000895A1E21A2EAA1BBB1BFD010DC0AA1F05
:10C4A000BB1FEE1FFF1FA217B307E407F50720F01D
:10C4B000A21BB30BE40BF50B661F771F881F991F98
:10C4C0001A9469F760957095809590959B01AC01E1
:10C4D000BD01CF010895A29FB001B39FC001A39FEA
:10C4E000700D811D1124911DB29F700D811D1124AD
:10C4F000911D08955058BB27AA270ED04ECF3FDF7D
:10C5000030F044DF20F031F49F3F11F41EF434CFBB
:10C510000EF4E095E7FB2ACFE92F50DF80F3BA173E
:10C52000620773078407950718F071F49EF568CFCA
:10C530000EF4E0950B2EBA2FA02D0B01B90190013E
:10C540000C01CA01A0011124FF27591B99F0593F82
:10C5500050F4503E68F11A16F040A22F232F342FCA
:10C560004427585FF3CF469537952795A795F04018
:10C570005395C9F77EF41F16BA0B620B730B840B2D
:10C58000BAF09150A1F0FF0FBB1F661F771F881FE5
:10C59000C2F70EC0BA0F621F731F841F48F487953D
:10C5A00077956795B795F7959E3F08F0B3CF93952C
:10C5B000880F08F09927EE0F979587950895DFDE8D
:10C5C00058F080E891E009F49EEFE0DE28F040E8C2
:10C5D00051E059F45EEF09C0CFCE12CFE92FE078D9
:10C5E000EDDE68F3092E052AC1F326173707480741
:10C5F000590738F00E2E07F8E02569F0E025E064D1
:10C600000AC0EF6307F8009407FADB01B9019D0146
:10C61000DC01CA01AD01EF9343D0BFDE0AD05F91C8
:10C62000552331F02BED3FE049E450FD49EC63CF59
:10C630000895DF93DD27B92FBF7740E85FE3161633
:10C64000170648075B0710F4D92F0ED19F938F93DD
:10C650007F936F9352D2E0E3F1E0DDD09EDE2F9125
:10C660003F914F915F9128DEDD2349F09058A2EA77
:10C670002AED3FE049EC5FE3D0785D274DDFDF91A5
:10C680008CCE0CD08ACE82DE40F079DE30F021F400
:10C690005F3F19F06BCE5111B4CE6ECE8FDE98F3A2
:10C6A0009923C9F35523B1F3951B550BBB27AA2733
:10C6B00062177307840738F09F5F5F4F220F331FA5
:10C6C000441FAA1FA9F333D00E2E3AF0E0E830D071
:10C6D00091505040E695001CCAF729D0FE2F27D074
:10C6E000660F771F881FBB1F261737074807AB0742
:10C6F000B0E809F0BB0B802DBF01FF2793585F4FB7
:10C700002AF09E3F510568F031CE7BCE5F3FECF3BF
:10C71000983EDCF3869577956795B795F7959F5F7B
:10C72000C9F7880F911D9695879597F90895E1E0CF
:10C73000660F771F881FBB1F621773078407BA072E
:10C7400020F0621B730B840BBA0BEE1F88F7E09589
:10C75000089519F40EF00ACE53CE0ECE37DEC8F38C
:10C760009638C0F707F80F92E8942BE33AEA48EBC3
:10C770005FE7A4DD0F920F920F924DB75EB70F9255
:10C78000FBD0EDE5F1E047D04F915F91EF91FF9144
:10C79000E595EE1FFF1F49F0FE57E0684427EE0FB6
:10C7A000441FFA95E1F74195550B67D00F9007FEAE
:10C7B0005BC0089504D06894B11123CE089506DEBD
:10C7C00088F09F5790F0B92F9927B751A0F0D1F07A
:10C7D000660F771F881F991F1AF0BA95C9F712C004
:10C7E000B13081F00DDEB1E008950ACE672F782FC9
:10C7F0008827B85F39F0B93FCCF386957795679570
:10C80000B395D9F73EF490958095709561957F4FDB
:10C810008F4F9F4F0895DF93CF931F930F93FF92F6
:10C82000EF92DF927B018C01689405C0DA2EEF0154
:10C8300043DDFE01E894A5912591359145915591EF
:10C84000AEF3EF0169DEFE019701A801DA9479F7F2
:10C85000DF90EF90FF900F911F91CF91DF9108959E
:10C86000FBDC08F48FEF08959B01AC0160E070E001
:10C8700080E89FE306CF7ACD47C1A8DDE8F399238E
:10C88000D9F3940F511DBBF39150504094F059F0DF
:10C89000882332F0660F771F881F91505040C1F7F0
:10C8A0009E3F510544F7880F911D9695879597F9FE
:10C8B00008955F3FACF0983E9CF0BB278695779536
:10C8C0006795B79508F4B1609395C1F7BB0F58F71A
:10C8D00011F460FFE8CF6F5F7F4F8F4F9F4FE3CF23
:10C8E00090CD0AD029ED3BE54EED5EE3D9CC0EF0BC
:10C8F0000BC142CD68943ACD69DDC8F39923D1F3D9
:10C90000C6F3DF93CF931F930F93FF92C92FDD27B9
:10C9100088232AF02197660F771F881FDAF720E017
:10C9200030E040E85FEB9FE3883920F0803E30F054
:10C9300021968F77E0DDE5E8F1E003C0DCDDE2EB96
:10C94000F1E069DF8B01BE01EC01FB2E6F5771092D
:10C950007595771F880B990B44DC28E132E741E39A
:10C960005FE3AADCAF2D9801AE01FF900F911F91FC
:10C97000CF91DF91D1DD11CDFA01DC01AA0FBB1FF0
:10C980009B01AC01BF5728F4222733274427507856
:10C990001FC0B75188F4AB2F0024469537952795D3
:10C9A000011CA395D2F3002069F0220F331F441F0E
:10C9B000B395DAF30DD09ECD61307105A0E88A07FA
:10C9C000B94630F49B01AC01662777278827907819
:10C9D000309621F020833183428353830895FA01F6
:10C9E000EE0FFF1F30962105310599F16115710594
:10C9F00061F48038BFE39B0749F168949038810562
:10CA000061F08038BFEF9B0741F0992342F5FF3F6B
:10CA1000E1053105210511F1E8940894E795D90164
:10CA2000AA2329F4AB2FBE2FF85FD0F310C0FF5F0D
:10CA300070F4A695E0F7F73950F019F0FF3A38F4A2
:10CA40009F779F930CD00F9007FC905808953EF06D
:10CA500093CC60E070E080E89FE308954FE79F7714
:10CA60005F934F933F932F9347DF2F913F914F91C8
:10CA70005F9116DC73CE11F40EF47ECC45C0A6DCBB
:10CA8000D0F39923D9F3CEF39F57550B87FF4AD0A4
:10CA90000024A0E640EA900180585695979528F426
:10CAA000805C660F771F881F20F02617370748071E
:10CAB00030F4621B730B840B202931294A2BA69575
:10CAC00017940794202531254A2758F7660F771FBA
:10CAD000881F20F026173707480730F4620B730BC6
:10CAE000840B200D311D411DA09581F7B901842FC4
:10CAF0009158880F9695879508959B01AC01D0CBEE
:10CB0000ABDB880B990B08959F3F31F0915020F4D7
:10CB1000879577956795B795880F911D9695879519
:10CB200097F9089591505040660F771F881FD2F7EC
:10CB30000895DB018F939F939CDCBF91AF91A29FDF
:10CB4000800D911DA39F900DB29F900D112408950B
:10CB500097FB072E16F4009406D077FD08D04AD034
:10CB600007FC05D03EF4909581959F4F08957095F0
:10CB700061957F4F0895EE0FFF1F881F8BBF0790B1
:10CB8000F691E02D19940F93083090F0982F872F8D
:10CB9000762F652F542F432F322F22270850F4CFA2
:10CBA000220F331F441F551F661F771F881F991FB1
:10CBB0000A95B2F70F91089597FB10F816940008A4
:10CBC0000F93083098F00850232F342F452F562FFD
:10CBD000672F782F892F902DF4CF059497958795FF
:10CBE0007795679557954795379527950A95AAF7AD
:10CBF0000F910895AA1BBB1B51E107C0AA1FBB1FC1
:10CC0000A617B70710F0A61BB70B881F991F5A95D8
:10CC1000A9F780959095BC01CD010895CF93DF933E
:10CC20008230910510F482E090E0E0915E15F09181
:10CC30005F1520E030E0C0E0D0E0309711F1408196
:10CC4000518148175907C0F04817590761F482818C
:10CC50009381209719F09B838A832BC090935F1553
:10CC600080935E1526C02115310519F04217530730
:10CC700018F49A01BE01DF01EF010280F381E02D7B
:10CC8000DCCF2115310509F1281B390B2430310582
:10CC900090F412968D919C9113976115710521F076
:10CCA000FB019383828304C090935F1580935E158C
:10CCB000FD01329644C0FD01E20FF31F8193919371
:10CCC000225031092D933C933AC020915C1530914C
:10CCD0005D15232B41F42091B8033091B9033093B3
:10CCE0005D1520935C152091B6033091B703211593
:10CCF000310541F42DB73EB74091BA035091BB03C3
:10CD0000241B350BE0915C15F0915D15E217F307DC
:10CD1000A0F42E1B3F0B2817390778F0AC014E5FAB
:10CD20005F4F2417350748F04E0F5F1F50935D1576
:10CD300040935C158193919302C0E0E0F0E0CF0155
:10CD4000DF91CF9108950F931F93CF93DF930097B7
:10CD500009F48CC0FC0132971382128200915E1597
:10CD600010915F150115110581F420813181820F29
:10CD7000931F20915C1530915D152817390779F5BF
:10CD8000F0935D15E0935C1571C0D80140E050E070
:10CD9000AE17BF0750F412962D913C911397AD0139
:10CDA0002115310509F1D901F3CF9D01DA01338352
:10CDB000228360817181860F971F8217930769F420
:10CDC000EC0128813981260F371F2E5F3F4F3183B9
:10CDD00020838A819B8193838283452B29F4F0935E
:10CDE0005F15E0935E1542C01396FC93EE93129785
:10CDF000ED01499159919E01240F351FE217F30768
:10CE000071F480819181840F951F029611969C93F5
:10CE10008E938281938113969C938E931297E0E078
:10CE2000F0E0D80112968D919C911397009719F01C
:10CE3000F8018C01F6CF8D919C9198012E5F3F4FA8
:10CE4000820F931F20915C1530915D1528173907CB
:10CE500069F4309729F410925F1510925E1502C0A4
:10CE60001382128210935D1500935C15DF91CF91B0
:10CE70001F910F9108956F927F928F929F92AF9220
:10CE8000BF92CF92DF92EF92FF920F931F93CF93B7
:10CE9000DF93EC01009781F4CB01DF91CF911F91DB
:10CEA0000F91FF90EF90DF90CF90BF90AF909F9049
:10CEB0008F907F906F90B2CEFC01E60FF71F9C0120
:10CEC00022503109E217F30708F4A8C0D9010D91E7
:10CED0001C91119706171707A8F00530110508F4E3
:10CEE0009BC0C80104978617970708F495C00250A5
:10CEF0001109061B170B019311936D937C93CF01BE
:10CF000022DF8AC05B01A01AB10A4C01800E911E7B
:10CF1000A0915E15B0915F1540E050E0E12CF12C3E
:10CF2000109709F44AC0A815B905D1F56D907C9009
:10CF30001197630182E0C80ED11CCA14DB0480F192
:10CF4000A3014A195B096A0182E0C80ED11C12963E
:10CF5000BC9012971396AC91B5E0CB16D10440F07B
:10CF6000B282A38351834083D9016D937C930AC01D
:10CF70000E5F1F4FC301800F911FF90191838083C2
:10CF8000EB2DFA2FE114F10431F0D7011396FC9345
:10CF9000EE93129741C0F0935F15E0935E153CC08D
:10CFA0008D919C9111974817590708F4AC017D01A8
:10CFB00012960D90BC91A02DB3CF80915C159091ED
:10CFC0005D1588159905E1F446175707C8F4809157
:10CFD000B6039091B703009741F48DB79EB7409187
:10CFE000BA035091BB03841B950BE817F907B0F403
:10CFF000F0935D15E0935C15F901718360830CC0BB
:10D00000CB010CDE7C01009749F0A801BE011BD0CA
:10D01000CE0199DEC70104C0CE0102C080E090E0DD
:10D02000DF91CF911F910F91FF90EF90DF90CF9004
:10D03000BF90AF909F908F907F906F90089581E008
:10D0400090E0F89447C0FB01DC0102C001900D9212
:10D0500041505040D8F70895FB01DC0101900D923A
:10D060000020E1F70895FB01DC014150504030F011
:10D070008D910190801919F40020B9F7881B990B44
:10D080000895FB01DC014150504048F001900D92A1
:10D090000020C9F701C01D9241505040E0F70895AB
:10D0A000FB0151915523A9F0BF01DC014D914517BA
:10D0B0004111E1F759F4CD010190002049F04D9163
:10D0C00040154111C9F3FB014111EFCF81E090E020
:10D0D0000197089512E0CCE1D2E000E005C0802F76
:10D0E000FE0149DD2196011DCD31D10780E0080701
:06D0F000B1F7F894FFCF38
:10D0F6000000F0410AD7C3BF9A99F93F00002041CA
:10D10600756E646566696E65640000000000005413
:10D11600656D702B48756D000000000000004952D7
:10D1260020466C616D6500000000000000476173D9
:10D13600000000000000000000000000547572624C
:10D1460069646974790000000000007048000000FE
:10D1560000000000000000000000434F3200000005
:10D166000000000000000000004F32000000000038
:10D17600000000000000000049522054656D700058
:10D186000000000000000049522054656D70000048
:10D19600000000000000504D0000000000000000EC
:10D1A60000000000004348340000000000000000BA
:10D1B60000000000416C636F686F6C0000000000A7
:10D1C600000000434F0000000000000000000000C7
:10D1D60000004832000000000000000000000000CF
:10D1E600004F7A6F6E65000000000000000000002E
:10D1F6004832530000000000000000000000004E0E
:10D206004833000000000000000000000000013963
:10D21600003D003F0008003E000800010002000338
:10D2260000050004000600080009000000A8416689
:10D2360066A63FA167333D7C8C010000803B45001C
:10D2460000803F0AD78B40CDCC2C400162BE3C39D2
:10D2560093522A409352AA4017D900418C96814195
:10D26600B73AC9418B899D3E0000A041000020428B
:10D2760000007042133BF142ECC43A430000804088
:10D2860027882640643B5F3E21B0B23E3D002E30EB
:10D2960032342F3133353132334134353642373833
:10D2A60039432A3023440000601580000800370007
:10D2B600380039003F003E003D001100100000001C
:10D2C6000000C034033447340635783456346A34A3
:10D2D600000000008C455D45BB453145554541453F
:10D2E600324500000000103AD139A0390000000094
:10D2F60011460334BB45BA4507002D37002D3400CF
:10D306002D35002D33002D32002D310073657269E5
:10D31600616C3A200042543A20005300410042001A
:10D32600736574005345540023506172616D6574D2
:10D3360065727300235365612D6C6576656C2050AC
:10D34600726573737572653D00234D61676E657412
:10D356006963206465636C696E6174696F6E2041F0
:10D366006E676C653D0023436F6D70617373205368
:10D3760063616C653D0023547572626964697479F2
:10D3860020766F6C74616765733A005640004E54A0
:10D39600552C20004E5455200023426C7565746F41
:10D3A6006F7468204E616D653D0023434F32207ACD
:10D3B60065726F20766F6C74616765280070706D9A
:10D3C600293D0056200023434F32206D6178207698
:10D3D6006F6C746167652028002343616C69627213
:10D3E60061746564204F3220636F6E63203D0020B8
:10D3F600766F6C25200023736C6F74202300292020
:10D40600697320002354696D6520696E74657276B0
:10D41600616C3D002354696D6520647572617469A1
:10D426006F6E3D00476976656E20736561206C6599
:10D4360076656C20503D00506120697320756E6CD6
:10D44600696B656C792100536561206C6576656C46
:10D4560020503D002068506100736C6F743D00538E
:10D466004C4F543D0042543D0062743D0041542BE4
:10D476004E414D450043533D0063733D00234572C5
:10D48600726F7220746F20736574206E65772063E7
:10D496006F6D70617373207363616C653D00456EDB
:10D4A6007465726564207363616C652077617320AF
:10D4B6006E6F742076616C69642C2076616C696489
:10D4C6002067617573732076616C75657320617270
:10D4D600653A20302E38382C20312E332C20312E30
:10D4E600392C20322E352C20342E302C20342E3759
:10D4F6002C20352E362C20382E310023436F6E74A7
:10D50600696E756F7573204D6F6465204572726F15
:10D516007220746F20736574206E657720636F6D5B
:10D5260070617373207363616C653D00234E65778C
:10D5360020636F6D70617373207363616C653D006A
:10D5460050494E3D0070696E3D0041542B50494E86
:10D5560000706800704800504800706834007048D9
:10D566003400566F6C746167652870483D34293AFB
:10D576000070683130007048313000566F6C74614D
:10D5860067652870483D3130293A0074696D6569D0
:10D596003D0074696D65643D00544231007462312A
:10D5A60000547572626964697479204C6F7765728C
:10D5B600204C696D69742056313A20002354422864
:10D5C6005631293D004F3243414C006F3263616C46
:10D5D600004F322063616C6962726174696F6E3AE2
:10D5E6002000234F3220766F6C253D00434F325A80
:10D5F60000636F327A00434F32207A65726F20766D
:10D606006F6C7420280070706D293A200023434FF8
:10D616003220566F3D005600434F324D00636F3245
:10D626006D00434F32204D415820766F6C74202890
:10D636000023434F3220566D3D0054424900746228
:10D646006900547572626964697479204C6F7765F4
:10D6560072204C696D69742056696E663A20002303
:10D6660054422856696E66293D0054424C00746245
:10D676006C00547572626964697479204C6F7765C1
:10D6860072204C696D69743A200020766F6C746163
:10D6960067653D002354422856293D0054425500F3
:10D6A6007462750054757262696469747920557084
:10D6B600706572204C696D69743A20006B65793D1E
:10D6C60000616E6F7468657220495220696E7075CC
:10D6D600743D007265706C6965733D0073204F324E
:10D6E60020436F6E6300566F6C25007320434F32E4
:10D6F60020436F6E6300434F323D0070706D004DE6
:10D706006561737572696E6720504D322E35002043
:10D71600504D313A322E353A313000504D28312EA7
:10D72600302C322E352C3130293D00206E672F4C9F
:10D736000042543A00313A54656D702048756D695F
:10D746006469747900323A54656D7020507265735D
:10D756007375726500323A616E6420486569676860
:10D766007400333A4C6967687420496E742E00342D
:10D776003A495220466C616D6500353A476173201F
:10D786004C6576656C00363A4D61676E6574696303
:10D79600206669656C6400373A49522054656D709D
:10D7A60000383A70482076616C756500393A496EE2
:10D7B600636C2E20616E672E00393A6F72203344F7
:10D7C60020616363656C2E0044313A547572626958
:10D7D600646974790044323A504D28313A322E3514
:10D7E6003A3130290044333A434F3220636F6E6337
:10D7F6002E0044343A4F3220636F6E632E002A3A6D
:10D80600546869732048656C7000233A53686F77D3
:10D81600204C4344006F4320413D006F43202000CD
:10D826004C6967687420496E74656E736974790013
:10D836007320202000206C78004C3D00206C78205E
:10D84600004C6576656C3D00495220466C616D65FD
:10D856002000476173206C6576656C3D00536561F9
:10D8660072636820446972656374696F6E00482D3F
:10D876006669656C64007320200049522046616920
:10D886006C65640049522054656D703D006F43001D
:10D8960070483D004E6F2070482073656E736F723E
:10D8A600210057656C636F6D6520746F2045645564
:10D8B600484B00456455484B205345534C6F6767AA
:10D8C600657200206D6F62696C65206C6F676765B5
:10D8D60072207374617274656420616E642072656F
:10D8E600616479210049324320696E74657266610C
:10D8F60063652E006E657720484D43353838334CC6
:10D90600007363616C65203D2000204761006D6FE8
:10D91600646520746F20636F6E74696E6F75730033
:10D9260023536561206C6576656C20502863616CB5
:10D9360063293D002343616C6962726174696F6E8D
:10D946002050726573737572653D006761696E7309
:10D956005F6F7269675B5D3A007365742067616922
:10D966006E735B5D3A0058595A20434F554E5453D7
:10D976003A200058595A2047733A20006765745474
:10D9860061705468726573686F6C6428293A200068
:10D99600676574417869734F66667365742826787F
:10D9A6002C2026792C20267A293A20006765745483
:10D9B60061704475726174696F6E28293A20006738
:10D9C6006574446F75626C655461704C6174656E04
:10D9D600637928293A2000676574446F75626C651F
:10D9E60054617057696E646F7728292000676574E3
:10D9F60041637469766974795468726573686F6C8B
:10DA06006428292000676574496E616374697669C4
:10DA160074795468726573686F6C6428292000678E
:10DA2600657454696D65496E616374697669747964
:10DA360028293A20006765744672656546616C6CF4
:10DA46005468726573686F6C6428293A20006765AC
:10DA5600744672656546616C6C4475726174696F73
:10DA66006E28293A2000697341637469766974796E
:10DA760058456E61626C656428293A2000697341D5
:10DA86006374697669747959456E61626C65642858
:10DA9600293A2000697341637469766974795A4535
:10DAA6006E61626C656428293A20006973496E616B
:10DAB6006374697669747958456E61626C65642829
:10DAC600293A20006973496E6163746976697479CD
:10DAD60059456E61626C656428293A20006973496C
:10DAE6006E61637469766974795A456E61626C65B4
:10DAF6006428293A200069734163746976697479E8
:10DB0600416328293A200067657453757070726501
:10DB1600737342697428293B20747275653F20002F
:10DB260067657453757070726573734269742829DA
:10DB36003B2066616C73653F2000697354617044D5
:10DB46006574656374696F6E4F6E5828293B20743F
:10DB56007275653F2000697354617044657465632E
:10DB660074696F6E4F6E5828293B2066616C736529
:10DB76003F20006973546170446574656374696F0E
:10DB86006E4F6E5928293B20747275653F200069D7
:10DB960073546170446574656374696F6E4F6E5932
:10DBA60028293B2066616C73653F200069735461C8
:10DBB60070446574656374696F6E4F6E5A28293BAD
:10DBC60020747275653F20006973546170446574F2
:10DBD600656374696F6E4F6E5A28293B2066616CC7
:10DBE60073653F200069734163746976697479537C
:10DBF6006F757263654F6E5828293A20006163631A
:10DC0600656C2E69734163746976697479536F75AF
:10DC16007263654F6E5928293A2000616363656C0B
:10DC26002E69734163746976697479536F7572638B
:10DC3600654F6E5A28293A2000616363656C2E6928
:10DC460073546170536F757263654F6E5828293A25
:10DC56002000616363656C2E6973546170536F7540
:10DC66007263654F6E5928293A2000616363656CBB
:10DC76002E6973546170536F757263654F6E5A28BF
:10DC8600293A2000616363656C2E697341736C6584
:10DC9600657028293A2000616363656C2E69734CB0
:10DCA6006F77506F77657228293A2000676574523E
:10DCB60061746528293A20332E31343135393F00D5
:10DCC600676574496E74657272757074536F757298
:10DCD600636528293A2000676574496E7465727217
:10DCE600757074536F757263652831293A20006721
:10DCF6006574496E746572727570744D6170706981
:10DD06006E672831293A20006973496E746572720C
:10DD1600757074456E61626C65642831293A20001D
:10DD260067657453656C6654657374426974282913
:10DD36003A2000307830303A20003078002345729F
:10DD4600726F723A707265737375726520424D50C8
:10DD56003038352C20636865636B20776972696E8D
:10DD66006721006E616E00696E66006F76660073ED
:10DD7600205475726269646974790054423D004E9C
:10DD86005455000D0A0054656D702048756D696420
:10DD9600697479202020007320202020006F432002
:10DDA600483D004320002520200049742773207633
:10DDB60065727920686F7421200049742773207179
:10DDC6007569746520686F742100497320616972F2
:10DDD6002D636F6E64206F6E3F0054656D70206911
:10DDE600732066696E6521202000497427732074AC
:10DDF6006F6F20636F6F6C2120004F66662061692C
:10DE0600722D636F6E64212020006128782C792C96
:10DE16007A292F673A20007320613D002067004968
:10DE26006E636C2E20616E672E28782079207A2901
:10DE36002F6465673A20007320496E636C2E20417B
:10DE46006E672E007320617A3D00672000534553AC
:10DE560032310020202020202020202020202020B9
:10DE660020202000436F6D706173733A2000286490
:10DE760065672920004E20002045005320002057CA
:10DE860000482D6669656C643A202800296D4700B4
:10DE9600203D3E00482D6669656C643D006B6579E2
:04DEA600323D000009
:020000023000CC
:10E000000D9489F10D94B2F10D94B2F10D94B2F129
:10E010000D94B2F10D94B2F10D94B2F10D94B2F1F0
:10E020000D94B2F10D94B2F10D94B2F10D94B2F1E0
:10E030000D94B2F10D94B2F10D94B2F10D94B2F1D0
:10E040000D94B2F10D94B2F10D94B2F10D94B2F1C0
:10E050000D94B2F10D94B2F10D94B2F10D94B2F1B0
:10E060000D94B2F10D94B2F10D94B2F10D94B2F1A0
:10E070000D94B2F10D94B2F10D94B2F10D94B2F190
:10E080000D94B2F10D94B2F10D94B2F10D94B2F180
:10E090000D94B2F10D94B2F10D94B2F10D94B2F170
:10E0A0000D94B2F10D94B2F10D94B2F10D94B2F160
:10E0B0000D94B2F10D94B2F10D94B2F10D94B2F150
:10E0C0000D94B2F10D94B2F10D94B2F10D94B2F140
:10E0D0000D94B2F10D94B2F10D94B2F10D94B2F130
:10E0E0000D94B2F141546D656761323536300041AF
:10E0F000726475696E6F206578706C6F72657220DE
:10E1000073746B3530305632206279204D4C530099
:10E11000426F6F746C6F616465723E004875683F52
:10E1200000436F6D70696C6564206F6E203D200048
:10E130004350552054797065202020203D20005FF9
:10E140005F4156525F415243485F5F3D2000415658
:10E1500052204C696243205665723D20004743437C
:10E160002056657273696F6E203D20004350552024
:10E1700049442020202020203D20004C6F7720663D
:10E18000757365202020203D20004869676820665F
:10E190007573652020203D200045787420667573D6
:10E1A00065202020203D20004C6F636B2066757336
:10E1B000652020203D20004D617220203720323024
:10E1C000313300312E362E3800342E332E350056A2
:10E1D00023202020414444522020206F7020636F70
:10E1E00064652020202020696E73747275637469E1
:10E1F0006F6E2061646472202020496E74657272B3
:10E20000757074006E6F20766563746F7200726A49
:10E210006D702020006A6D70200057686174207056
:10E220006F72743A00506F7274206E6F7420737541
:10E2300070706F72746564004D7573742062652030
:10E2400061206C6574746572002000577269747483
:10E25000696E672045450052656164696E672045B7
:10E26000450045452065727220636E743D00504F35
:10E27000525400303D5A65726F2061646472003FF1
:10E280003D43505520737461747300403D454550C3
:10E29000524F4D207465737400423D426C696E6B41
:10E2A000204C454400453D44756D70204545505215
:10E2B0004F4D00463D44756D7020464C415348001B
:10E2C000483D48656C70004C3D4C69737420492F83
:10E2D0004F20506F72747300513D51756974005234
:10E2E0003D44756D702052414D00563D73686F7707
:10E2F00020696E7465727275707420566563746FF0
:10E30000727300593D506F727420626C696E6B00BD
:10E310002A0011241FBECFEFD1E2DEBFCDBF01E046
:10E320000CBF12E0A0E0B2E0EEE1FDEF03E00BBFB6
:10E3300002C007900D92A030B107D9F712E0A0E01B
:10E34000B2E001C01D92AE30B107E1F70F9460F367
:10E350000D948DFE01E20EBF0FEF0DBF11241FBE05
:10E360000D9460F30D9400F020E030E040ED57E0B4
:10E3700005C0FA013197F1F72F5F3F4F2817390792
:10E38000C0F308959C01260F311DC901A0E0B0E043
:10E390002F5F3F4FABBFFC018791882361F08093D3
:10E3A000C6008091C00086FFFCCF8091C0008064D1
:10E3B0008093C000EACF08958DE08093C6008091DD
:10E3C000C00086FFFCCF8091C00080648093C000B5
:10E3D0008AE08093C6008091C00086FFFCCF8091C8
:10E3E000C00080648093C00008950F94C2F10F9420
:10E3F000DCF10895FC019081992359F09093C600B7
:10E400008091C00086FFFCCF8091C0008064809323
:10E41000C0003196992379F70895282F982F929567
:10E420009F70892F805D8A3308F0895F8093C600D2
:10E430008091C00086FFFCCF8091C00080648093F3
:10E44000C000822F8F70982F905D9A3308F0995FEB
:10E450009093C6008091C00086FFFCCF8091C000E1
:10E4600080648093C00008959C01FB01853691056E
:10E470001CF46330710594F0C90164E670E00F94F8
:10E480002EFE605D7F4F6093C6008091C00086FFC6
:10E49000FCCF8091C00080648093C0002B30310598
:10E4A00014F43297B4F0C90164E670E00F942EFEC4
:10E4B0006AE070E00F942EFE605D7F4F6093C600AF
:10E4C0008091C00086FFFCCF8091C0008064809363
:10E4D000C000C9016AE070E00F942EFEC0968093E0
:10E4E000C6008091C00086FFFCCF8091C000806490
:10E4F0008093C00008951F93182F8EE692EE60E07F
:10E500000F94C2F11093C6008091C00086FFFCCF2B
:10E510008091C00080648093C0000F94DCF11F9153
:10E5200008952F923F924F925F926F927F928F92B7
:10E530009F92AF92BF92CF92DF92EF92FF920F9392
:10E540001F93DF93CF93CDB7DEB762970FB6F894E2
:10E55000DEBF0FBECDBF382E622ECA01DB015C01CB
:10E560006D01772420E2222E2E010894411C511CBB
:10E570008BC081E0A81680E0B80681E0C80680E084
:10E58000D80628F0C601AA27BB270F940DF2BB2797
:10E59000AD2D9C2D8B2D0F940DF28A2D0F940DF225
:10E5A0002092C6008091C00086FFFCCF8091C00001
:10E5B00080648093C0009DE29093C6008091C0006B
:10E5C00086FFFCCF8091C00080648093C0002092C1
:10E5D000C6008091C00086FFFCCF8091C00080649F
:10E5E0008093C00019828601750188249924A1E0D6
:10E5F0003A1651F03A1620F0B2E03B1661F409C029
:10E600000BBFF701779007C0C7010F9477FE782EF4
:10E6100002C0F7017080872D0F940DF22092C60082
:10E620008091C00086FFFCCF8091C0008064809301
:10E63000C000872D8052F401EF70F0708F3520F408
:10E64000E40DF51D708204C0E40DF51D8EE280839B
:10E650000894E11CF11C011D111D0894811C911CE2
:10E6600090E18916910409F0C2CF80E190E0A0E02A
:10E67000B0E0A80EB91ECA1EDB1E198AC2010F9493
:10E68000FAF10F94DCF16A94662009F072CF629679
:10E690000FB6F894DEBF0FBECDBFCF91DF911F91B3
:10E6A0000F91FF90EF90DF90CF90BF90AF909F9031
:10E6B0008F907F906F905F904F903F902F90089534
:10E6C0002F923F924F925F926F927F928F929F9282
:10E6D000AF92BF92CF92DF92EF92FF920F931F9370
:10E6E000DF93CF93CDB7DEB7CD53D1400FB6F894BB
:10E6F000DEBF0FBECDBF01E20EBF0FEF0DBF94B75F
:10E70000F894A89514BE80916000886180936000A1
:10E7100010926000789493FF05C0E0910002F091A0
:10E7200001021995279A2F9A8091C00082608093E8
:10E73000C00080E18093C40088E18093C1000000A4
:10E74000EE24FF24870144E0A42EB12CCC24DD2448
:10E7500024C0C5010197F1F70894E11CF11C011DCB
:10E76000111D21E2E2162EE4F20620E0020720E06D
:10E77000120718F031E0C32ED12CC801B70127ECE5
:10E780003BE140E050E00F9441FE611571058105C9
:10E79000910519F485B1805885B98091C00087FD35
:10E7A00003C0C114D104A9F2A6014F5F5F4FC25E3E
:10E7B000DE4F59834883CE51D140C25EDE4F8881FF
:10E7C0009981CE51D140019711F00D9410FEC05D9A
:10E7D000DE4F19821882C053D14060E0C15DDE4F28
:10E7E0001882CF52D14088249924C35DDE4F19820C
:10E7F0001882CD52D140C05EDE4F188219821A8233
:10E800001B82C052D140CE5CDE4F188219821A8220
:10E810001B82C253D140EE24FF2487010BBFF701B6
:10E8200007911691C45CDE4F19830883CC53D14005
:10E830000D940BFEC25EDE4F28813981CE51D1404E
:10E840002130310509F52091C600C25EDE4F1982E4
:10E850001882CE51D14022C02F5F3F4F4F4F5F4FA4
:10E86000213082E138078AE7480780E0580780F0C6
:10E87000C45CDE4FE881F981CC53D140EF5FFF4F9C
:10E8800019F0EE27FF27099420E030E040E050E047
:10E890008091C00087FFE0CF2091C600C35DDE4FAE
:10E8A00048815981CD52D1404F5F5F4FC35DDE4FEC
:10E8B00059834883CD52D140213209F063C64A3092
:10E8C000510508F05FC60894811C911C53E0851621
:10E8D000910409F059C600E010E018C081E280936D
:10E8E000C6008091C00086FFFCCF8091C00080648C
:10E8F0008093C0002F5F3F4F2931310579F70F9486
:10E90000DCF10F5F1F4F0530110519F020E030E0FA
:10E91000E5CF10920A0210920B0210920C02109294
:10E920000D02109206021092070210920802109235
:10E930000902109202021092030210920402109235
:10E9400005028FEE90EE60E00F94F5F180E191EE1C
:10E9500060E00F94C2F18091C00087FFFCCF9091DE
:10E96000C600903608F09F759032B8F09093C600BC
:10E970008091C00086FFFCCF8091C00080648093AE
:10E98000C000A0E2A093C6008091C00086FFFCCF2B
:10E990008091C00080648093C000983409F4D7C18E
:10E9A0009934B8F4923409F459C1933458F490333B
:10E9B00019F1903308F4E3C59F33A1F1903409F0C5
:10E9C000DEC5BDC0953409F470C1963409F0D7C5D1
:10E9D00098C1923509F42BC2933538F49C3409F46C
:10E9E000F5C1913509F0CBC518C2963509F445C279
:10E9F000993509F0C4C567C483E792EE62E00F94CD
:10EA0000F5F110920602109207021092080210927D
:10EA1000090210920A0210920B0210920C0210923C
:10EA20000D0213C18FE792EE62E00F94F5F18FEEC5
:10EA300090EE60E00F94F5F181E291EE60E00F94CA
:10EA4000C2F187EB91EE60E00F94F5F180E391EE77
:10EA500060E00F94C2F184EE90EE60E00F94F5F167
:10EA60008FE391EE60E00F94C2F186E090E061E008
:10EA700070E00F9434F20F94DCF18DE591EE60E0DC
:10EA80000F94C2F189EC91EE60E00F94F5F18EE401
:10EA900091EE60E00F94C2F183EC91EE60E00F9490
:10EAA000F5F18CE691EE60E00F94C2F18EE10F94E7
:10EAB0000DF288E90F940DF281E00F940DF20F949E
:10EAC000DCF18BE791EE60E00F94C2F119E0E0E039
:10EAD000F0E010935700E4918E2F0F940DF20F94F5
:10EAE000DCF18AE891EE60E00F94C2F1E3E0F0E03F
:10EAF00010935700E4918E2F0F940DF20F94DCF1D8
:10EB000089E991EE60E00F94C2F1E2E0F0E0109349
:10EB10005700E4918E2F0F940DF20F94DCF188EAE8
:10EB200091EE60E00F94C2F1E1E0F0E01093570045
:10EB30001491812F0F940DF20F94DCF107CF8BE825
:10EB400092EE62E00F94F5F18BE492EE60E00F94A8
:10EB5000F5F10F94DCF100E010E019C0C8016F2D51
:10EB60000F947FFEFF2031F489E492EE60E00F9471
:10EB7000C2F10BC0F092C6008091C00086FFFCCFAE
:10EB80008091C00080648093C0000F5F1F4FC80158
:10EB900081519F41A0E0B0E0ABBFFC01F790BAE229
:10EBA000FB1621F0E2E000301E07C1F60F94DCF105
:10EBB0000F94DCF187E592EE60E00F94F5F10F948D
:10EBC000DCF1CC24DD2400E010E01EC0C8010F946D
:10EBD00077FEF82E882331F489E492EE60E00F94FA
:10EBE000C2F10BC08093C6008091C00086FFFCCFAD
:10EBF0008091C00080648093C000FE1419F00894D6
:10EC0000C11CD11C0F5F1F4FC80181519F41A0E063
:10EC1000B0E0ABBFFC01E790FAE2EF1621F022E092
:10EC20000030120799F60F94DCF10F94DCF182E6C4
:10EC300092EE60E00F94C2F1C60161E070E00F94C3
:10EC400034F20F94DCF10F94DCF110920202109276
:10EC50000302109204021092050278CE89E992EE26
:10EC600062E00F94F5F1279A2F9A16C02F9880E052
:10EC700090E0E0EDF7E03197F1F7019684369105E9
:10EC8000C1F72F9A80E090E0E0EDF7E03197F1F7DF
:10EC9000019684369105C1F78091C00087FFE6CFC9
:10ECA0008091C00087FFFCCF64C485EA92EE62E0E9
:10ECB0000F94F5F140910202509103026091040219
:10ECC0007091050281E020E10F9491F2809102029F
:10ECD00090910302A0910402B091050280509F4FD1
:10ECE000AF4FBF4F8093020290930302A0930402A0
:10ECF000B093050280509041A040B04008F426CE69
:10ED0000A4CF83EB92EE62E00F94F5F140910602FE
:10ED100050910702609108027091090280E020E1A1
:10ED20000F9491F28091060290910702A09108023F
:10ED3000B091090280509F4FAF4FBF4F80930602A2
:10ED400090930702A0930802B0930902FFCD80ECD4
:10ED500092EE62E00F94F5F183E792EE60E00F949B
:10ED6000F5F18FE792EE60E00F94F5F18BE892EE0B
:10ED700060E00F94F5F189E992EE60E00F94F5F10F
:10ED800085EA92EE60E00F94F5F183EB92EE60E09D
:10ED90000F94F5F180EC92EE60E00F94F5F187ECC2
:10EDA00092EE60E00F94F5F188ED92EE60E00F9442
:10EDB000F5F18FED92EE60E00F94F5F18AEE92EEB0
:10EDC00060E00F94F5F183E093EEBDCD87EC92EE19
:10EDD00062E00F94F5F181E40F947BF282E40F94EA
:10EDE0007BF283E40F947BF284E40F947BF285E45E
:10EDF0000F947BF286E40F947BF287E40F947BF20E
:10EE000088E40F947BF28AE40F947BF28BE40F94F6
:10EE10007BF28CE40F947BF299CD88ED92EE62E068
:10EE20000F94F5F1772473948824992409C48FED05
:10EE300092EE62E00F94F5F140910A0250910B02BC
:10EE400060910C0270910D0282E020E10F9491F22A
:10EE500080910A0290910B02A0910C02B0910D02D8
:10EE600080509F4FAF4FBF4F80930A0290930B0289
:10EE7000A0930C02B0930D0269CD8AEE92EE62E08F
:10EE80000F94F5F184EE90EE60E00F94F5F18FECC5
:10EE900091EE60E00F94F5F1662477244301CC5D98
:10EEA000DE4F19821882C452D140D401C301B695F5
:10EEB000A79597958795CA5DDE4F88839983AA8326
:10EEC000BB83C652D140CC5DDE4FA881B981C4520C
:10EED000D1401196CC5DDE4FB983A883C452D14096
:10EEE000CD0162E070E00F9434F2B0E2B093C6005E
:10EEF0008091C00086FFFCCF8091C0008064809329
:10EF0000C000EDE2E093C6008091C00086FFFCCF18
:10EF10008091C00080648093C000F0E2F093C6004E
:10EF20008091C00086FFFCCF8091C00080648093F8
:10EF3000C000CA5DDE4FE880F9800A811B81C6529D
:10EF4000D140BB27A12F902F8F2D0F940DF2CA5DBA
:10EF5000DE4F8881C652D1400F940DF2B0E2FB2EF5
:10EF6000F092C6008091C00086FFFCCF8091C00067
:10EF700080648093C0000DE30093C6008091C000C0
:10EF800086FFFCCF8091C00080648093C00010E2B7
:10EF90001093C6008091C00086FFFCCF8091C00016
:10EFA00080648093C0008BBEF3012791C65DDE4F65
:10EFB0002883CA52D140A22EBB24CC24DD2408943D
:10EFC000611C711C811C911C8BBEF3018791282E42
:10EFD0003324442455240894611C711C811C911C09
:10EFE0008BBEF3013791C55DDE4F3883CB52D140E4
:10EFF0000894611C711C811C911C8BBEF30147910C
:10F00000C45DDE4F4883CC52D140ADEFEA2EAFEF66
:10F01000FA2EAFEF0A2FAFEF1A2F6E0C7F1C801E57
:10F02000911E142D032DF22CEE24EA0CFB1C0C1D5A
:10F030001D1D0F940DF220E22093C6008091C000A8
:10F0400086FFFCCF8091C00080648093C000C65DC5
:10F05000DE4F8881CA52D1400F940DF230E23093D6
:10F06000C6008091C00086FFFCCF8091C000806404
:10F070008093C000C45DDE4F8881CC52D1400F9494
:10F080000DF240E24093C6008091C00086FFFCCFA5
:10F090008091C00080648093C000C55DDE4F888190
:10F0A000CB52D1400F940DF250E25093C6008091A4
:10F0B000C00086FFFCCF8091C00080648093C000B8
:10F0C0008FEFE8168FEFF80680E0080780E018075A
:10F0D00031F484E092EE60E00F94C2F1DFC0D80119
:10F0E000C7018070907CA070B0708050904CA040A0
:10F0F000B040D1F52FEF3FE340E050E0E222F322B1
:10F1000004231523CA5DDE4FA880B980CA80DB8046
:10F11000C652D140AE0CBF1CC01ED11EAA0CBB1CD7
:10F12000CC1CDD1C8EE092EE60E00F94C2F1BB2798
:10F13000A12F902F8F2D0F940DF28E2D0F940DF285
:10F1400030E23093C6008091C00086FFFCCF8091F2
:10F15000C00080648093C0004EE34093C60080915D
:10F16000C00086FFFCCF87C08EE09EEFA0E0B0E03D
:10F17000E822F9220A231B239CE0E91694E9F90608
:10F1800090E0090790E0190709F088C0C45DDE4FE0
:10F19000A881CC52D140EA2EFF2400E010E0102FCD
:10F1A0000F2DFE2CEE24C55DDE4FB881CB52D14031
:10F1B000EB0EF11C011D111DD601C501817090706F
:10F1C000A070B070DC0199278827E80EF91E0A1F8D
:10F1D0001B1F20EF30E040E050E0A222B322C42207
:10F1E000D52241E1AA0CBB1CCC1CDD1C4A95D1F7F1
:10F1F000EA0CFB1C0C1D1D1D81E090E0A0E0B0E0BE
:10F20000282239224A225B2235E1220C331C441C7D
:10F21000551C3A95D1F7E20CF31C041D151D57013E
:10F220006801AA0CBB1CCC1CDD1C85E192EE60E0E1
:10F230000F94C2F1C801AA27BB270F940DF2BB2778
:10F24000A12F902F8F2D0F940DF28E2D0F940DF274
:10F2500090E29093C6008091C00086FFFCCF809121
:10F26000C00080648093C000AEE3A093C60080918C
:10F27000C00086FFFCCF8091C00080648093C000F6
:10F28000C601AA27BB270F940DF2BB27AD2D9C2DDD
:10F290008B2D0F940DF28A2D0F940DF20F94DCF14B
:10F2A000CC5DDE4FE881F981C452D140F99709F471
:10F2B0004DCBF4E0EF2EF12C012D112D6E0C7F1CA7
:10F2C000801E911EF2CD83E093EE62E00F94F5F183
:10F2D0008AE192EE60E00F94C2F18091C00087FF56
:10F2E000FCCF1091C6001F751093C6008091C0001E
:10F2F00086FFFCCF8091C00080648093C0000F9493
:10F30000DCF1812F81548A3108F036C1163409F4BA
:10F3100095C0173490F4133409F44EC0143430F40B
:10F320001134F1F0123409F01DC130C0143409F465
:10F3300059C0153409F016C16BC01A3409F4C4C0A1
:10F340001B3438F4173409F48FC0183409F00AC19B
:10F35000A1C01B3409F4D2C01C3409F003C1E8C0B9
:10F360008FEF81B90DC082B1809582B980E090E0C5
:10F37000E0EDF7E03197F1F70196883C9105C1F790
:10F380008091C00087FFEFCF12B8EFC08FEF84B934
:10F390000DC085B1809585B980E090E0E0EDF7E0A3
:10F3A0003197F1F70196883C9105C1F78091C00033
:10F3B00087FFEFCF15B8D9C08FEF87B90DC088B1DF
:10F3C000809588B980E090E0E0EDF7E03197F1F7C3
:10F3D0000196883C9105C1F78091C00087FFEFCF6F
:10F3E00018B8C3C08FEF8AB90DC08BB180958BB9A7
:10F3F00080E090E0E0EDF7E03197F1F70196883C8E
:10F400009105C1F78091C00087FFEFCF1BB8ADC059
:10F410008FEF8DB90DC08EB180958EB980E090E0F0
:10F42000E0EDF7E03197F1F70196883C9105C1F7DF
:10F430008091C00087FFEFCF1EB897C08FEF80BBD1
:10F440000DC081B3809581BB80E090E0E0EDF7E0F6
:10F450003197F1F70196883C9105C1F78091C00082
:10F4600087FFEFCF11BA81C08FEF83BB0DC084B38C
:10F47000809584BB80E090E0E0EDF7E03197F1F714
:10F480000196883C9105C1F78091C00087FFEFCFBE
:10F4900014BA6BC08FEF809301010FC080910201FD
:10F4A00080958093020180E090E0E0EDF7E03197F5
:10F4B000F1F70196883C9105C1F78091C00087FF64
:10F4C000EDCF1092020151C08FEF809304010FC065
:10F4D0008091050180958093050180E090E0E0ED4A
:10F4E000F7E03197F1F70196883C9105C1F78091DB
:10F4F000C00087FFEDCF1092050137C08FEF8093DA
:10F5000007010FC08091080180958093080180E079
:10F5100090E0E0EDF7E03197F1F70196883C910536
:10F52000C1F78091C00087FFEDCF109208011DC088
:10F530008FEF80930A010FC080910B01809580931B
:10F540000B0180E090E0E0EDF7E03197F1F70196F4
:10F55000883C9105C1F78091C00087FFEDCF1092E4
:10F560000B0103C085E292EEEEC98091C00087FFD7
:10F57000FCCF8091C600EAC988E392EEE4C98CE131
:10F5800091EEE1C988249924933011F1943028F444
:10F59000913089F09230B8F408C0953061F195301F
:10F5A000F0F0963009F048C043C02B3109F042C951
:10F5B00091E06BE13FC96227C15DDE4F2883CF52E6
:10F5C000D14092E037C9B22FA0E0622793E032C960
:10F5D000822F90E0A82BB92B622794E02BC92E3004
:10F5E00009F039C3622795E0C05DDE4F19821882A9
:10F5F000C053D1401FC9E1E0F0E0EC0FFD1FC05D3A
:10F60000DE4F08811981C053D140E00FF11F2083E4
:10F610000F5F1F4FC05DDE4F19830883C053D14079
:10F6200062270A171B0709F005C9D80196E002C92D
:10F63000261709F010C303C0973009F0FBC87724E0
:10F640009981933109F412C19431C8F4963009F4C8
:10F65000D8C0973050F4923009F406C1933009F4C1
:10F660006DC0913009F059C253C0913109F477C08F
:10F67000923108F0BBC0903109F04FC2F5C098310B
:10F6800009F487C0993150F4953109F4EFC09531F0
:10F6900008F4C6C1963109F040C2C2C19A3109F4DA
:10F6A0006CC09A3108F491C09B3109F45BC09D3164
:10F6B00009F033C29D81903359F48F81882311F46E
:10F6C0009EE11CC0813011F091E018C098E916C08D
:10F6D000892F807591F0903539F4E0E0F0E089E011
:10F6E0008093570094910AC0983539F4E3E0F0E034
:10F6F00089E080935700949101C090E01A821B82A8
:10F700008D818C831D829E831F8227E030E009C299
:10F710001A8288E08B8381E48C8386E58D8382E581
:10F720008E8389E48F8383E5888780E589878FE5E9
:10F730008A8782E38B872BE030E0F3C18A818139AD
:10F7400041F0823941F0803911F48FE005C080E04A
:10F7500003C082E001C08AE01A828B8344C0772410
:10F76000739482C08D81882311F48EE12CC0813086
:10F7700011F081E028C088E926C01A82E1E0F0E0BB
:10F7800089E08093570084918B831C8224E030E0D1
:10F79000C8C18B81803589F48C81883039F4E2E0EE
:10F7A000F0E089E08093570084910DC0E0E0F0E044
:10F7B00089E080935700849106C0E3E0F0E089E09F
:10F7C0008093570084911A82DFCF8D81836C99E0FA
:10F7D000E1E0F0E0082E90935700E89507B600FCB2
:10F7E000FDCF1A821B8223E030E09BC180EC8A832C
:10F7F000CE5CDE4F188219821A821B82C253D1401E
:10F800008EC18A8190E0A0E0B0E0582F44273327D2
:10F8100022278B8190E0A0E0B0E0DC0199278827C7
:10F82000282B392B4A2B5B2B8D8190E0A0E0B0E098
:10F83000282B392B4A2B5B2B8C8190E0A0E0B0E089
:10F84000BA2FA92F982F8827282B392B4A2B5B2BCF
:10F85000220F331F441F551FC05EDE4F288339839C
:10F860004A835B83C052D1401A8259C13A81C95C34
:10F87000DE4F3883C753D140CA5CDE4F1882C6536F
:10F88000D1408B81C82EDD24CA5CDE4F488159816E
:10F89000C653D140C42AD52A933109F082C0CE5C28
:10F8A000DE4F88819981AA81BB81C253D1408050AB
:10F8B000904CA340B04030F583E0CE5CDE4FE88052
:10F8C000F9800A811B81C253D140F70100935B008C
:10F8D00080935700E89507B600FCFDCFCE5CDE4F65
:10F8E000088119812A813B81C253D14000501F4FAA
:10F8F0002F4F3F4FCE5CDE4F088319832A833B8313
:10F90000C253D140C05EDE4F488159816A817B81FC
:10F91000C052D140DE011B9631E08C9111962C91A2
:10F9200011971296C75CDE4F2883C953D140C85C3B
:10F93000DE4F1882C853D14090E0C85CDE4FE881AA
:10F94000F981C853D1408E2B9F2B0C01FA01609393
:10F950005B0030935700E89511244E5F5F4F6F4F67
:10F960007F4F0EEFE02E0FEFF02ECE0CDF1CC114F8
:10F97000D10499F685E0C05EDE4F088119812A81A5
:10F980003B81C052D140F80120935B008093570027
:10F99000E89507B600FCFDCF81E180935700E8951C
:10F9A00035C0C05EDE4F88819981AA81BB81C0527B
:10F9B000D140B695A795979587957C018601ABE0D8
:10F9C000AA2EB12CAC0EBD1E0BC0D5016D915D01F0
:10F9D000C7010F947FFE0894E11CF11C01501040F8
:10F9E0000115110591F7A60160E070E0440F551F65
:10F9F000661F771FC05EDE4FE880F9800A811B8199
:10FA0000C052D1404E0D5F1D601F711F1A82C05E33
:10FA1000DE4F488359836A837B83C052D1407FC0C5
:10FA2000FA80C55CDE4FF882CB53D140C65CDE4F16
:10FA30001882CA53D1408B81C82EDD24C65CDE4FAC
:10FA400008811981CA53D140C02AD12A1A828981DA
:10FA5000BE016D5F7F4F843121F59601C05EDE4FA0
:10FA6000E880F9800A811B81C052D1400BBFF701A9
:10FA700087919691DB018C9311969C936E5F7F4FDB
:10FA8000D801C7010296A11DB11DC05EDE4F88835B
:10FA90009983AA83BB83C052D14022503040F1F6F3
:10FAA00036C0C05EDE4F288139814A815B81C052F9
:10FAB000D1400894C108D108760100E010E0089414
:10FAC000C11CD11C0894E11CF11C011D111DE20E8A
:10FAD000F31E041F151F21BDBB27A52F942F832FB5
:10FAE00082BD2F5F3F4F4F4F5F4FF89A80B5DB01CC
:10FAF0008D93BD012E153F054007510761F7C05E8C
:10FB0000DE4F288339834A835B83C052D1409601FC
:10FB10002D5F3F4FFB01108204C080EC8A8322E0FE
:10FB200030E08BE18093C6008091C00086FFFCCF5F
:10FB30008091C00080648093C000C15DDE4FF88179
:10FB4000CF52D140F093C6008091C00086FFFCCF19
:10FB50008091C00080648093C000432F3093C60022
:10FB60008091C00086FFFCCF8091C00080648093AC
:10FB7000C000922F2093C6008091C00086FFFCCF6A
:10FB80008091C00080648093C0008EE08093C600A6
:10FB90008091C00086FFFCCF8091C000806480937C
:10FBA000C00065E1C15DDE4FE880CF52D1406E25D7
:10FBB00069276427FE01319610C090819093C6009A
:10FBC0008091C00086FFFCCF31968091C000806498
:10FBD0008093C0006927215030402115310569F715
:10FBE0006093C6008091C00086FFFCCF8091C0006A
:10FBF00080648093C00085B1805885B9772081F4F6
:10FC0000C15DDE4F0881CF52D1400F5FC15DDE4F35
:10FC10000883CF52D14090E0A0E0B0E00D941AF4F8
:10FC200027982F9880E090E020ED37E0F901319798
:10FC3000F1F7019684369105C9F700008091C00064
:10FC40008D7F8093C00081E180935700E895EE2777
:10FC5000FF270994FFCF90E00D941AF497FB092E2B
:10FC600007260AD077FD04D02ED006D000201AF443
:10FC7000709561957F4F0895F6F7909581959F4F08
:10FC80000895A1E21A2EAA1BBB1BFD010DC0AA1FDD
:10FC9000BB1FEE1FFF1FA217B307E407F50720F0F5
:10FCA000A21BB30BE40BF50B661F771F881F991F70
:10FCB0001A9469F760957095809590959B01AC01B9
:10FCC000BD01CF010895AA1BBB1B51E107C0AA1FAC
:10FCD000BB1FA617B70710F0A61BB70B881F991FED
:10FCE0005A95A9F780959095BC01CD010895F99991
:10FCF000FECF92BD81BDF89A992780B50895262F31
:10FD0000F999FECF1FBA92BD81BD20BD0FB6F89400
:0EFD1000FA9AF99A0FBE01960895F894FFCF63
:040000033000E000E9
:00000001FF
